S01C00005354345F537065637472756D5F576F726B696E672E737265633B
S3150800800000000220ED0B05083D0C05083D0C05088F
S315080080103D0C05083D0C05083D0C05080000000050
S315080080200000000000000000000000003D0C0508EC
S315080080303D0C0508000000003D0C05084D0105082B
S315080080403D0C05083D0C05083D0C05083D0C0508CA
S315080080503D0C05083D0C05083D0C05083D0C0508BA
S315080080603D0C05083D0C05083D0C05083D0C0508AA
S315080080703D0C05083D0C05083D0C05083D0C05089A
S31508008080590105086D0105083D0C05083D0C050854
S315080080903D0C05083D0C05083D0C05087102050850
S315080080A03D0C05083D0C05083D0C05083D0C05086A
S315080080B081010508950105083D0C05083D0C0508D4
S315080080C03D0C05083D0C05083D0C05083D0C05084A
S315080080D03D0C0508A9010508BD0105083D0C050864
S315080080E0A50205083D0C05083D0C05083D0C0508CC
S315080080F03D0C05083D0C05083D0C0508D101050891
S315080081003D0C0508E50105083D0C0508F9010508BB
S315080081103D0C05083D0C05083D0C05083D0C0508F9
S315080081203D0C05083D0C05080D0205082102050849
S315080081303D0C050800000000000000003D0C050885
S315080081403D0C05083D0C05083D0C050835020508DB
S315080081503D0C0508490205085D0205083D0C0508A1
S315080081603D0C05083D0C05083D0C05083D0C0508A9
S315080081703D0C05083D0C05083D0C050800000000EF
S31508008180000000003D0C050800000000000000008B
S315080081903D0C050800000000000000003D0C050825
S315080081A00000000000000000000000003D0C05086B
S315080081B03D0C05083D0C05083D0C05083D0C050859
S30D080081C03D0C050844332211A9
S315080081D010B5054C237833B9044B13B10448AFF3F3
S315080081E000800123237010BDE80F00200000000066
S315080081F0A483060808B5034B1BB103490348AFF32C
S31508008200008008BD00000000EC0F0020A4830608CB
S3150800821010F8012B11F8013B012A28BF9A42F7D022
S31508008220D01A7047034613F8012B002AFBD1181AF7
S315080082300138704700000000000000000000000040
S3150800824001F0FF01102A2BDB10F0070F08D010F8F9
S31508008250013B013A8B422DD010F0070F42B3F6D1FD
S31508008260F0B441EA012141EA014122F007047FF016
S3150800827000070023F0E80256083C85EA010586EA6D
S31508008280010685FA47F5A3FA87F586FA47F6A5FAA9
S3150800829087F68EB9EED1F0BC01F0FF0102F00702B5
S315080082A032B110F8013B013A83EA010313B1F8D160
S315080082B00020704701387047002D06BF3546033841
S315080082C0073815F0010F07D1013015F4807F02BF7A
S315080082D0013015F4C03F0130F0BC0138704700BFCB
S315080082E081F0004102E000BF83F0004330B54FEA59
S315080082F041044FEA430594EA050F08BF90EA020FC6
S315080083001FBF54EA000C55EA020C7FEA645C7FEA58
S31508008310655C00F0E2804FEA5454D4EB5555B8BF7B
S315080083206D420CDD2C4480EA020281EA030382EAEC
S31508008330000083EA010180EA020281EA0303362D7E
S3150800834088BF30BD11F0004F4FEA01314FF4801C51
S315080083504CEA113102D0404261EB410113F0004F63
S315080083604FEA03334CEA133302D0524263EB43031A
S3150800837094EA050F00F0A780A4F10104D5F1200EB8
S315080083800DDB02FA0EFC22FA05F2801841F1000113
S3150800839003FA0EF2801843FA05F359410EE0A5F1E7
S315080083A020050EF1200E012A03FA0EFC28BF4CF018
S315080083B0020C43FA05F3C01851EBE37101F00045CE
S315080083C007D54FF0000EDCF1000C7EEB00006EEBDB
S315080083D00101B1F5801F1BD3B1F5001F0CD3490865
S315080083E05FEA30004FEA3C0C04F101044FEA4452BC
S315080083F012F5800F80F09A80BCF1004F08BF5FEA43
S31508008400500C50F1000041EB045141EA050130BD22
S315080084105FEA4C0C404141EB0101013C28BFB1F534
S31508008420801FE9D291F0000F04BF01460020B1FA7F
S3150800843081F308BF2033A3F10B03B3F120020CDA52
S315080084400C3208DD02F1140CC2F10C0201FA0CF030
S3150800845021FA02F10CE002F11402D8BFC2F1200C95
S3150800846001FA02F120FA0CFCDCBF41EA0C0190404B
S31508008470E41AA2BF01EB0451294330BD6FEA040494
S315080084801F3C1CDA0C340EDC04F11404C4F120027F
S3150800849020FA04F001FA02F340EA030021FA04F391
S315080084A045EA030130BDC4F10C04C4F1200220FAE8
S315080084B002F001FA04F340EA0300294630BD21FA26
S315080084C004F0294630BD94F0000F83F4801306BFEC
S315080084D081F480110134013D4EE77FEA645C18BFE0
S315080084E07FEA655C29D094EA050F08BF90EA020F77
S315080084F005D054EA000C04BF1946104630BD91EA6F
S31508008500030F1EBF0021002030BD5FEA545C05D171
S315080085104000494128BF41F0004130BD14F58004B0
S315080085203CBF01F5801130BD01F0004545F0FE4124
S3150800853041F470014FF0000030BD7FEA645C1ABF59
S31508008540194610467FEA655C1CBF0B46024650EA90
S31508008550013406BF52EA033591EA030F41F40021BC
S3150800856030BD00BF90F0000F04BF0021704730B542
S315080085704FF4806404F132044FF000054FF0000117
S3150800858050E700BF90F0000F04BF0021704730B5D8
S315080085904FF4806404F1320410F0004548BF4042AD
S315080085A04FF000013EE700BF42004FEAE2014FEA02
S315080085B031014FEA02701FBF12F07F4393F07F4FDD
S315080085C081F06051704732F07F4208BF704793F0E0
S315080085D07F4F04BF41F40021704730B54FF46074F3
S315080085E001F0004521F000411CE700BF50EA0102F6
S315080085F008BF704730B54FF000050AE050EA01029F
S3150800860008BF704730B511F0004502D5404261EB0E
S3150800861041014FF4806404F132045FEA915C3FF44F
S31508008620D8AE4FF003025FEADC0C18BF03325FEAEC
S31508008630DC0C18BF033202EBDC02C2F1200300FA9D
S3150800864003FC20FA02F001FA03FE40EA0E0021FAC2
S3150800865002F11444BDE600BF70B54FF0FF0C4CF4B0
S31508008660E06C1CEA11541DBF1CEA135594EA0C0F62
S3150800867095EA0C0F00F0DEF82C4481EA030621EA9D
S315080086804C5123EA4C5350EA013518BF52EA0335D8
S3150800869041F4801143F4801338D0A0FB02CE4FF08A
S315080086A00005E1FB02E506F00042E0FB03E54FF0BA
S315080086B00006E1FB03569CF0000F18BF4EF0010EB2
S315080086C0A4F1FF04B6F5007F64F5407404D25FEAAE
S315080086D04E0E6D4146EB060642EAC62141EA555161
S315080086E04FEAC52040EA5E504FEACE2EB4F1FD0CA3
S315080086F088BFBCF5E06F1ED8BEF1004F08BF5FEA21
S31508008700500E50F1000041EB045170BD06F00046D2
S3150800871046EA010140EA020081EA0301B4EB5C047F
S31508008720C2BFD4EB0C0541EA045170BD41F4801177
S315080087304FF0000E013C00F3AB8014F1360FDEBF9C
S31508008740002001F0004170BDC4F10004203C35DA78
S315080087500C341BDC04F11404C4F1200500FA05F3FB
S3150800876020FA04F001FA05F240EA020001F000429C
S3150800877021F0004110EBD37021FA04F642EB060112
S315080087805EEA430E08BF20EAD37070BDC4F10C043C
S31508008790C4F1200500FA04F320FA05F001FA04F200
S315080087A040EA020001F0004110EBD37041F10001EC
S315080087B05EEA430E08BF20EAD37070BDC4F12005F7
S315080087C000FA05F24EEA020E20FA04F301FA05F25F
S315080087D043EA020321FA04F001F0004121FA04F207
S315080087E020EA020000EBD3705EEA430E08BF20EAD7
S315080087F0D37070BD94F0000F0FD101F00046400011
S3150800880041EB010111F4801F08BF013CF7D041EA92
S31508008810060195F0000F18BF704703F00046520096
S3150800882043EB030313F4801F08BF013DF7D043EA67
S315080088300603704794EA0C0F0CEA135518BF95EA1D
S315080088400C0F0CD050EA410618BF52EA4306D1D1A4
S3150800885081EA030101F000414FF0000070BD50EAC3
S31508008860410606BF1046194652EA430619D094EA4D
S315080088700C0F02D150EA013613D195EA0C0F05D137
S3150800888052EA03361CBF104619460AD181EA03018B
S3150800889001F0004141F0FE4141F470014FF0000043
S315080088A070BD41F0FE4141F4780170BD70B54FF0DE
S315080088B0FF0C4CF4E06C1CEA11541DBF1CEA13555E
S315080088C094EA0C0F95EA0C0F00F0A7F8A4EB050440
S315080088D081EA030E52EA03354FEA013100F0888037
S315080088E04FEA03334FF0805545EA131343EA126300
S315080088F04FEA022245EA111545EA10654FEA0026B5
S315080089000EF000419D4208BF964244F1FD0404F56D
S31508008910407402D25B084FEA3202B61A65EB0305C9
S315080089205B084FEA32024FF480104FF4002CB6EB86
S31508008930020E75EB030E22BFB61A754640EA0C0006
S315080089405B084FEA3202B6EB020E75EB030E22BF46
S31508008950B61A754640EA5C005B084FEA3202B6EB87
S31508008960020E75EB030E22BFB61A754640EA9C0046
S315080089705B084FEA3202B6EB020E75EB030E22BF16
S31508008980B61A754640EADC0055EA060E18D04FEAD4
S31508008990051545EA16754FEA06164FEAC30343EA74
S315080089A052734FEAC2025FEA1C1CC0D111F4801F41
S315080089B00BD141EA00014FF000004FF0004CB6E73A
S315080089C011F4801F04BF01430020B4F1FD0C88BFD9
S315080089D0BCF5E06F3FF6AFAEB5EB030C04BFB6EBE4
S315080089E0020C5FEA500C50F1000041EB045170BDD7
S315080089F00EF0004E4EEA113114EB5C04C2BFD4EB04
S31508008A000C0541EA045170BD41F480114FF0000E87
S31508008A10013C90E645EA060E8DE60CEA135594EA03
S31508008A200C0F08BF95EA0C0F3FF43BAF94EA0C0F06
S31508008A300AD150EA01347FF434AF95EA0C0F7FF47B
S31508008A4025AF104619462CE795EA0C0F06D152EACF
S31508008A5003353FF4FDAE1046194622E750EA4106B3
S31508008A6018BF52EA43067FF4C5AE50EA41047FF4C4
S31508008A700DAF52EA43057FF4EBAE12E74FF0FF3C29
S31508008A8006E000BF4FF0010C02E000BF4FF0010CFA
S31508008A904DF804CD4FEA410C7FEA6C5C4FEA430C73
S31508008AA018BF7FEA6C5C1BD001B050EA410C0CBFC2
S31508008AB052EA430C91EA030F02BF90EA020F002024
S31508008AC0704710F1000F91EA030F58BF994208BF8B
S31508008AD090422CBFD8176FEAE37040F00100704748
S31508008AE04FEA410C7FEA6C5C02D150EA013C07D19F
S31508008AF04FEA430C7FEA6C5CD6D152EA033CD3D0EA
S31508008B005DF8040B704700BF8446104662468C46E3
S31508008B101946634600E000BF01B5FFF7B7FF002816
S31508008B2048BF10F1000F01BD4DF808EDFFF7F4FF3F
S31508008B300CBF012000205DF808FB00BF4DF808EDCA
S31508008B40FFF7EAFF34BF012000205DF808FB00BFED
S31508008B504DF808EDFFF7E0FF94BF012000205DF80F
S31508008B6008FB00BF4DF808EDFFF7CEFF94BF0120C4
S31508008B7000205DF808FB00BF4DF808EDFFF7C4FFBD
S31508008B8034BF012000205DF808FB00BF4FEA410C06
S31508008B907FEA6C5C02D150EA013C0AD14FEA430CE9
S31508008BA07FEA6C5C02D152EA033C02D14FF0000026
S31508008BB070474FF0010070474FEA410212F5001264
S31508008BC015D211D56FF47873B3EB625212D94FEA06
S31508008BD0C12343F0004343EA505311F0004F23FAF0
S31508008BE002F018BF404270474FF00000704750EA45
S31508008BF0013005D111F0004008BF6FF00040704702
S31508008C004FF00000704700BF4A0011D212F500125B
S31508008C1011D20DD56FF47873B3EB62520ED44FEAC6
S31508008C20C12343F0004343EA505323FA02F0704746
S31508008C304FF00000704750EA013002D14FF0FF3084
S31508008C4070474FF0000070474FEA4102B2F1E04327
S31508008C5024BFB3F5001CDCF1FE5C0DD901F0004C15
S31508008C604FEAC0024CEA5070B2F1004F40EB830065
S31508008C7008BF20F00100704711F0804F21D113F191
S31508008C803872BCBF01F00040704741F480114FEACA
S31508008C905252C2F11802C2F1200C10FA0CF320FA53
S31508008CA002F018BF40F001004FEAC1234FEAD32370
S31508008CB003FA0CFC40EA0C0023FA02F34FEA4303DA
S31508008CC0CCE77FEA625307D150EA01331EBF4FF063
S31508008CD0FE4040F44000704701F0004040F0FE407E
S31508008CE040F40000704700BF53B94AB9002908BFCD
S31508008CF000281CBF4FF0FF314FF0FF3000F0A4B939
S31508008D00ADF1080C6DE904CE00F03CF8DDF804E09E
S31508008D10DDE9022304B0704738B500220023044673
S31508008D200D46FFF70BFF28B920462946BDE838400F
S31508008D3000F00AB8204605F1004100F005F8404267
S31508008D4061EB410138BD00BFD0B50C4B0022064689
S31508008D500F46FFF781FCFFF757FF0446FFF702FCB3
S31508008D60074B0022FFF778FC02460B463046394689
S31508008D70FFF7BAFAFFF748FF2146D0BD0000F03DDD
S31508008D800000F0412DE9F047089D04468C46002B6B
S31508008D9040F083808A42174647D9B2FA82F242B136
S31508008DA0C2F1200024FA00F09140974040EA010CF5
S31508008DB094404FEA1748230CBCFBF8F61FFA87FEC7
S31508008DC008FB16C143EA014306FB0EF1994209D98D
S31508008DD0FB1806F1FF3080F01981994240F216819E
S31508008DE0023E3B445B1AA4B2B3FBF8F008FB10330F
S31508008DF044EA034400FB0EFEA64509D93C1900F1D6
S31508008E00FF3380F00581A64540F2028102383C44D2
S31508008E1040EA0640A4EB0E0400261DB1D440002308
S31508008E20C5E900433146BDE8F08702B9FFDEB2FA6C
S31508008E3082F2002A50D1CB1B4FEA174E1FFA87F849
S31508008E400126B3FBFEFC210C0EFB1C3341EA034151
S31508008E5008FB0CF38B4207D979180CF1FF3002D2C4
S31508008E608B4200F2E9808446C91AA3B2B1FBFEF030
S31508008E700EFB101143EA014408FB00F8A04507D988
S31508008E803C1900F1FF3302D2A04500F2D9801846FA
S31508008E90A4EB080440EA0C40BFE78B4209D9002D31
S31508008EA000F0B1800026C5E9000130463146BDE82C
S31508008EB0F087B3FA83F6002E4AD18B4202D3824258
S31508008EC000F2B880841A61EB030101208C46002D5C
S31508008ED0A8D0C5E9004CA5E7C2F1200320FA03F69D
S31508008EE0974001FA02F04FEA174ED9403043030C77
S31508008EF0B1FBFEF61FFA87F80EFB161143EA01438B
S31508008F0006FB08F1994204FA02F409D9FB1806F19E
S31508008F10FF3C80F08D80994240F28A80023E3B44B5
S31508008F205B1A81B2B3FBFEF00EFB103341EA034134
S31508008F3000FB08F38B4207D9791800F1FF3C73D27E
S31508008F408B4271D902383944CB1A40EA064678E78B
S31508008F50C6F1200C03FA06F422FA0CF31C4320FA95
S31508008F600CF701FA06F34FEA144E21FA0CF11F43E7
S31508008F703B0CB1FBFEF91FFA84F80EFB191143EA04
S31508008F80014109FB08FA8A4502FA06F200FA06F3D5
S31508008F9008D9611809F1FF3048D28A4546D9A9F19E
S31508008FA002092144A1EB0A01BFB2B1FBFEF00EFB98
S31508008FB0101147EA014700FB08F8B84507D9E71931
S31508008FC000F1FF312ED2B8452CD90238274440EAA1
S31508008FD00940A7EB0807A0FB02894F45C646494644
S31508008FE01AD317D05DB1B3EB0E0267EB010707FA88
S31508008FF00CFCF2404CEA0202F740C5E900270026BD
S315080090003146BDE8F0872E4628460BE70646E9E6D0
S315080090101846FDE64345E5D2B8EB020E69EB0401B6
S315080090200138DFE70846D2E760468DE78146B9E7AB
S31508009030664675E730464AE7ACF1020C394413E751
S3150800904002383C4424E700BF704700BF80B483B0B1
S3150800905000AF78607B689B6818460C37BD465DF89C
S31508009060047B704780B483B000AF78607B681B6868
S3150800907018460C37BD465DF8047B704790B583B03B
S3150800908000AF786039603B68002B01D100230DE002
S315080090907B681B6804331C683868FFF7C3F8034607
S315080090A01A4639687868A047034600BF18460C3741
S315080090B0BD4690BD80B586B000AFF860B9607A60ED
S315080090C000237B617B685A1E7A60002B14BF01233C
S315080090D00023DBB2002B0ED0FB681B681A68BB683E
S315080090E0591CB9601B781946F868904702467B698F
S315080090F013447B61E6E77B6918461837BD4680BD91
S3150800910080B582B000AF7860396039687868FFF753
S31508009110B5FF034618460837BD4680BD80B582B000
S3150800912000AF786004497868FFF7A8FF0346184639
S315080091300837BD4680BD00BFC083060880B584B029
S3150800914000AF7860396039687868FFF7D9FFF8604A
S315080091507868FFF7E3FF0246FB681344FB60FB6889
S3150800916018461037BD4680BD80B582B000AF78601E
S315080091700B46FB707B681B6804331B68F91C0122CD
S3150800918078689847034618460837BD4680BD80B5B7
S3150800919086B000AFF860B9607A60BB687B61FB682F
S315080091A018697B689AB24FF0FF3379694FF0E2FE8F
S315080091B07B6818461837BD4680BD80B584B000AFB9
S315080091C078607B68186907F10F014FF0FF330122B9
S315080091D04FF062FFFB7B18461037BD4680BD80B452
S315080091E083B000AF78604FF0FF3318460C37BD46A2
S315080091F05DF8047B704780B483B000AF78604FF0A9
S31508009200FF3318460C37BD465DF8047B704780B4BB
S3150800921083B000AF786000BF0C37BD465DF8047BAD
S31508009220704780B582B000AF78600B46FB70FB785C
S315080092301946786800F0A6F97B6818460837BD46CF
S3150800924080BD80B582B000AF78603960786800F07C
S3150800925041F83B68002B08D03868FEF7E3FF034661
S315080092601A463968786800F0ACF87B6818460837FB
S31508009270BD4680BD80B582B000AF78603960786839
S3150800928000F028F83968786800F0FCF87B6818461A
S315080092900837BD4680BD80B582B000AF78603960BA
S315080092A0786800F017F83968786800F0AFF87B68D6
S315080092B018460837BD4680BD80B582B000AF7860D5
S315080092C07B681B6818465AF0A1FD7B681846083764
S315080092D0BD4680BD80B483B000AF78607B6800224D
S315080092E01A607B6800225A607B6800229A6000BF79
S315080092F00C37BD465DF8047B704780B582B000AF79
S3150800930078607B681B68002B04D07B681B6818464E
S315080093105AF07CFD7B6800221A607B6800229A60FE
S315080093207B689A687B685A6000BF0837BD4680BD6F
S3150800933080B582B000AF786039607B681B68002B07
S3150800934006D07B685B683A689A4201D8012316E022
S315080093503968786800F017F80346002B14BF012314
S315080093600023DBB2002B09D07B689B68002B03D156
S315080093707B681B6800221A70012300E00023184648
S315080093800837BD4680BD80B584B000AF78603960C7
S315080093907B681A683B680133194610465BF09AFAEF
S315080093A0F860FB68002B07D07B68FA681A607B6850
S315080093B03A685A60012300E0002318461037BD4674
S315080093C080BD80B584B000AFF860B9607A6079680E
S315080093D0F868FFF7ADFF0346002B0CBF01230023F7
S315080093E0DBB2002B04D0F868FFF787FFFB6809E0BB
S315080093F0FB687A689A60FB681B68B96818465BF070
S3150800940035FBFB6818461037BD4680BD80B582B06F
S3150800941000AF786039607B681B68002B1AD07B68C0
S315080094205A683B689B689A420FD37B681A683B6800
S315080094301B68194610465BF019FB3B689A687B68FF
S315080094409A603B6800229A6019E07B681B68184698
S315080094505AF0DCFC3B681A687B681A603B685A68F5
S315080094607B685A603B689A687B689A603B6800220A
S315080094701A603B6800225A603B6800229A600837E7
S31508009480BD4680BD80B582B000AF786039607A6825
S315080094903B689A4201D17B6810E03B681B68002B49
S315080094A008D03B6819683B689B681A467868FFF7D6
S315080094B088FF02E07868FFF720FF7B6818460837C0
S315080094C0BD4680BD80B582B000AF786039607A68E5
S315080094D03B689A4203D039687868FFF797FF7B683C
S315080094E018460837BD4680BD80B582B000AF7860A3
S315080094F039603B68002B09D03868FEF793FE0346AF
S315080095001A4639687868FFF75CFF02E07868FFF763
S31508009510F4FE7B6818460837BD4680BD80B586B020
S3150800952000AFF860B9607A60FB689B687A68134494
S315080095307B61BB68002B01D100231FE07B68002BF1
S3150800954001D101231AE07969F868FFF7F1FE0346AD
S31508009550002B0CBF01230023DBB2002B01D0002314
S315080095600CE0FB681A68FB689B681344B9681846E0
S315080095705BF07CFAFB687A699A600123184618370B
S31508009580BD4680BD80B584B000AF78600B46FB70E1
S31508009590FB783B7300237B7307F10C030122194602
S315080095A07868FFF7BBFF034618461037BD4680BDEF
S315080095B080B582B000AF786039607B689B68002B05
S315080095C00AD13B68002B03D03B681B78002B01D1DE
S315080095D0012300E0002317E03B68002B08D17B68D5
S315080095E01B681B78002B0CBF01230023DBB20BE0A2
S315080095F07B681B6839681846FEF70AFE0346002B87
S315080096000CBF01230023DBB218460837BD4680BDD0
S3150800961080B483B000AF786039607B689B683A682D
S315080096209A4203D27B681B68002B04D1074B0022A1
S315080096301A70064B03E07B681A683B6813441846A1
S315080096400C37BD465DF8047B704700BF0410002048
S3150800965080B586B000AFF8600B467A60FB72FB688F
S315080096609B687A689A4202D34FF0FF3313E0FB688F
S315080096701A687B681344FA7A114618465BF0E9F9CA
S3150800968078617B69002B02D14FF0FF3303E0FB685A
S315080096901B687A69D31A18461837BD4680BD00007C
S315080096A080B586B000AFF860B9607A603B607A68CA
S315080096B03B689A4205D93B687B617B683B607B695E
S315080096C07B601849F868FFF7BCFDBB689B687A6839
S315080096D09A4222D2BB689B683A689A4202D9BB680A
S315080096E09B683B60BB681A683B6813441B78FB742D
S315080096F0BB681A683B68134400221A70BB681A686C
S315080097007B6813441946F868FFF7EEFEBB681A68CB
S315080097103B681344FA7C1A7000E000BFF8681837F3
S31508009720BD4680BDD483060880B582B000AF786098
S315080097307B681B68002B06D07B681B6818465AF0A6
S315080097402EFB034600E0002318460837BD4680BDB9
S3150800975080B588B004AF03463960FB801346BB80EA
S31508009760FA88BB88134440F2FE32934201DD002397
S3150800977019E0FB88184600F048F90346FB73FB8896
S31508009780BB73FB7B99B2BB7B9AB20E230293BB8851
S3150800979001933B6800930123054849F02DFA0420FC
S315080097A047F0C0FA012318461037BD4680BD00BFF2
S315080097B0DCC2012080B588B004AF03463960FB805F
S315080097C01346BB803B68FB60FA88BB88134440F2AB
S315080097D0FE32934201DD002319E0FB88184600F0AB
S315080097E014F90346FB72FB88BB72FB7A99B2BB7A03
S315080097F09AB20E230293BB880193FB680093012358
S31508009800054849F0F9F9042047F08CFA012318466F
S315080098101037BD4680BD00BFDCC2012080B588B0C8
S3150800982004AF03463960FB801346BB803B681B8840
S315080098301B12DBB23B733B681B88DBB27B73FA886F
S31508009840BB88134440F2FE32934201DD00231AE03E
S31508009850FB88184600F0D9F80346FB73FB88BB73F0
S31508009860FB7B99B2BB7B9AB20E230293BB8801930A
S3150800987007F10C0300930123054849F0BDF90420BC
S3150800988047F050FA012318461037BD4680BD00BF81
S31508009890DCC2012080B588B004AF03463960FB807E
S315080098A01346BB80FA88BB88134440F2FE329342C3
S315080098B001DD002316E0FB88184600F083F803460E
S315080098C0FB73FB88BB73FB7B99B2BB7B9AB20E23F7
S315080098D00293BB8801933B6800930123034849F030
S315080098E085FA012318461037BD4680BDDCC2012023
S315080098F080B588B004AF03463960FB801346BB8049
S31508009900FA88BB88134440F2FE32934201DD0023F5
S3150800991022E0FB88184600F055F80346FB73FB88DF
S31508009920BB73FB7B99B2BB7B9AB20E230293BB88AF
S31508009930019307F1080300930123094849F056FAF1
S315080099403B7A1B021AB27B7A1BB213431BB2BB814A
S315080099503B68BA891A80012318461037BD4680BD70
S31508009960DCC2012080B588B004AF03463960FB80AD
S315080099701346BB803B68FB60FA88BB88134440F2F9
S31508009980FE32934201DD002316E0FB88184600F0FC
S3150800999019F80346FB72FB88BB72FB7A99B2BB7A4D
S315080099A09AB20E230293BB880193FB6800930123A6
S315080099B0034849F01BFA012318461037BD4680BDF7
S315080099C0DCC2012080B483B000AF0346FB80FB886D
S315080099D0FF2B01D8A12312E0FB88B3F5007F01D243
S315080099E0A3230CE0FB88B3F5407F01D2A52306E04C
S315080099F0FB88B3F5806F01D2A72300E0A72318469A
S31508009A000C37BD465DF8047B704780B483B000AF61
S31508009A100346FB80FB88FF2B01D8A02312E0FB88B6
S31508009A20B3F5007F01D2A2230CE0FB88B3F5407F93
S31508009A3001D2A42306E0FB88B3F5806F01D2A623E2
S31508009A4000E0A62318460C37BD465DF8047B704730
S31508009A5080B584B000AF78600B46FB70FB7819467A
S31508009A60786800F04DFA0346FB73FB7B002B03D1A5
S31508009A70786800F029F81BE0FB7B012B17D0FB7BED
S31508009A80052B04D10C490D48FFF758FB10E0FB7B6A
S31508009A90022B04D10A490948FFF750FB08E0FB7B73
S31508009AA0032B05D107490548FFF748FB00E000BF2F
S31508009AB01037BD4680BD00BFD8830608FC4201208A
S31508009AC0E8830608F483060880B582B000AF78609C
S31508009AD0786800F019F97B6803F5197319467868F0
S31508009AE000F0B4FA02467B68DA637B68DA6B7B6857
S31508009AF0D3F850321A447B681A607B6803F51A73E8
S31508009B001946786800F0A2FA02467B681A647B68F0
S31508009B101A6C7B68D3F854321A447B685A607B689F
S31508009B2003F51B731946786800F090FA02467B68BD
S31508009B305A647B685A6C7B68D3F858321A447B6837
S31508009B409A607B6803F51C731946786800F07EFAFC
S31508009B5002467B68DA607B6803F51D7319467868E8
S31508009B6000F074FA02467B681A617B6803F51E7377
S31508009B701946786800F054FA03461A467B681A8331
S31508009B807B6803F27A231946786800F049FA034697
S31508009B901A467B685A837B6803F51F7319467868EB
S31508009BA000F03EFA03461A467B689A837B6893F868
S31508009BB07E227B6883F824207B6893F87F227B6863
S31508009BC083F825207B6893F880227B6883F8262013
S31508009BD07B6893F881227B6883F827207B6893F853
S31508009BE082227B6883F82E207B6893F883227B6821
S31508009BF083F82F207B6893F884227B6883F83020CB
S31508009C007B6893F885227B6883F831207B6893F814
S31508009C1086227B6883F832207B6893F887227B68E4
S31508009C2083F833207B6893F888227B6883F834208E
S31508009C307B6893F889227B6883F835207B6893F8DC
S31508009C408A227B6883F836207B6893F88B227B68A8
S31508009C5083F837207B6893F88C227B6883F8382052
S31508009C607B6893F88D227B6883F839207B6893F8A4
S31508009C708E227B6883F83A207B6893F88F227B686C
S31508009C8083F83B207B6803F523731946786800F050
S31508009C90DDF902467B685A617B6803F52473194629
S31508009CA0786800F0BDF903461A467B689A857B6892
S31508009CB093F892227B6883F848207B6893F893226E
S31508009CC07B6883F849207B6893F89432A3F1800275
S31508009CD07B681A627B6893F89532803B07EE903A68
S31508009CE0B8EEE77AF2EE046AC7EE267A7B68C3ED29
S31508009CF00A7A786800F019F87B68012283F85C22F2
S31508009D0000BF0837BD4680BD80B582B000AF786019
S31508009D107B687A6803F5FC7311464C2218465AF09C
S31508009D207DF800BF0837BD4680BD80B582B000AF5C
S31508009D3078607B689B8D002B3AD07B68B3F8242229
S31508009D407B689B8D9A4210D07B689A8D7B68A3F8B6
S31508009D50F4217B68D3F8F8117B68D3F8FC217B687B
S31508009D60D3F80032786800F027F87B6893F8482023
S31508009D707B6893F877309A4204D17B68012283F88E
S31508009D804A2003E07B68002283F84A207B6893F820
S31508009D9049207B6893F897309A4204D17B68012260
S31508009DA083F84B2005E07B68002283F84B2000E00F
S31508009DB000BF0837BD4680BD80B485B000AFF860E7
S31508009DC0B9607A603B60FB68DB6BBA68D21AFB68DD
S31508009DD0C3F85022FB681B6C7A68D21AFB68C3F872
S31508009DE05422FB685B6C3A68D21AFB68C3F858229F
S31508009DF000BF1437BD465DF8047B704780B485B054
S31508009E0000AFF860B9607A603B60FB68DB7B0133C2
S31508009E10DAB2FB68DA73FB68DB7B002B02D1FB68DE
S31508009E200122DA73FB68BA681A61FB687A685A61B4
S31508009E30FB683A689A61BB699AB2FB689A8300BF65
S31508009E401437BD465DF8047B7047000080B582B0C4
S31508009E5000AF78607B6893F85C32002B16D07B687D
S31508009E60002283F85C227B68012283F818210A4BBA
S31508009E701B7883F00103DBB2002B05D0786800F06D
S31508009E8027F8054B01221A70012300E00023184623
S31508009E900837BD4680BD00BF0510002080B483B0DA
S31508009EA000AF78607B689A8D084B1B889A4205D06C
S31508009EB07B689A8D054B1A80012300E0002318461B
S31508009EC00C37BD465DF8047B704700BF06100020BE
S31508009ED080B582B000AF78600121786800F000FB99
S31508009EE00221786800F0FCFA0321786800F0F8FA95
S31508009EF00421786800F0F4FA00BF0837BD4680BD33
S31508009F0080B592B000AF78600B46FB7001237B6486
S31508009F107B6C3C2B10DC7B6C013B79687A6C0A44C1
S31508009F2002F25D2211787A6813440A4683F85D22A4
S31508009F307B6C01337B64EBE77B68FA7883F89922BC
S31508009F407B6893F85D32492B01D0012364E07B6876
S31508009F5093F85E32572B01D001235DE07B6893F8B6
S31508009F605F32412B01D0012356E07B6893F86032BB
S31508009F70502B01D001234FE07B6893F86132492BBF
S31508009F8001D0012348E07B6893F86232022B01D0A6
S31508009F90052341E07B6893F897323B2B01D00223D7
S31508009FA03AE07B6893F89832212B01D0022333E0FC
S31508009FB07B6893F899323B2B01D002232CE00023CF
S31508009FC03B643B6C332B0FDC3B6C05337A681344DC
S31508009FD093F85D1207F108023B6C13440A461A709F
S31508009FE03B6C01333B64ECE77B6893F8963287F861
S31508009FF03F3007F1080334221946786800F0C4FA9E
S3150800A000034687F83E3097F83F2097F83E309A4245
S3150800A01001D0032300E0002318464837BD4680BD1B
S3150800A02080B483B000AF786039603B681B781B0248
S3150800A0301AB23B6801331B781BB253401BB29BB262
S3150800A04018460C37BD465DF8047B704780B483B06C
S3150800A05000AF786039603B681B781A063B680133A5
S3150800A0601B781B045A403B6802331B781B0253407B
S3150800A0703A6803321278534018460C37BD465DF8E5
S3150800A080047B704780B5BCB002AF78600023C7F880
S3150800A090E0307B6803F219117B6803F24522D7F892
S3150800A0A0E03000930523786800F004FAC7F8E0006A
S3150800A0B07B6803F219117B6803F51172D7F8E03053
S3150800A0C000930123786800F0F5F9C7F8E0007B688B
S3150800A0D003F219117B6803F5FA72D7F8E03000939A
S3150800A0E00223786800F0E6F9C7F8E0007B6803F217
S3150800A0F019117A68D7F8E03000930423786800F0DD
S3150800A100D9F9C7F8E0007B6803F219117B681A1DB4
S3150800A110D7F8E03000930423786800F0CBF9C7F845
S3150800A120E0007B6803F219117B6803F10802D7F88F
S3150800A130E03000930423786800F0BCF9C7F8E00023
S3150800A1407B6803F219117B6803F14C02D7F8E030FB
S3150800A15000930923786800F0ADF9C7F8E0007B683A
S3150800A16003F219117B6803F16402D7F8E030009313
S3150800A1700123786800F09EF9C7F8E0007B6803F2CF
S3150800A18019117B6803F15502D7F8E03000930F23C5
S3150800A190786800F08FF9C7F8E0007B6803F21911B8
S3150800A1A07B6803F16802D7F8E03000930F237868DC
S3150800A1B000F080F9C7F8E0007B6803F219117B68A4
S3150800A1C003F17802D7F8E03000930423786800F0AA
S3150800A1D071F9C7F8E0007B6803F219117B6803F18F
S3150800A1E07C02D7F8E03000930423786800F062F91F
S3150800A1F0C7F8E0007B6803F219117B6803F1800257
S3150800A200D7F8E03000930423786800F053F9C7F8CC
S3150800A210E0007B6803F219117B6803F18402D7F822
S3150800A220E03000930223786800F044F9C7F8E000AC
S3150800A2307B6803F219117B6803F17702D7F8E030DF
S3150800A24000930123786800F035F9C7F8E0007B68C9
S3150800A25003F219117B6803F18802D7F8E0300093FE
S3150800A2600F23786800F026F9C7F8E0007B6803F248
S3150800A27019117B6803F19802D7F8E030009304239C
S3150800A280786800F017F9C7F8E0007B6803F219113F
S3150800A2907B6803F19C02D7F8E030009304237868C2
S3150800A2A000F008F9C7F8E0007B6803F219117B682B
S3150800A2B003F1A002D7F8E03000930423786800F091
S3150800A2C0F9F8C7F8E0007B6803F219117B6803F117
S3150800A2D0A402D7F8E03000930223786800F0EAF881
S3150800A2E0C7F8E0007B6803F219117B6803F197024F
S3150800A2F0D7F8E03000930123786800F0DBF8C7F858
S3150800A300E0007B6803F219117B6803F1A802D7F80D
S3150800A310E03000930F23786800F0CCF8C7F8E00027
S3150800A3207B6803F219117B6803F1B702D7F8E030AE
S3150800A33000930F23786800F0BDF8C7F8E0007B6843
S3150800A34003F219117B6803F1C602D7F8E0300093CF
S3150800A3500F23786800F0AEF8C7F8E0007B6803F2D0
S3150800A36019117B6803F1D502D7F8E03000930F2363
S3150800A370786800F09FF8C7F8E0007B6803F21911C7
S3150800A3807B6803F1E402D7F8E03000930F2378687E
S3150800A39000F090F8C7F8E0007B6803F219117B68B3
S3150800A3A003F1F302D7F8E03000930F23786800F042
S3150800A3B081F8C7F8E0007B6803F219117B6803F59A
S3150800A3C08272D7F8E03000930423786800F072F8B8
S3150800A3D0C7F8E0007B6803F219117B6803F58472FD
S3150800A3E0D7F8E03000930423786800F063F8C7F8DC
S3150800A3F0E0007B6803F219117B6803F58672D7F8CB
S3150800A400E03000930423786800F054F8C7F8E000B9
S3150800A4107B6803F219117B6803F58872D7F8E03078
S3150800A42000930823786800F045F8C7F8E000002391
S3150800A430C7F8E430D7F8E430D12B13DCD7F8E4308A
S3150800A44005337A68134493F8191107F10C02D7F803
S3150800A450E43013440A461A70D7F8E4300133C7F8D3
S3150800A460E430E7E707F10C03D2221946786800F0D2
S3150800A4708BF80346FB727B6803F2191107F10B028E
S3150800A480D7F8E03000930123786800F013F8C7F88E
S3150800A490E0007B6803F219117B6803F24A22D7F8B9
S3150800A4A0E03000930323786800F004F800BFE8372B
S3150800A4B0BD4680BD80B584B000AFF860B9607A60EB
S3150800A4C03B60BB69BA6813443A687968184659F01C
S3150800A4D0A5FCBA693B68134418461037BD4680BDCB
S3150800A4E080B483B000AF78600B46FB70FB78012B15
S3150800A4F00DD17B6893F82E20224B5B789A4239D08F
S3150800A5007B6893F82E201F4B5A70012333E0FB78A3
S3150800A510022B0DD17B6893F82F201A4B9B789A4211
S3150800A52028D07B6893F82F20164B9A70012322E0D7
S3150800A530FB78032B0DD17B6893F83020114BDB7821
S3150800A5409A4217D07B6893F830200E4BDA700123B5
S3150800A55011E0FB78042B0DD17B6893F83120094B69
S3150800A5601B799A4206D07B6893F83120054B1A71FD
S3150800A570012300E0002318460C37BD465DF8047B2E
S3150800A580704700BF0810002080B487B000AFF8609D
S3150800A590B9607A600023FB7400237B617A697B6863
S3150800A5A09A420ADABB685A1CBA601A78FB7C1344CA
S3150800A5B0FB747B6901337B61F0E7FB7C18461C372B
S3150800A5C0BD465DF8047B704780B483B000AF786001
S3150800A5D000BF0C37BD465DF8047B704780B483B076
S3150800A5E000AF786039603B681B68002B06D17B6832
S3150800A5F000221A607B6800225A6005E07B68054ADB
S3150800A6001A607B6800225A6078680C37BD465DF888
S3150800A610047B7047C9A5000880B483B000AF786092
S3150800A620002318460C37BD465DF8047B704780B496
S3150800A63083B000AF7860002318460C37BD465DF836
S3150800A640047B704780B485B000AFF860B9601346E4
S3150800A650FB7100BF1437BD465DF8047B704780B4B4
S3150800A66083B000AF786000BF0C37BD465DF8047B49
S3150800A670704780B483B000AF7860002318460C3763
S3150800A680BD465DF8047B7047B0B588B002AFF86088
S3150800A6907A603B600B46FB72F868F97A02230093EE
S3150800A6A0FB6A7A6801F0BAFB224AFB681A60FB6803
S3150800A6B01C3300221A605A601A81FB68303303245F
S3150800A6C01D46002C06DB1C492846FEF7BAFD0C354C
S3150800A6D0013CF6E73B68002B1ED000237B617B69B3
S3150800A6E0032B16DC7A6913465B0013449B00303350
S3150800A6F0FA68D0187A6913465B0013449B001A4619
S3150800A7003B6813441946FEF7BDFE7B6901337B613E
S3150800A710E5E7FB683A6B9A62BB6A002B02D0FB68D6
S3150800A720BA6ADA62FB680122DA71FB6818461837DA
S3150800A730BD46B0BD2CB406080484060890B585B09D
S3150800A74000AF78600B46FB707B68184601F042FC48
S3150800A7507B6830331846FEF779FC0346002B0CBF9E
S3150800A76001230023DBB2002B32D07A687B681B7C7E
S3150800A7701946104601F0AEFCFB78002B08D0544B66
S3150800A7801988544B1B789AB2534B54480DF0DBF892
S3150800A790534B1B881C467B689B6819464F480DF02F
S3150800A7A0DBF90346E31ADA0F13445B109AB2484BF7
S3150800A7B01B8813449AB2464B1A80454B1988454B59
S3150800A7C01B789AB27B689B6844480DF0BCF87BE01E
S3150800A7D07A687B681B7C013BDBB21946104601F0A0
S3150800A7E079FCFB78002B08D0394B1988394B1B7834
S3150800A7F09AB2394B39480DF0A6F87B689B681A4619
S3150800A800384939485AF0C2F8354B1B881C46364930
S3150800A81032480DF0A1F90346E31A9AB22C4B1B886D
S3150800A82013449AB22A4B1A80294B1988294B1B784C
S3150800A8309AB22D4B29480DF086F87B689B6A1B78DF
S3150800A8401A4613465B0013449B0030337A681A4451
S3150800A85007F1080311461846FFF7C0FEBB68002B30
S3150800A86006D1FB6803F00103002B01D1012300E0A8
S3150800A870002383F00103DBB2002B25D07A687B68BE
S3150800A8801B7C0133DBB21946104601F023FC7B68BA
S3150800A8909B6A1B781A4613465B0013449B003033A9
S3150800A8A07A6813441846FEF7DDFB03461A460F4935
S3150800A8B00D485AF06BF8064B1988064B1B789AB266
S3150800A8C0094B06480DF03FF800BF1437BD4690BD4A
S3150800A8D010100020121000200884060814C2012057
S3150800A8E00E1000200C840608141000201484060894
S3150800A8F080B483B000AF7860396000BF0C37BD46BE
S3150800A9005DF8047B704780B582B000AF78600B466F
S3150800A910FB707B68FA781146184601F0D3FA7B6813
S3150800A920DB6A18460837BD4680BD80B483B000AFE1
S3150800A9307860002318460C37BD465DF8047B7047DF
S3150800A94080B582B000AF786039607B681C3339689F
S3150800A95018465AF08BF800BF0837BD4680BD000080
S3150800A96090B583B000AF78600E4A7B681A607B6842
S3150800A9703033002B0CD07B68303303F130047B680E
S3150800A98030339C4204D00C3C2046FEF795FCF6E793
S3150800A9907B68184601F080FA7B6818460C37BD4676
S3150800A9A090BD00BF2CB4060880B582B000AF7860B1
S3150800A9B07868FFF7D5FF6021786858F03DF87B681E
S3150800A9C018460837BD4680BD80B483B000AF7860AE
S3150800A9D0396000BF0C37BD465DF8047B704780B40C
S3150800A9E083B000AF786039603B6818460C37BD46BF
S3150800A9F05DF8047B704780B582B000AF78607868F0
S3150800AA0000F010FD7B6818460837BD4680BD80B546
S3150800AA1082B000AF78607B68184600F0F3FC7B686C
S3150800AA2018460837BD4680BD80B582B000AF78604D
S3150800AA307B681846FFF7EBFF7B6818460837BD4664
S3150800AA4080BD000080B588B002AFF8607A603B60D0
S3150800AA500B46FB72F868F97A022300933B6A7A6818
S3150800AA6001F0DCF9434AFB681A60FB681C3342496B
S3150800AA701846FEF7E6FBFB682C333F491846FEF7F7
S3150800AA80E0FBFB683D4A3C3311469822184659F0CC
S3150800AA90C5F9FB68D4331846FFF7C6FFFB683A6862
S3150800AAA05A61FB68002283F82820FB682C33F96A70
S3150800AAB01846FEF7E7FCFB680422DA7100237B617F
S3150800AAC0FB685B691846FEF7C1FA02467B699A423B
S3150800AAD08CBF01230023DBB2002B2AD0FB685B69FD
S3150800AAE01846FEF7BFFA02467B6913441B7897F8A7
S3150800AAF024209A420CBF01230023DBB2002B0AD084
S3150800AB00FB68D4332522BA7407F112021146184697
S3150800AB1000F0C7FC09E0FB68D4332422FA7407F175
S3150800AB2013021146184600F0BCFC7B6901337B61B1
S3150800AB30C6E7FB685B691846FEF788FA0346DAB289
S3150800AB40FB681A76FB6803F11C02FB685B69194609
S3150800AB501046FEF797FCFB6897F8282083F8E02054
S3150800AB60FB6897F8242083F83820FB6818461837BE
S3150800AB70BD4680BD64B40608B0840608B4840608D9
S3150800AB8080B588B002AFF8607A603B600B46FB720E
S3150800AB90F868F97A97F8203000937B6A7A6801F0AA
S3150800ABA03DF9414AFB681A60FB681C333F49184661
S3150800ABB0FEF747FBFB682C333C491846FEF741FB7A
S3150800ABC0FB683B4A3C3311469822184659F026F949
S3150800ABD0FB68D4331846FFF727FFFB683A685A61C3
S3150800ABE0FB68002283F82820FB680422DA71002318
S3150800ABF07B61FB685B691846FEF728FA02467B69A3
S3150800AC009A428CBF01230023DBB2002B2AD0FB68B3
S3150800AC105B691846FEF726FA02467B6913441B78D9
S3150800AC2097F828209A420CBF01230023DBB2002B99
S3150800AC300AD0FB68D4332522BA7407F112021146EA
S3150800AC40184600F02EFC09E0FB68D4332422FA7477
S3150800AC5007F113021146184600F023FC7B690133FD
S3150800AC607B61C6E7FB685B691846FEF7EFF90346A2
S3150800AC70DAB2FB681A76FB6803F11C02FB685B69AB
S3150800AC8019461046FEF7FEFBFB6897F82C2083F85A
S3150800AC90E020FB6897F8282083F83820FB681846D8
S3150800ACA01837BD4680BD00BF64B40608B0840608E0
S3150800ACB0B484060880B582B000AF78600D4A7B6818
S3150800ACC01A607B68D433184600F0D0FB7B682C33B7
S3150800ACD01846FEF7F1FA7B681C331846FEF7ECFABD
S3150800ACE07B68184601F0D8F87B6818460837BD46D1
S3150800ACF080BD00BF64B4060880B582B000AF786036
S3150800AD007868FFF7D7FFE421786857F095FE7B68E7
S3150800AD1018460837BD4680BD80B582B000AF78605A
S3150800AD200B46FB707B68FA781146184601F0CAF89C
S3150800AD307B6893F8E030002B04D07B6893F8E0300A
S3150800AD40012B04D17B68002283F8392008E07B6850
S3150800AD5093F8E030022B03D17B681A2283F8392056
S3150800AD607B68002283F82820002318460837BD464A
S3150800AD7080BD80B483B000AF786000BF18460C373A
S3150800AD80BD465DF8047B7047B0B588B002AF786001
S3150800AD900B46FB707B68184601F01CF97A687B68DD
S3150800ADA01B7C1946104601F095F9FB78002B08D054
S3150800ADB0834B1988834B1B789AB2834B83480CF0D4
S3150800ADC0C2FD7B689B681A468149824859F0DEFDB8
S3150800ADD0814B1B881C467F497C480CF0BDFE034608
S3150800ADE0E31A9AB2764B1B8813449AB2744B1A80AC
S3150800ADF0734B1988734B1B789AB2764B73480CF0D1
S3150800AE00A2FD7B681B79002B40F092807A687B68EC
S3150800AE101B7C0233DBB21946104601F05BF96F4919
S3150800AE206A480CF099FE03461A46654B1B8813447C
S3150800AE309AB2634B1A8000237B617B685B6918466C
S3150800AE40FEF704F902467B699A428CBF0123002368
S3150800AE50DBB2002B00F0AF8003215C480DF017F938
S3150800AE607B6893F828301A467B69934237D17B680A
S3150800AE7093F939307A680E339B0013445B68FB609C
S3150800AE804F4B1C884F4B1B789DB2F9684F480CF006
S3150800AE9063FE03461A46524B1B789BB20093134631
S3150800AEA02A46214649480DF01AFD002147480DF06B
S3150800AEB0EEF8434B1988434B1B789AB2FB68434814
S3150800AEC00CF041FDF96841480CF046FE03461A4667
S3150800AED03B4B1B8813449AB2394B1A8024E07B6893
S3150800AEE0D4337A691146184600F0ECFA034693F90A
S3150800AEF000307A680E339B0013445B683B61304B25
S3150800AF001988304B1B789AB23B6930480CF01BFD08
S3150800AF1039692E480CF020FE03461A46284B1B8832
S3150800AF2013449AB2264B1A807B6901337B6184E706
S3150800AF307A687B681B7C0233DBB21946104601F03F
S3150800AF40C9F87B682C331846FEF78CF803461A4670
S3150800AF502449204859F01AFD194B1988194B1B78B2
S3150800AF609AB21C4B19480CF0EEFC7B682C33184639
S3150800AF70FEF778F80346194614480CF0EDFD03462B
S3150800AF801A460F4B1B8813449AB20D4B1A807B68DE
S3150800AF905B691846FEF766F803461A4611490D48D6
S3150800AFA059F0F4FC064B1988064B1B789AB2094BE4
S3150800AFB006480CF0C8FC00BF1837BD46B0BD00BF38
S3150800AFC010100020121000204C85060814C201201B
S3150800AFD050850608141000200E1000205885060813
S3150800AFE0281000205C85060890B585B000AF78600B
S3150800AFF039603B681B780B3B202B00F2F38101A2DA
S3150800B00052F823F089B0000821B20008E5B3000819
S3150800B01097B20008E5B30008E5B3000809B30008CD
S3150800B020E5B3000877B30008E5B30008E5B3000800
S3150800B030E5B30008E5B30008E5B30008E5B3000882
S3150800B040E5B30008E5B30008E5B30008E5B3000872
S3150800B050E5B30008E5B30008E5B30008E5B3000862
S3150800B060E5B30008E5B30008E5B30008E5B3000852
S3150800B070E5B30008E5B30008E5B30008E5B3000842
S3150800B080E5B30008FBB100087B6803F1D4027B68CE
S3150800B09093F828301946104600F014FA02467B68E1
S3150800B0A093F9393013707B6893F828301C467B680F
S3150800B0B05B691846FDF7CAFF0346013B9C4234BF4D
S3150800B0C001230023DBB2002B38D07B6893F82830A5
S3150800B0D00133DAB27B6883F828207B6893F8383026
S3150800B0E0002B11D07B685B691846FDF7BBFF02464B
S3150800B0F07B6893F8283013441A787B6893F83830BD
S3150800B1009A4201D1012300E00023002B00F06C8154
S3150800B1107B6803F1D4027B6893F8283019461046F9
S3150800B12000F0D0F9034625221A707B6893F8283078
S3150800B1300133DAB27B6883F8282055E10023FB60E7
S3150800B1407B681B7E1A46FB68934247DA7B68D433D2
S3150800B150FA681146184600F0B5F9034693F9003027
S3150800B160252B0CBF01230023DBB2002B19D07B68EB
S3150800B170D433FA681146184600F0A4F9034693F941
S3150800B18000307A680E339B0013445C687B681C3376
S3150800B190FA6811461846FEF73BFA034622781A70F3
S3150800B1A018E07B68D433FA681146184600F08AF925
S3150800B1B0034693F900307A680E339B0013445C68A3
S3150800B1C07B681C33FA6811461846FEF721FA0346CF
S3150800B1D022781A70FB680133FB60B1E77B685A690D
S3150800B1E07B681C3319461046FEF74CF97B6801222A
S3150800B1F05A717B6801221A71F6E07B6893F8283049
S3150800B200002B08D07B6893F82830013BDAB27B68BC
S3150800B21083F82820F1E07B685A797B681A71ECE09C
S3150800B2207B6893F93930DBB20133DBB25AB27B68FB
S3150800B23083F839207B6893F8E030002B0AD17B68C5
S3150800B24093F93930232B40F3D1807B68002283F8A9
S3150800B2503920CBE07B6893F8E030012B0AD17B6874
S3150800B26093F93930192B40F3C1807B68002283F8A3
S3150800B2703920BBE07B6893F8E030022B40F0B680BB
S3150800B2807B6893F93930232B40F3B0807B681A2208
S3150800B29083F83920AAE07B6893F93930DBB2013BA1
S3150800B2A0DBB25AB27B6883F839207B6893F8E030C2
S3150800B2B0002B0AD17B6893F93930002B80F29880ED
S3150800B2C07B68232283F8392092E07B6893F8E03084
S3150800B2D0012B0AD17B6893F93930002B80F28880DC
S3150800B2E07B68192283F8392082E07B6893F8E0307E
S3150800B2F0022B7DD17B6893F93930192B78DC7B6872
S3150800B300232283F8392073E07B6893F93930DBB25E
S3150800B3100133DBB25AB27B6883F839207B6893F82D
S3150800B320E030002B09D17B6893F93930232B61DD96
S3150800B3307B68002283F839205CE07B6893F8E0306C
S3150800B340012B09D17B6893F93930192B52DD7B68BB
S3150800B350002283F839204DE07B6893F8E030022B11
S3150800B36048D17B6893F93930232B43DD7B681A2251
S3150800B37083F839203EE07B6893F93930DBB2013B2C
S3150800B380DBB25AB27B6883F839207B6893F8E030E1
S3150800B390002B09D17B6893F93930002B2CDA7B68AE
S3150800B3A0232283F8392027E07B6893F8E030012BC5
S3150800B3B009D17B6893F93930002B1DDA7B6819228D
S3150800B3C083F8392018E07B6893F8E030022B13D114
S3150800B3D07B6893F93930192B0EDC7B68232283F8B6
S3150800B3E0392009E000BF08E000BF06E000BF04E01E
S3150800B3F000BF02E000BF00E000BF00BF1437BD4633
S3150800B40090BD00BF80B582B000AF7860786800F064
S3150800B41068F87B68184600F070F87B6818460837A5
S3150800B420BD4680BD80B582B000AF7860786800F010
S3150800B43078F87B6818460837BD4680BD80B582B067
S3150800B44000AF78607B6819687B689A687B681B68B8
S3150800B450D31A1A46786800F06FF87B681846FFF723
S3150800B460CAFA7B6818460837BD4680BDB0B582B0B3
S3150800B47000AF78607B681C687B685D687B681846E7
S3150800B48000F06DF803461A462946204600F072F881
S3150800B4907B681846FFF7D2FF7B6818460837BD4613
S3150800B4A0B0BD80B582B000AF78603960386800F00A
S3150800B4B06FF803461946786800F075F800BF083734
S3150800B4C0BD4680BD80B483B000AF786039607B68C4
S3150800B4D01A683B68134418460C37BD465DF8047B6A
S3150800B4E0704780B582B000AF7860786800F089F858
S3150800B4F07B6818460837BD4680BD80B483B000AF68
S3150800B50078607B6800221A607B6800225A607B6834
S3150800B51000229A607B6818460C37BD465DF8047BA6
S3150800B520704780B483B000AF78607B6818460C37E4
S3150800B530BD465DF8047B704780B584B000AFF860FF
S3150800B540B9607A60BB68002B05D0FB687A68B96871
S3150800B550184600F061F800BF1037BD4680BD80B4BC
S3150800B56083B000AF78607B6818460C37BD465DF837
S3150800B570047B704780B584B000AFF860B9607A6024
S3150800B580B968F86800F057F800BF1037BD4680BDA7
S3150800B59080B483B000AF78607B6818460C37BD4628
S3150800B5A05DF8047B7047B0B582B000AF786039604B
S3150800B5B07B685A687B689B689A4211D07C687B686E
S3150800B5C05D68386800F044F803461A46294620465E
S3150800B5D000F049F87B685B685A1C7B685A600CE087
S3150800B5E0786800F053F80446386800F031F80346E6
S3150800B5F01A462146786800F071F800BF0837BD463C
S3150800B600B0BD80B483B000AF78607B6818460C374D
S3150800B610BD465DF8047B704780B584B000AFF8601E
S3150800B620B9607A607A68B968F86800F00FF900BFFF
S3150800B6301037BD4680BD80B582B000AF78603960EE
S3150800B6403968786800F00FF900BF0837BD4680BD35
S3150800B65080B483B000AF78607B6818460C37BD4667
S3150800B6605DF8047B704780B584B000AFF860B960B8
S3150800B6707A607868FFF7ECFF03461A46B968F868F7
S3150800B68000F0FCF800BF1037BD4680BD80B584B019
S3150800B69000AF78607B681A1D07F10C03114618463F
S3150800B6A000F004F9FB6818461037BD4680BD80B522
S3150800B6B082B000AF184600F005F80346184608376A
S3150800B6C0BD4680BD80B483B000AF387101231846EB
S3150800B6D00C37BD465DF8047B70470000B0B58CB0EA
S3150800B6E000AFF860B9607A60574A0121F86800F03F
S3150800B6F0EDF8B862FB681B687B62FB685B683B62B7
S3150800B700F86800F02AF903467B6107F1140207F18D
S3150800B71008031146184600F030F90346FB61FB683A
S3150800B720B96A184600F03DF9B861BB69FB62FC6866
S3150800B730BA69FB69D5187868FFF78AFF03461A467F
S3150800B74029462046FFF78FFF0023FB62FFF7AFFF6E
S3150800B7500346002B27D007F10803184600F049F9DD
S3150800B76003461C68FB681846FFF7F9FE0346BA69E4
S3150800B7702146786A00F029F9F862FB6A0133FB6210
S3150800B78007F10803184600F034F903461C68FB68FD
S3150800B7901846FFF7E4FE0346FA6A396A204600F0BF
S3150800B7A014F9F86226E007F10803184600F021F9B3
S3150800B7B003461C68FB681846FFF7D1FE0346BA69BC
S3150800B7C02146786A00F020F9F862FB6A0133FB62C9
S3150800B7D007F10803184600F00CF903461C68FB68D5
S3150800B7E01846FFF7BCFE0346FA6A396A204600F097
S3150800B7F00BF9F862FFF75BFF034683F00103DBB240
S3150800B800002B09D0FB681846FFF7A9FE03461A461F
S3150800B810396A786AFFF7AEFEF868FB689A687B6A49
S3150800B820D31A1A46796AFFF787FEFB68BA691A605F
S3150800B830FB68FA6A5A60BA69BB6A1A44FB689A6076
S3150800B84000BF3037BD46B0BD6085060880B584B0F8
S3150800B85000AFF860B9607A60B86857F0EBF800BFD7
S3150800B8601037BD4680BD80B483B000AF78603960BC
S3150800B87000BF0C37BD465DF8047B704790B585B0B0
S3150800B88000AFF860B9607A607868FFF7E1FE0346B2
S3150800B89093F90040BB6819460120FFF7A0F8034654
S3150800B8A022461A7000BF1437BD4690BD80B483B0D7
S3150800B8B000AF786039603B681A687B681A607B68F5
S3150800B8C018460C37BD465DF8047B704790B587B0BF
S3150800B8D000AFF860B9607A60F86800F0AEF8044620
S3150800B8E0F86800F0BBF80346E21ABB689A4234BF10
S3150800B8F001230023DBB2002B02D0786857F0B7F893
S3150800B900F86800F0ABF80446F86800F0A7F80346B4
S3150800B9103B6107F1080207F110031146184600F0CB
S3150800B920ACF803461B6823447B61F86800F096F878
S3150800B93002467B69934206D3F86800F07EF8024611
S3150800B9407B69934204D9F86800F077F8034600E06B
S3150800B9507B6918461C37BD4690BD80B584B000AFDC
S3150800B96078607A6807F10C0311461846FFF79EFFC0
S3150800B970FB6818461037BD4680BD90B583B000AF4A
S3150800B98078603960786800F034F803461C683868CF
S3150800B99000F02FF803461B68E31A18460C37BD4615
S3150800B9A090BD80B582B000AF786039603B68002BE7
S3150800B9B006D07B683968184600F073F8034600E03D
S3150800B9C0002318460837BD4680BD90B589B002AF3A
S3150800B9D0F860B9607A603B608DF800403B687A6829
S3150800B9E0B968F86800F06CF8034618461C37BD4677
S3150800B9F090BD80B483B000AF78607B6818460C377A
S3150800BA00BD465DF8047B704790B585B000AFF86019
S3150800BA10B9607A603B60F86800F064F80446B86874
S3150800BA2000F060F801463B687A68204600F069F83D
S3150800BA30034618461437BD4690BD80B582B000AFA0
S3150800BA4078607B68184600F087F80346184600F0C9
S3150800BA5069F8034618460837BD4680BD80B483B0EA
S3150800BA6000AF78607B685A687B681B68D31A1846EB
S3150800BA700C37BD465DF8047B704780B483B000AFD1
S3150800BA80786039607B681A683B681B689A4201D2FD
S3150800BA903B6800E07B6818460C37BD465DF8047BBA
S3150800BAA0704780B582B000AF786039600022396887
S3150800BAB0786800F05CF8034618460837BD4680BD2E
S3150800BAC080B584B000AFF860B9607A603B603B68C7
S3150800BAD07A68B968F86800F066F8034618461037B9
S3150800BAE0BD4680BD80B584B000AF786007F10C0311
S3150800BAF07968184600F074F8FB6818461037BD4692
S3150800BB0080BD80B584B000AFF860B9607A603B60EC
S3150800BB107A68B968F86800F072F80346184610376C
S3150800BB20BD4680BD80B584B000AF78606FF0004335
S3150800BB30FB60786800F075F80346BB6007F10802F9
S3150800BB4007F10C031146184600F077F803461B6800
S3150800BB5018461037BD4680BD80B483B000AF786004
S3150800BB607B6818460C37BD465DF8047B704780B580
S3150800BB7084B000AFF860B9607A60F86800F071F8D0
S3150800BB800246BB6893428CBF01230023DBB2002B1D
S3150800BB9001D056F069FFB86856F050FF03461846BC
S3150800BBA01037BD4680BDB0B584B000AFF860B96047
S3150800BBB07A603B60F86800F060F80446B86800F000
S3150800BBC05CF80546786800F058F802463B6829464E
S3150800BBD0204600F05DF8034618461037BD46B0BD4E
S3150800BBE080B483B000AF786039607B683A681A60C1
S3150800BBF07B6818460C37BD465DF8047B704780B5F0
S3150800BC0086B000AFF860B9607A600123FB757A6880
S3150800BC10B968F86800F057F8034618461837BD465D
S3150800BC2080BD80B582B000AF7860786800F019F8FA
S3150800BC30034618460837BD4680BD80B483B000AFBA
S3150800BC40786039603B681A687B681B689A4201D23B
S3150800BC503B6800E07B6818460C37BD465DF8047BF8
S3150800BC60704780B483B000AF78606FF00043184621
S3150800BC700C37BD465DF8047B704780B483B000AFCF
S3150800BC8078607B6818460C37BD465DF8047B7047BC
S3150800BC9080B586B000AFF860B9607A603B60BA6874
S3150800BCA0FB68D31A7B617B69002B05DD7B691A4625
S3150800BCB0F968786858F0C0F87B697A6813441846BA
S3150800BCC01837BD4680BD80B584B000AFF860B9604E
S3150800BCD07A607A68B968F86800F005F80346184685
S3150800BCE01037BD4680BD90B585B000AFF860B96025
S3150800BCF07A60F86800F00FF80446B86800F00BF8A8
S3150800BD0003467A681946204600F016F80346184690
S3150800BD101437BD4690BD80B582B000AF78603B1D34
S3150800BD20184600F02CF80346184600F034F8034687
S3150800BD3018460837BD4680BDB0B584B000AFF86078
S3150800BD40B9607A60F868FFF798FF0446B868FFF7A5
S3150800BD5094FF05467B681846FFF78FFF03461A4689
S3150800BD602946204600F022F802463B1D1146184691
S3150800BD7000F02EF8034618461037BD46B0BD80B40D
S3150800BD8083B000AF78607B681B6818460C37BD46E1
S3150800BD905DF8047B704780B483B000AF78607B6839
S3150800BDA018460C37BD465DF8047B704780B586B0EB
S3150800BDB000AFF860B9607A600123FB757A68B968E4
S3150800BDC0F86800F011F8034618461837BD4680BDD6
S3150800BDD080B483B000AF786039603B6818460C378A
S3150800BDE0BD465DF8047B704780B586B000AFF86045
S3150800BDF0B9607A60BA68FB68D31A7B617B69002BE5
S3150800BE0005D07B691A46F968786858F015F87B6991
S3150800BE107A68134418461837BD4680BD80B485B085
S3150800BE2000AFF8607A603B600B46FB72194AFB6804
S3150800BE301A60FB6802221A71FB6802225A71FB68B3
S3150800BE4000229A71FB680522DA71FB6800221A74CF
S3150800BE50FB6808225A74FB6800229A74FB7A0F2B37
S3150800BE6002D8FB7A002B01D10023FB72FB68FA7A11
S3150800BE701A74FB687A689A60FB683A68DA60FB6845
S3150800BE803A7E1A71FB6818461437BD465DF8047B7E
S3150800BE90704700BF9CB4060880B582B000AF7860D2
S3150800BEA0074A7B681A607B689B68002B03D00121D0
S3150800BEB0184656F0C1FD7B6818460837BD4680BD52
S3150800BEC09CB4060880B582B000AF78600B46FB705C
S3150800BED07B689B79012B11D07B681B79032B0DD0CE
S3150800BEE0FB781946786800F00EF87B68DB68002B4B
S3150800BEF004D07B68DB68FA78104698470023184612
S3150800BF000837BD4680BD80B483B000AF78600B4665
S3150800BF10FB707B681B79FA789A4203D07B681A799A
S3150800BF207B685A717B68FA781A7100BF0C37BD4670
S3150800BF305DF8047B704780B483B000AF78607B6897
S3150800BF405A797B681A7100BF0C37BD465DF8047BC9
S3150800BF50704780B483B000AF78607B681B79184659
S3150800BF600C37BD465DF8047B704780B483B000AFDC
S3150800BF7078607B689B7918460C37BD465DF8047B6C
S3150800BF80704780B483B000AF78607B6800229A71EE
S3150800BF9000BF0C37BD465DF8047B704780B483B09C
S3150800BFA000AF78600B46FB707B68FA789A7100BF21
S3150800BFB00C37BD465DF8047B704780B483B000AF8C
S3150800BFC078607B68DB7918460C37BD465DF8047BDC
S3150800BFD07047000080B582B000AF78607B685B7CF4
S3150800BFE0082B04D1214922480BF0D9FD07E07B68CC
S3150800BFF05B7C062B03D11F491D480BF0D0FD1C485E
S3150800C0000BF04FFD1A480BF097FD194B93F92930A1
S3150800C010DAB2174B93F92A30DBB2D31ADAB2164BD7
S3150800C0201A707B689B7C002B04D1114B1A88134B22
S3150800C0301A8004E07B689B7C9AB2104B1A807B6856
S3150800C0409B79012B03D07B681B79032B04D1012133
S3150800C05007480CF01CF804E0032105480CF017F813
S3150800C06000BF00BF0837BD4680BD00BFECDA060832
S3150800C07014C2012004BD0608281000202A1000203A
S3150800C08080B483B000AF78600B46FB707B68FA78A3
S3150800C0909A7400BF0C37BD465DF8047B704780B4C0
S3150800C0A083B000AF78607B689B6818460C37BD463E
S3150800C0B05DF8047B704780B483B000AF7860396060
S3150800C0C07B683A689A6000BF0C37BD465DF8047B0A
S3150800C0D07047000080B483B000AF78600B46FB70F1
S3150800C0E0FB78013B0E2B00F2E58001A252F823F003
S3150800C0F02DC1000849C1000861C1000883C10008B4
S3150800C100A3C10008BFC10008E5C1000809C20008AC
S3150800C11029C2000853C2000873C200088FC200086B
S3150800C120B5C20008B5C20008B5C20008654B1A7842
S3150800C130654B1A70654B1B885B089AB2644B1A806C
S3150800C140644B00221A80B6E05E4B1A785E4B1A7072
S3150800C1505E4B1A885E4B1A805E4B00221A80AAE054
S3150800C160584B1A78584B1A70584B1B885B089AB26A
S3150800C170574B1A80554B1B885B089AB2554B1A8049
S3150800C18099E0504B1B785B00DAB24F4B1A704F4B55
S3150800C1901B885B089AB24E4B1A804E4B00221A80B7
S3150800C1A089E0484B1B785B00DAB2474B1A70474B5D
S3150800C1B01A88474B1A80474B00221A807BE0414B6E
S3150800C1C01B785B00DAB2404B1A70404B1B885B0841
S3150800C1D09AB23F4B1A803D4B1B885B089AB23D4B7F
S3150800C1E01A8068E0374B1B781A4652001344DAB2B5
S3150800C1F0354B1A70354B1B885B089AB2344B1A803C
S3150800C200344B00221A8056E02E4B1B781A465200F1
S3150800C2101344DAB22C4B1A702C4B1A882C4B1A8002
S3150800C2202C4B00221A8046E0264B1B781A465200F1
S3150800C2301344DAB2244B1A70244B1B885B089AB253
S3150800C240234B1A80214B1B885B089AB2214B1A8014
S3150800C25031E01C4B1B789B00DAB21B4B1A701B4B48
S3150800C2601B885B089AB21A4B1A801A4B00221A804E
S3150800C27021E0144B1B789B00DAB2134B1A70134B50
S3150800C2801A88134B1A80134B00221A8013E00D4BA1
S3150800C2901B789B00DAB20C4B1A700C4B1B885B0898
S3150800C2A09AB20B4B1A80094B1B885B089AB2094B4A
S3150800C2B01A8000E000BF00BF0C37BD465DF8047B5E
S3150800C2C0704700BF28100020121000202A100020F6
S3150800C2D00E1000201010002080B586B002AFF8605E
S3150800C2E07A603B600B46FB72F868F97A0223009382
S3150800C2F07B6A7A68FFF792FD144AFB681A60FB6846
S3150800C30000221A76FB680022DA61FB68002283F8AD
S3150800C3102020FB68002283F82120FB6897F820205C
S3150800C32083F82820FB680322DA713B68002B05D0C6
S3150800C330FB683A685A61FB683A7E1A76FB68FA69BE
S3150800C3405A62FB6818461037BD4680BDD4B4060845
S3150800C35080B582B000AF7860134A7B681A60786847
S3150800C36000F0BDFB7B685B6A002B03D001211846F1
S3150800C37056F062FB7B68DB69002B03D00121184667
S3150800C38056F05AFB7B689B68002B03D001211846A0
S3150800C39056F052FB7B681846FFF77EFD7B68184609
S3150800C3A00837BD4680BD00BFD4B4060880B582B044
S3150800C3B000AF78607868FFF7CBFF2C21786856F0D5
S3150800C3C03BFB7B6818460837BD4680BD80B586B0FE
S3150800C3D002AFF8607A601A460B46FB721346BB72C8
S3150800C3E0F868F97ABB7A0093BB697A68FFF716FD95
S3150800C3F0154AFB681A60FB6800221A76FB68002259
S3150800C400DA61FB68002283F82020FB68002283F8A3
S3150800C4102120FB6897F8282083F82820FB68032248
S3150800C420DA713B6A002B06D0FB683A6A5A61FB68E8
S3150800C43097F824201A76FB68FA695A62FB68184648
S3150800C4401037BD4680BD00BFD4B4060880B586B097
S3150800C45000AF786039603B681B782B2B19D02B2BE3
S3150800C46000F3A1800E2B19D00E2B00F39C800B2B0A
S3150800C47002D00C2B54D096E07B681B680C331B68E3
S3150800C480786898477B6801225A717B6801221A717D
S3150800C4908EE07B685A797B681A7189E07B6893F924
S3150800C4A02130DBB20133DBB25AB27B6883F8212034
S3150800C4B00123FB75FB7D002B25D00023FB7500238C
S3150800C4C03B617B6893F820301A463B699342F1DA60
S3150800C4D07B6893F9213019467B68DA693B6913440E
S3150800C4E01B7899420BD17B6893F92130DBB2013373
S3150800C4F0DBB25AB27B6883F821200123FB753B69BE
S3150800C50001333B61DDE77B681B7E1A467B6893F93E
S3150800C51021309A4249DC7B68002283F8212044E0D6
S3150800C5207B6893F92130DBB2013BDBB25AB27B68F8
S3150800C53083F821200123FB73FB7B002B25D00023E6
S3150800C540FB730023BB607B6893F820301A46BB68F0
S3150800C5509342F1DA7B6893F9213019467B68DA69E8
S3150800C560BB6813441B7899420BD17B6893F9213039
S3150800C570DBB2013BDBB25AB27B6883F82120012388
S3150800C580FB73BB680133BB60DDE77B6893F9213039
S3150800C590002B0CDA7B681B7E013BDBB25AB27B6848
S3150800C5A083F8212003E000BF02E000BF00E000BFDF
S3150800C5B000BF1837BD4680BD80B582B000AF786031
S3150800C5C00B46FB707B68FA7811461846FFF77AFC2B
S3150800C5D07B6893F82830022B21D17B6893F92130A8
S3150800C5E0DBB20133DBB25AB27B6883F821207B6861
S3150800C5F01B7E1A467B6893F921309A4203DC7B68D6
S3150800C600002283F821207B681B680C331B68786836
S3150800C61098477B6801225A717B6801221A710023A8
S3150800C62018460837BD4680BD80B483B000AF786031
S3150800C6307B685B6A002B06D07B6893F921207B68B0
S3150800C6405B6AD2B21A70002318460C37BD465DF8ED
S3150800C650047B704790B585B000AF78600B46FB70D9
S3150800C6607B681846FFF7B6FC7B6893F82830012BE1
S3150800C67040F096807A687B681B7C19461046FFF75F
S3150800C68029FDFB78002B08D09D4B19889D4B1B78FC
S3150800C6909AB29D4B9D480BF056F97B681B79002B87
S3150800C6A056D10023FB600023FB60FB68032B47DCA5
S3150800C6B07A68FB680133DBB2194649000B44DBB2E2
S3150800C6C019461046FFF706FD7B6893F92130002BC3
S3150800C6D000DA03339B105BB29B00FA681344BB6015
S3150800C6E07B6893F921301A46BB6893420FD1884B71
S3150800C6F01C88884985480BF02FFA0346E31A99B235
S3150800C700804B1B789AB2834B80480BF01CF97B68E8
S3150800C7101B7E1A46BB6893420EDA794B1988794B09
S3150800C7201B7898B27B685A69BB689B0013441B68E0
S3150800C730024676480BF007F9FB680133FB60B4E75D
S3150800C7407B689B681A467449744858F01FF906E0D6
S3150800C7507B689B681A467249704858F017F97A68D8
S3150800C7607B681B7C19461046FFF7B4FC6D4B1B888B
S3150800C7701C466A4965480BF0EFF90346E31A9AB274
S3150800C7805F4B1B8813449AB25D4B1A805C4B198821
S3150800C7905C4B1B789AB2614B5C480BF0D4F875E198
S3150800C7A07B6893F82830002B40F0C2807A687B6853
S3150800C7B01B7C19461046FFF78DFCFB78002B08D02A
S3150800C7C04F4B19884F4B1B789AB24F4B4F480BF07B
S3150800C7D0BAF87B681B79002B38D17A687B681B7C92
S3150800C7E00233DBB219461046FFF774FC7B681B7EE2
S3150800C7F0002B0DD14C49494858F0C8F8404B1988C8
S3150800C800404B1B789AB2454B40480BF09CF815E014
S3150800C8107B685A697B6893F921309B0013441B682F
S3150800C8201A4642493D4858F0B1F8354B1988354BF8
S3150800C8301B789AB2394B35480BF085F87B689B68AC
S3150800C8401A463549354858F0A1F837E07A687B68C2
S3150800C8501B7C0233DBB219461046FFF73BFC7B68AC
S3150800C8601B7E002B0DD130492C4858F08FF8244BED
S3150800C8701988244B1B789AB2284B24480BF063F886
S3150800C88015E07B685A697B685B6A1B789B001344D2
S3150800C8901B681A462549214858F078F8184B198814
S3150800C8A0184B1B789AB21D4B18480BF04CF87B684E
S3150800C8B09B681A461849194858F068F87A687B68D8
S3150800C8C01B7C19461046FFF705FC164B1B881C46B1
S3150800C8D012490E480BF040F90346E31A9AB2084B80
S3150800C8E01B8813449AB2064B1A80054B1988054BC8
S3150800C8F01B789AB2094B05480BF025F8C6E000BF2D
S3150800C90010100020121000207C85060814C2012091
S3150800C9102A10002080850608848506081410002041
S3150800C920888506080E1000208C8506089885060856
S3150800C9307B6893F82830022B40F0A8807A687B68D9
S3150800C9401B7C19461046FFF7C5FBFB78002B08D061
S3150800C950504B1988504B1B789AB2504B50480AF0E6
S3150800C960F2FF7B681B79002B38D17A687B681B7CC1
S3150800C9700233DBB219461046FFF7ACFB7B681B7E19
S3150800C980002B0DD14749484858F000F8414B198803
S3150800C990414B1B789AB2444B41480AF0D4FF15E044
S3150800C9A07B685A697B6893F921309B0013441B689E
S3150800C9B01A463E493C4857F0E9FF364B1988364B2C
S3150800C9C01B789AB2384B36480AF0BDFF7B689B68DD
S3150800C9D01A463749344857F0D9FF37E07A687B68F2
S3150800C9E01B7C0233DBB219461046FFF773FB7B68E4
S3150800C9F01B7E002B0DD12B492B4857F0C7FF254B23
S3150800CA001988254B1B789AB2274B25480AF09BFFB5
S3150800CA1015E07B685A697B685B6A1B789B00134440
S3150800CA201B681A462149204857F0B0FF194B198848
S3150800CA30194B1B789AB21C4B19480AF084FF7B687D
S3150800CA409B681A461A49184857F0A0FF7A687B6807
S3150800CA501B7C19461046FFF73DFB164B1B881C46E8
S3150800CA6011490F480BF078F80346E31A9AB2094BB6
S3150800CA701B8813449AB2074B1A80064B1988064B33
S3150800CA801B789AB2084B06480AF05DFF00BF1437B8
S3150800CA90BD4690BD10100020121000207C850608A7
S3150800CAA014C201208C8506081410002098850608F3
S3150800CAB0848506080E10002080B485B000AFF860A3
S3150800CAC0B9601346FB71FB68BA685A61FB68FA7964
S3150800CAD01A7600BF1437BD465DF8047B704780B5EB
S3150800CAE084B000AF78607B685B69002B1DD000239B
S3150800CAF0FB607B681B7E1A46FB68934215DA7B68E7
S3150800CB005A69FB689B0013441B68002B09D07B6895
S3150800CB105A69FB689B0013441B680121184655F0A7
S3150800CB208BFFFB680133FB60E3E700BF1037BD46A8
S3150800CB3080BD80B483B000AF78607B685A697B6833
S3150800CB4093F921309B0013441B6818460C37BD46E1
S3150800CB505DF8047B704780B483B000AF78607B686B
S3150800CB6093F8283018460C37BD465DF8047B7047A5
S3150800CB7080B483B000AF7860064A7B681A607B6829
S3150800CB800022DA607B6818460C37BD465DF8047BE0
S3150800CB90704700BF7CB5060880B586B002AFF8605E
S3150800CBA07A603B600B46FB72F868F97A02230093B9
S3150800CBB0FB697A68FFF732F9114AFB681A60FB6865
S3150800CBC01C3300221A605A601A81FB68002283F817
S3150800CBD026203B68002B07D03B685A68FB689A6199
S3150800CBE03B681A68FB685A61FB68BA699A62FB680F
S3150800CBF00222DA71FB6818461037BD4680BD00BFB1
S3150800CC000CB5060880B582B000AF7860054A7B6827
S3150800CC101A607B681846FFF73FF97B68184608379D
S3150800CC20BD4680BD0CB5060880B582B000AF7860F9
S3150800CC307868FFF7E7FF2C21786855F0FDFE7B68DA
S3150800CC4018460837BD4680BD80B483B000AF78600B
S3150800CC50396000BF0C37BD465DF8047B704780B568
S3150800CC6082B000AF78600B46FB707B68FA78114695
S3150800CC701846FFF727F97B689B6A18460837BD46AA
S3150800CC8080BD80B483B000AF786000BF18460C370B
S3150800CC90BD465DF8047B704790B583B000AF7860F9
S3150800CCA00B46FB707B681846FFF794F97A687B6831
S3150800CCB01B7C013BDBB219461046FFF70BFAFB78E3
S3150800CCC0002B08D02B4B19882B4B1B789AB22B4B71
S3150800CCD02B480AF038FE7B689B681A4629492A4879
S3150800CCE057F054FE294B1B881C46274924480AF04E
S3150800CCF033FF0346E31A9AB21E4B1B8813449AB2B3
S3150800CD001C4B1A801B4B19881B4B1B789AB21E4B5F
S3150800CD101B480AF018FE7B681B79022B07D17B6833
S3150800CD205B691A461A49184857F030FE0CE07B68CA
S3150800CD301B79012B08D17B6803F11C027B689B6970
S3150800CD401449114857F022FE7A687B681B7C013328
S3150800CD50DBB219461046FFF7BDF9064B1988064B94
S3150800CD601B789AB2084B06480AF0EDFD00BF0C374F
S3150800CD70BD4690BD10100020121000209C850608A4
S3150800CD8014C20120A0850608141000200E100020E9
S3150800CD90A8850608AC85060880B483B000AF78601D
S3150800CDA07B6893F8263018460C37BD465DF8047B39
S3150800CDB0704780B582B000AF786039607B681C33F5
S3150800CDC03968184657F052FE00BF0837BD4680BD81
S3150800CDD080B483B000AF786039607B683A685A617E
S3150800CDE000BF0C37BD465DF8047B704780B584B03C
S3150800CDF000AFF8607A601A460B46FB721346BB72A0
S3150800CE00FB6800221A70FB6808225A70FB68043314
S3150800CE1012491846FCF715FAFB6810330F491846ED
S3150800CE20FCF70FFAFB6800225A84FB68002283F895
S3150800CE302420FB68043379681846FCF755FBFB6821
S3150800CE40FA7A1A77FB68BA7A9A77FB683A7E5A773B
S3150800CE50FB6818461037BD4680BD00BFB485060876
S3150800CE6080B582B000AF78607B6810331846FCF74F
S3150800CE7023FA7B6804331846FCF71EFA7B681846C3
S3150800CE800837BD4680BD80B483B000AF78607B6844
S3150800CE909B7F18460C37BD465DF8047B704700003B
S3150800CEA090B591B000AF78607B681B78012B4FD0A6
S3150800CEB0786800F09BF8786800F0E2F87B6804333D
S3150800CEC01846FCF7CFF804467B6810331846FCF77B
S3150800CED0C9F8034607F10C0022461F4957F056FDCC
S3150800CEE07B681B7F002B16D07B681B8C1C4607F1C2
S3150800CEF00C03194619480AF02FFE0346E31ADA0FFF
S3150800CF0013445B1019467B685A8C8BB213449AB249
S3150800CF107B685A8411E07B681B8C1C4607F10C035E
S3150800CF2019460E480AF018FE0346E11A7B685A8C21
S3150800CF308BB213449AB27B685A847B68598C7B6897
S3150800CF4093F824309AB207F10C0304480AF0FBFC64
S3150800CF5000BF4437BD4690BDB885060814C20120F7
S3150800CF6080B582B000AF786039607B681033396865
S3150800CF701846FCF787FA00BF0837BD4680BD80B55E
S3150800CF8082B000AF786039607B6804333968184628
S3150800CF90FCF778FA00BF0837BD4680BD80B483B079
S3150800CFA000AF78600B46FB707B68FA781A7000BF92
S3150800CFB00C37BD465DF8047B704780B483B000AF7C
S3150800CFC078607B681B7818460C37BD465DF8047B8D
S3150800CFD0704780B483B000AF78607B685B7F184683
S3150800CFE00C37BD465DF8047B7047000080B582B0FB
S3150800CFF000AF78607B685B78082B04D11549164822
S3150800D0000AF0CDFD07E07B685B78062B03D1134950
S3150800D01011480AF0C4FD10480AF043FD0E480AF00C
S3150800D0208BFD0D4B93F92930DAB20B4B93F92A3065
S3150800D030DBB2D31ADAB27B6883F82520064B1A8846
S3150800D0407B68DA84032104480BF021F800BF08370F
S3150800D050BD4680BDECDA060814C2012004BD0608E8
S3150800D06080B483B000AF78600B46FB707B68FA78B3
S3150800D0705A7000BF0C37BD465DF8047B7047000048
S3150800D08080B483B000AF78607B681B7F0F2B00F2FB
S3150800D090108101A252F823F0D9D00008FBD000086D
S3150800D0A01BD1000837D100085DD1000881D10008DE
S3150800D0B0A1D10008CBD10008F3D1000817D2000887
S3150800D0C045D2000869D2000889D20008B3D2000800
S3150800D0D0B3D20008B3D200087B68002283F8242064
S3150800D0E07B68DB8C5B089AB27B681A847B68DB8C6E
S3150800D0F05B089AB27B685A84DCE07B6893F8252043
S3150800D1007B6883F824207B68DB8C5B089AB27B6893
S3150800D1101A847B6800225A84CCE07B6893F8252021
S3150800D1207B6883F824207B68DA8C7B681A847B68A2
S3150800D13000225A84BEE07B6893F825207B6883F832
S3150800D14024207B68DB8C5B089AB27B681A847B6830
S3150800D150DB8C5B089AB27B685A84ABE07B6893F8F1
S3150800D16025305B00DAB27B6883F824207B68DB8C89
S3150800D1705B089AB27B681A847B6800225A8499E015
S3150800D1807B6893F825305B00DAB27B6883F8242045
S3150800D1907B68DA8C7B681A847B6800225A8489E06B
S3150800D1A07B6893F825305B00DAB27B6883F8242025
S3150800D1B07B68DB8C5B089AB27B681A847B68DB8C9D
S3150800D1C05B089AB27B685A8474E07B6893F82530CA
S3150800D1D01A4652001344DAB27B6883F824207B6827
S3150800D1E0DB8C5B089AB27B681A847B6800225A84B7
S3150800D1F060E07B6893F825301A4652001344DAB289
S3150800D2007B6883F824207B68DA8C7B681A847B68C1
S3150800D21000225A844EE07B6893F825301A4652005D
S3150800D2201344DAB27B6883F824207B68DB8C5B08BE
S3150800D2309AB27B681A847B68DB8C5B089AB27B6837
S3150800D2405A8437E07B6893F825309B00DAB27B680E
S3150800D25083F824207B68DB8C5B089AB27B681A8487
S3150800D2607B6800225A8425E07B6893F825309B006A
S3150800D270DAB27B6883F824207B68DA8C7B681A84A8
S3150800D2807B6800225A8415E07B6893F825309B005A
S3150800D290DAB27B6883F824207B68DB8C5B089AB259
S3150800D2A07B681A847B68DB8C5B089AB27B685A8435
S3150800D2B000E000BF00BF0C37BD465DF8047B704731
S3150800D2C080B586B002AFF8607A603B600B46FB72A9
S3150800D2D0F868F97A02230093BB697A68FEF79EFD1F
S3150800D2E0084AFB681A60FB6800229A61FB683A687C
S3150800D2F05A61FB680022DA71FB6818461037BD468A
S3150800D30080BD00BF44B5060880B582B000AF78601E
S3150800D310054A7B681A607B681846FEF7BDFD7B6880
S3150800D32018460837BD4680BD44B5060880B582B0A4
S3150800D33000AF78607868FFF7E7FF1C21786855F03A
S3150800D3407BFB7B6818460837BD4680BD90B583B021
S3150800D35000AF78600B46FB707B681846FEF73AFE0E
S3150800D3607A687B681B7C19461046FEF7B3FEFB7885
S3150800D370002B08D0154B1988154B1B789AB2154BFC
S3150800D38015480AF0E0FA154B1B881C467B689B6813
S3150800D390194611480AF0E0FB0346E31ADA0F13446C
S3150800D3A05B109AB2094B1B8813449AB2074B1A8032
S3150800D3B0064B1988064B1B789AB27B689B68064809
S3150800D3C00AF0C1FA00BF0C37BD4690BD1010002008
S3150800D3D012100020C085060814C201200E10002075
S3150800D3E080B483B000AF7860396000BF0C37BD46A3
S3150800D3F05DF8047B704780B582B000AF78600B4655
S3150800D400FB707B68FA7811461846FEF75BFD7B6869
S3150800D4105B6918460837BD4680BD80B483B000AF47
S3150800D42078607B689B6918460C37BD465DF8047BB7
S3150800D430704780B483B000AF7860002318460C3775
S3150800D440BD465DF8047B704780B582B000AF786052
S3150800D450396039687868FCF7ABF803461846083728
S3150800D460BD4680BD80B584B000AFF860B9607A600B
S3150800D470BB689B68F8687A68B968FCF711F9F868B8
S3150800D4801037BD4680BD80B485B000AFF860B9607E
S3150800D4907A603B60FB6800221A70FB680022DA7724
S3150800D4A0FB6800225A63FB6800229A63FB68002225
S3150800D4B0DA63FB68BA685A61FB683A689A61FB687E
S3150800D4C03A7E1A77FB687A685A62FB68FA695A6084
S3150800D4D0FB6897F820201A72FB687A6ADA60FB689C
S3150800D4E001221A74FB6897F828205A74FB6897F883
S3150800D4F02C2083F820203A7E97F82C30B2FBF3F3E1
S3150800D500DAB2FB689A773B7E97F82C20B3FBF2F1E8
S3150800D51002FB01F29B1ADBB2002B05D0FB689B7F4E
S3150800D5200133DAB2FB689A77FB6818461437BD46AA
S3150800D5305DF8047B704780B483B000AF78607B6881
S3150800D54018460C37BD465DF8047B704780B483B037
S3150800D55000AF786039607B683A685A6100BF0C375B
S3150800D560BD465DF8047B704780B586B000AF78602D
S3150800D5707B681B78052B00F0A980786800F0BAFF55
S3150800D58000237B617B68DB7F1A467B6893F8203033
S3150800D59003FB02F37A6892F8202013443B617B6808
S3150800D5A01B7F1A463B69934202DD7B681B7F3B6102
S3150800D5B07B68DB7F1A467B6893F8203003FB02F30F
S3150800D5C07B617A693B699A422DDA7B6893F91D304B
S3150800D5D01A467B69934211D17B689A697B699B00DD
S3150800D5E0134418687B689A697B699B0013441B6817
S3150800D5F01B6810331B680121984710E07B689A69FD
S3150800D6007B699B00134418687B689A697B699B0051
S3150800D61013441B681B6810331B68002198477B69F5
S3150800D62001337B61CDE700237B617B681B7A1A4651
S3150800D6307B6993422FDA7B685A687B699B0013449F
S3150800D6401B681846FFF71FFC03461A467B681B78BB
S3150800D6509A4210D17B685A687B699B0013441B6801
S3150800D6601846FFF7B6FC03461A467B68DB7F9A42E4
S3150800D67001D1012300E00023002B08D07B685A68FB
S3150800D6807B699B0013441B681846FFF709FC7B69F6
S3150800D69001337B61C9E77B681B78002B7DD1414B41
S3150800D6A01B780133DAB23F4B1A703E4B1B78072BB7
S3150800D6B073D97B6801221A703A4B00221A707B686C
S3150800D6C001221A74786801F01CF966E0354B1B785C
S3150800D6D00133DAB2334B1A70324B1B78072B5CD9FD
S3150800D6E0304B00221A707B6801221A74786801F0A0
S3150800D6F008F9786801F005F97B681B78002B19D1C1
S3150800D7007B681B6B01211846FEF7FDFB7B68DB6A0D
S3150800D710002B08D07B68DA6B7B68DB6A19461046F3
S3150800D72001F0CFF939E07B68DB6B0021184601F080
S3150800D730C8F932E07B681B78042B2ED17B6893F8F6
S3150800D74020301A467B68DB7F03FB02F3FB607B68AD
S3150800D7501B7F1A46FB6893421FDA7B6893F91D30D4
S3150800D7601A46FB6893420AD17B689A69FB689B0054
S3150800D77013441B6800211846FEF7C5FB09E07B68C1
S3150800D7809A69FB689B0013441B6801211846FEF73B
S3150800D79005FCFB680133FB60D9E700BF1837BD46B7
S3150800D7A080BD00BF2C10002090B589B000AF78600E
S3150800D7B07B681B78042B40F00C817B689A697B6830
S3150800D7C093F91D309B00134418687B689A697B6837
S3150800D7D093F91D309B0013441B681B6814331B68A0
S3150800D7E07A68526A114698477B685B6A1B782B2BC6
S3150800D7F032D17B689A697B6893F91D309B00134484
S3150800D8001B681846FEF7A5FB0346002B14BF012329
S3150800D8100023DBB2002B1AD0786801F072F87B6817
S3150800D82003221A700023FB617B681B7F1A46FB697B
S3150800D83093420CDA7B689A69FB699B0013441B6860
S3150800D8401846FEF79EFBFB690133FB61ECE77B6834
S3150800D85001221A7400F00EBE7B685B6A1B780B2BDC
S3150800D86040F0B2807B689A697B6893F91D309B000B
S3150800D87013441B681846FEF76CFB0346002B14BFBF
S3150800D88001230023DBB2002B00F099807B68DB685C
S3150800D890002B46D07B689A697B6893F91D309B00FC
S3150800D8A0134418687B689A697B6893F91D309B0056
S3150800D8B013441B681B6808331B680121984778685E
S3150800D8C001F01FF87B689A697B6893F91D309B0005
S3150800D8D013441B681846FEF770FB0346032B0CBF60
S3150800D8E001230023DBB2002B3FD07B6893F820305E
S3150800D8F01A467B68DB7F03FB02F3BB617B681B7FF1
S3150800D9001A46BB69934230DA7B689A69BB699B0001
S3150800D91013441B681846FEF734FBBB690133BB6129
S3150800D920ECE77B6803221A707B6893F820301A4666
S3150800D9307B68DB7F03FB02F37B617B681B7F1A46F0
S3150800D9407B6993420CDA7B689A697B699B0013446E
S3150800D9501B681846FEF7EFFA7B6901337B61ECE733
S3150800D9607B6801221A7400F085BD7B681B78032B3F
S3150800D97004D17B6801221A7400F07CBD7B681B7891
S3150800D980052B5CD17B689B6A0021184600F09EFF38
S3150800D9907B689C6A7B68DB6B184601F02EF90146AA
S3150800D9A07B68DB6B1A46204600F092FD7B68DA6BD3
S3150800D9B07B689B6A1946104601F083F83FE07B684E
S3150800D9C001221A7400F056BD7B6801221A7400F011
S3150800D9D051BD7B681B78052B28D17B68DB6A184606
S3150800D9E000F083FF0346052B0CBF01230023DBB29F
S3150800D9F0002B17D07B6802221A70786800F081FF26
S3150800DA007B68DA6B7B68DB6A1946104601F059F8C1
S3150800DA107B68DB6B184601F099F87B6801221A745B
S3150800DA2000F028BD786800F06CFF08E07B681B787A
S3150800DA30032B04D07B6800221A7400F01BBD7B6898
S3150800DA4001221A747B689B69002B0ED17B685B6A7E
S3150800DA501B780B2B09D07B685B6A1B782B2B04D0B1
S3150800DA607B6800221A7400F005BD7B685B6A1B7828
S3150800DA700B3B212B00F2EB8401A252F823F000BFE6
S3150800DA8009DB000893E0000841E10008CDDF000843
S3150800DA902DE300084FE400084FE400084FE40008AF
S3150800DAA04FE400084FE400084FE400084FE400087C
S3150800DAB04FE400084FE400084FE400084FE400086C
S3150800DAC04FE400084FE400084FE400084FE400085C
S3150800DAD04FE400084FE400084FE400084FE400084C
S3150800DAE04FE400084FE400084FE400084FE400083C
S3150800DAF04FE400084FE400084FE400084FE400082C
S3150800DB000DDF0008A3DF00087B689B69002B2ED178
S3150800DB107B6804221A70786800F0F3FE7B689B6ABB
S3150800DB20002B03D17B6802221A7020E07B689B6A6F
S3150800DB300021184600F0CAFE7B689C6A7B68DB6B8E
S3150800DB40184601F05AF801467B68DB6B1A462046F0
S3150800DB5000F0BEFC7B68DA6B7B689B6A1946104648
S3150800DB6000F0AFFF7B6801221A7400F083BC7B6863
S3150800DB701B78022B52D1786800F0C3FE7B6800221E
S3150800DB801A707B681B6B01211846FEF7BCF97B6887
S3150800DB90DB6A002B09D07B68DB6A184600F0A5FE15
S3150800DBA00346052B01D0012300E00023002B09D0F2
S3150800DBB07B68DA6B7B68DB6A1946104600F081FFE2
S3150800DBC000F049BC7B68DB6A002B0DD07B68DB6AFA
S3150800DBD0184600F08AFE0346052B05D17B689B6A2A
S3150800DBE0002B01D1012300E00023002B0ED07B6817
S3150800DBF0DA6B7B68DB6A1946104600F062FF7B68C1
S3150800DC00DB6B184600F0A2FF00F025BC7B68DB6BD7
S3150800DC100021184600F055FF00F01DBC7B689A6984
S3150800DC207B6893F91D309B0013441B681846FEF762
S3150800DC309CF90346FB737B689A697B6893F91D30E8
S3150800DC409B0013441B681846FEF783F90346BB730B
S3150800DC50FB7B012B00F0FF83BB7B032B00F0FB83D0
S3150800DC607B689A697B6893F91D309B0013441B688F
S3150800DC701846FEF7A2F903467B737B689A697B68A8
S3150800DC8093F91D309B00134418687B689A697B6872
S3150800DC9093F91D309B0013441B681B6808331B68E7
S3150800DCA000219847B860BB68002B02D17B7B002B0C
S3150800DCB013D17B68DB6A184600F017FE0346052B6E
S3150800DCC014BF01230023DBB2002B03D07B6800229C
S3150800DCD01A7002E07B6805221A707B7B002B39D10B
S3150800DCE0BB68002B1FD07B68BA689A627B689B6A00
S3150800DCF00021184600F0EAFD7B689C6A7B68DB6BAE
S3150800DD00184600F07AFF01467B68DB6B1A46204608
S3150800DD1000F0DEFB7B68DA6B7B689B6A1946104667
S3150800DD2000F0CFFE97E37B68DB6A002B08D07B68A0
S3150800DD30DA6B7B68DB6A1946104600F0C2FE8AE396
S3150800DD407B68D86B7B68596B7B689B6B1A4600F0BF
S3150800DD509BFE80E37B7B012B37D1BB68002B2CD045
S3150800DD607B68BA689A627B689B6A0021184600F04D
S3150800DD70ADFD7B68986A7B689A697B6893F91D3064
S3150800DD809B0013441B68194600F0CFFD7B689C6A0C
S3150800DD907B68DB6B184600F030FF01467B68DB6B5F
S3150800DDA01A46204600F094FB7B68DA6B7B689B6A10
S3150800DDB01946104600F085FE4DE3BB68002B40F07F
S3150800DDC04A83786800F09DFD45E37B7B022B30D1C2
S3150800DDD0BB68002B00F03F837B68BA689A627B6851
S3150800DDE09B6A0021184600F071FD7B68986A7B687B
S3150800DDF09A697B6893F91D309B0013441B68194682
S3150800DE0000F093FD7B689C6A7B68DB6B184600F024
S3150800DE10F4FE01467B68DB6B1A46204600F058FB89
S3150800DE207B68DA6B7B689B6A1946104600F049FEE8
S3150800DE3011E37B7B032B5CD17B681B78032B40F0BB
S3150800DE400A837B689A697B6893F91D309B001344A3
S3150800DE5019687B689A697B6893F91D309B0013449F
S3150800DE601B681B682C331B68084698470346022B19
S3150800DE7014BF01230023DBB2002B00F0EE82786882
S3150800DE8000F03FFD7B681B78042B02D07B680422D8
S3150800DE901A707B6893F820301A467B68DB7F03FB91
S3150800DEA002F33B617B681B7F1A463B69934280F20B
S3150800DEB0D2827B6893F91D301A463B6993420AD190
S3150800DEC07B689A693B699B0013441B6800211846C6
S3150800DED0FEF719F809E07B689A693B699B001344C9
S3150800DEE01B6801211846FEF759F83B6901333B6167
S3150800DEF0D8E77B7B042B40F0AE827B681B78032B2C
S3150800DF0040F0A9827B6804221A70A4E27B68DB6A67
S3150800DF10002B46D07B689B69002B1ED17B680022AC
S3150800DF201A70786800F0EDFC7B681B6B1846FEF7E4
S3150800DF3002F87B68DB6A002B08D07B68DA6B7B68A3
S3150800DF40DB6A1946104600F0BCFD0EE07B68DB6B09
S3150800DF500021184600F0B5FD07E07B681B6B1846E4
S3150800DF60FDF7E9FF7B6800221A707B68DB6A1846B2
S3150800DF7000F0BBFC0346052B0CBF01230023DBB2D4
S3150800DF80002B05D07B68DB6A0021184600F09EFC52
S3150800DF907B68DA6B7B68DB6A1946104600F091FDF0
S3150800DFA068E27B68DB6A002B40F059827B68D86B95
S3150800DFB07B68596B7B689B6B1A4600F065FD7B682E
S3150800DFC000221A70786800F09CFC48E27B6893F996
S3150800DFD01D30DBB20133DBB25AB27B685A777B68F5
S3150800DFE01B7F1A467B6893F91D309A420BDC7B68C7
S3150800DFF05B7C002B07D17B681B7F013BDBB25AB2E7
S3150800E0007B685A7744E07B681B7F1A467B6893F9DE
S3150800E0101D309A420FDC7B685B7C002B0BD07B683B
S3150800E0201B7F013BDBB25AB27B685A777B685B6A17
S3150800E03001221A702CE07B6893F91D307A6892F8F1
S3150800E040202093FBF2F102FB01F29B1A002B40F011
S3150800E05008827B68DB7F1A467B689B7F013B9A4276
S3150800E06080F2FF817B6893F82030042B06D17B6809
S3150800E070DB7F0133DAB27B68DA77F2E17B6893F902
S3150800E0801D30DBB2013BDBB25AB27B685A77E8E156
S3150800E090E7E17B6893F91D30DBB2013BDBB25AB28C
S3150800E0A07B685A777B6893F91D30002B07DA7B6803
S3150800E0B05B7C002B03D17B6800225A773FE07B68A4
S3150800E0C093F91D30002B10DA7B685B7C002B0CD093
S3150800E0D07B6800225A777B68D86B7B68596B7B68AC
S3150800E0E09B6B1A4600F0D0FC29E07B6893F91D303B
S3150800E0F001337A6892F8202093FBF2F102FB01F2D1
S3150800E1009B1A002B40F0AF817B68DB7F002B00F069
S3150800E110AA817B6893F82030042B06D17B68DB7FC5
S3150800E120013BDAB27B68DA779DE17B6893F91D30AB
S3150800E130DBB20133DBB25AB27B685A7793E192E1DC
S3150800E1407B6893F82030042B5BD97B6893F91D30E4
S3150800E150042B56D17B6893F91D30DBB2013BDBB249
S3150800E1605AB27B685A777B6893F91D30002B07DA19
S3150800E1707B685B7C002B03D17B6800225A773FE0E3
S3150800E1807B6893F91D30002B10DA7B685B7C002BCB
S3150800E1900CD07B6800225A777B68D86B7B68596BF2
S3150800E1A07B689B6B1A4600F06FFC29E07B6893F945
S3150800E1B01D3001337A6892F8202093FBF2F102FBB6
S3150800E1C001F29B1A002B40F0AF807B68DB7F002BA7
S3150800E1D000F0AA807B6893F82030042B06D17B6870
S3150800E1E0DB7F013BDAB27B68DA779DE07B6893F9DF
S3150800E1F01D30DBB20133DBB25AB27B685A7793E043
S3150800E20092E07B68DB7F002B29D07B6893F820306F
S3150800E210042B00F02A817B68DB7F013BDAB27B683E
S3150800E220DA777B6893F91D30DAB27B6893F8203089
S3150800E230D31ADBB25AB27B685A777B6893F91D30DA
S3150800E240002B80F212817B68DA7F7B6893F8203096
S3150800E25012FB03F3DBB25AB27B685A7705E17B6897
S3150800E260DB7F002B40F001817B68DB6A002B46D000
S3150800E2707B689B69002B1ED17B6800221A70786820
S3150800E28000F03FFB7B681B6B1846FDF754FE7B6866
S3150800E290DB6A002B08D07B68DA6B7B68DB6A194679
S3150800E2A0104600F00EFC0EE07B68DB6B002118467A
S3150800E2B000F007FC07E07B681B6B1846FDF73BFE82
S3150800E2C07B6800221A707B68DB6A184600F00DFB33
S3150800E2D00346052B0CBF01230023DBB2002B05D018
S3150800E2E07B68DB6A0021184600F0F0FA7B68DA6B77
S3150800E2F07B68DB6A1946104600F0E3FBBAE07B68E8
S3150800E300DB6A002B40F0B3807B68D86B7B68596B5F
S3150800E3107B689B6B1A4600F0B7FB7B6800221A7075
S3150800E320786800F0EEFAA2E000BF9EE07B6893F8FA
S3150800E3302030042B56D97B6893F91D30022B51DD0A
S3150800E3407B6893F91D30DBB20133DBB25AB27B68C6
S3150800E3505A777B681B7F1A467B6893F91D309A4269
S3150800E3600BDC7B685B7C002B07D17B681B7F013B42
S3150800E370DBB25AB27B685A7733E07B681B7F1A4652
S3150800E3807B6893F91D309A420FDC7B685B7C002B17
S3150800E3900BD07B681B7F013BDBB25AB27B685A778E
S3150800E3A07B685B6A01221A701BE07B6893F91D3053
S3150800E3B07A6892F8202093FBF2F102FB01F29B1A8D
S3150800E3C0002B42D17B68DB7F1A467B689B7F013B2B
S3150800E3D09A423ADA7B68DB7F0133DAB27B68DA770E
S3150800E3E033E032E07B68DB7F1A467B689B7F013B24
S3150800E3F09A423EDA7B6893F82030042B39D07B6842
S3150800E400DB7F0133DAB27B68DA777B6893F91D30F4
S3150800E410DAB27B6893F820301344DBB25AB27B68D1
S3150800E4205A777B681B7F1A467B6893F91D309A4298
S3150800E4301FDC7B68DA7F7B6893F8203012FB03F3D6
S3150800E440DBB25AB27B685A7713E000BF11E07B68EB
S3150800E45000221A740EE000BF0CE000BF0AE000BFFD
S3150800E46008E000BF06E000BF04E000BF02E000BF0E
S3150800E47000E000BF2437BD4690BD00BF80B483B01E
S3150800E48000AF786039607B683A685A6300BF0C371A
S3150800E490BD465DF8047B704780B483B000AF7860F2
S3150800E4A039607B683A689A6300BF0C37BD465DF8E9
S3150800E4B0047B704780B483B000AF786039607B68AE
S3150800E4C03A68DA6300BF0C37BD465DF8047B7047CF
S3150800E4D080B485B000AFF860B9607A60FB68BA6846
S3150800E4E0DA62FB687A68DA6300BF1437BD465DF8FE
S3150800E4F0047B704790B59DB000AF7860B949BA48BB
S3150800E50009F04DFBB84809F017FB0321B64809F096
S3150800E510BEFD7B6893F82030042B1FD17B68DB7F18
S3150800E520002B0CD0B149B04809F016FB0346C3F1DD
S3150800E530F90399B2AD4B0522AB4809F004FA7B689A
S3150800E540DB7F1A467B689B7F013B9A423AD0A84BF1
S3150800E5500522F921A44809F0F6F933E0A24B1B88F5
S3150800E56087F86F30A349A04809F0F6FA0346DBB2EC
S3150800E57097F86F20D31A87F86F307B68DB7F1A46C7
S3150800E5807B689B7F013B9A4207D097F86F3099B218
S3150800E590984B0322944809F0D6F99749924809F00E
S3150800E5A0DBFA0346DBB297F86F20D31A87F86F3089
S3150800E5B097F86F309BB2013B99B28F4B03228A487A
S3150800E5C009F0C1F98D49884809F0E9FA864809F041
S3150800E5D068FA854809F0B0FA0321834809F057FD1F
S3150800E5E07B685A6907F1180311461846FAF729FE97
S3150800E5F007F10C0382491846FAF723FE07F11803B8
S3150800E60080491846FEF720FF0346002B14BF012356
S3150800E6100023DBB2002B00F04281002387F86E301E
S3150800E62007F1240007F1180108230022FBF738F840
S3150800E63007F1240207F10C0311461846FAF742FFC0
S3150800E64007F124031846FAF737FE07F10C031846B4
S3150800E650FAF708FD034600220021634809F073F91A
S3150800E66007F10C031846FAF7FDFC034619465E48FF
S3150800E67009F072FA0346DAB297F86E30134487F84F
S3150800E6806E3007F1300007F118010C230822FBF75A
S3150800E69007F807F1300207F10C0311461846FAF796
S3150800E6A011FF07F130031846FAF706FE7B68DB7F91
S3150800E6B0002B04D103214C4809F0E9FC03E00121B1
S3150800E6C0494809F0E4FC97F86E309CB207F10C0350
S3150800E6D01846FAF7C7FC034600222146424809F0C5
S3150800E6E032F907F10C031846FAF7BCFC034619463B
S3150800E6F03D4809F031FA0346DAB297F86E3013440A
S3150800E70087F86E300321384809F0C1FC7B68DB7F47
S3150800E710002B15D107F13C0007F118010F230D2234
S3150800E720FAF7BEFF07F13C0207F10C03114618463B
S3150800E730FAF7C8FE07F13C031846FAF7BDFD14E0E0
S3150800E74007F1480007F118010E230C22FAF7A8FF73
S3150800E75007F1480207F10C0311461846FAF7B2FE0C
S3150800E76007F148031846FAF7A7FD97F86E309CB2EA
S3150800E77007F10C031846FAF775FC034600222146F2
S3150800E780194809F0E0F807F10C031846FAF76AFC8D
S3150800E79003461946144809F0DFF90346DAB297F832
S3150800E7A06E30134487F86E3007F1540007F11801EC
S3150800E7B013230F22FAF774FF07F1540207F10C032B
S3150800E7C011461846FAF77EFE07F154031846FAF77B
S3150800E7D073FD7B68DB7F012B16D10321024809F004
S3150800E7E056FC15E054E3060814C20120C485060841
S3150800E7F0C8850608CC850608D0850608ECDA06081A
S3150800E800D4850608D885060801212F4809F03FFC5B
S3150800E81097F86E309CB207F10C031846FAF722FCFB
S3150800E820034600222146284809F08DF807F10C0313
S3150800E8301846FAF717FC03461946234809F08CF9D7
S3150800E8400346DAB297F86E30134487F86E30032120
S3150800E8501D4809F01CFC07F1600307F11801132293
S3150800E8601846FEF7FFFD07F1600207F10C03114693
S3150800E8701846FAF727FE07F160031846FAF71CFD53
S3150800E88097F86E309CB207F10C031846FAF7EAFBC4
S3150800E8900346002221460C4809F055F806E07B6835
S3150800E8A05B6900220021084809F04DF807F10C03BE
S3150800E8B01846FAF701FD07F118031846FAF7FCFCA3
S3150800E8C000BF7437BD4690BD14C2012080B483B022
S3150800E8D000AF78600B46FB707B68FA781A7000BF49
S3150800E8E00C37BD465DF8047B704780B483B000AF33
S3150800E8F078607B681B7818460C37BD465DF8047B44
S3150800E900704780B582B000AF78607B68DB68002B03
S3150800E91007D07B68DB687868984703461A467B68A1
S3150800E9201A7000BF0837BD4680BD80B483B000AFFB
S3150800E930786039607B683A681A6300BF0C37BD4651
S3150800E9405DF8047B704780B483B000AF78607B685D
S3150800E95000221A7400BF0C37BD465DF8047B704769
S3150800E96080B483B000AF78607B6801221A7400BF58
S3150800E9700C37BD465DF8047B704780B483B000AFA2
S3150800E98078607B681B7C18460C37BD465DF8047BAF
S3150800E990704780B485B000AFF860B9601346FB7164
S3150800E9A0FB68BA689A61FB68FA791A77FB6893F884
S3150800E9B02030FA79B2FBF3F3DAB2FB689A77FB6890
S3150800E9C093F82020FB79B3FBF2F102FB01F29B1AC4
S3150800E9D0DBB2002B05D0FB689B7F0133DAB2FB68FC
S3150800E9E09A7700BF1437BD465DF8047B704780B43C
S3150800E9F083B000AF78607B689A697B6893F91D30AD
S3150800EA009B0013441B6818460C37BD465DF8047B0B
S3150800EA10704780B483B000AF78607B681B6B18467C
S3150800EA200C37BD465DF8047B704780B483B000AFF1
S3150800EA30786039607B683A689A6200BF0C37BD46D1
S3150800EA405DF8047B704780B483B000AF78607B685C
S3150800EA509B6A002B01D1002300E0012318460C37DE
S3150800EA60BD465DF8047B704780B483B000AF78601C
S3150800EA707B6800221A707B6801221A7400BF0C3763
S3150800EA80BD465DF8047B704780B584B000AFF8607A
S3150800EA90B9607A60FB680022DA60FB6801221A74A2
S3150800EAA0FB681B681B68B968F8689847FB681B68A9
S3150800EAB004331B687968F868984700BF1037BD4665
S3150800EAC080BD80B483B000AF786039603B68002BA6
S3150800EAD002D17B6801221A747B683A68DA6000BF43
S3150800EAE00C37BD465DF8047B704780B483B000AF31
S3150800EAF0786039607B683A685A6000BF0C37BD4653
S3150800EB005DF8047B704780B483B000AF78603960E5
S3150800EB107B683A689A6000BF0C37BD465DF8047B8F
S3150800EB20704780B582B000AF78607B68DB68002BE1
S3150800EB3005D07B68DB681846FEF716FD02E07B68A1
S3150800EB405B68984700BF0837BD4680BD80B582B070
S3150800EB5000AF78607B68DB68002B05D07B68DB68D4
S3150800EB601846FEF721FE02E07B689B68984700BFBF
S3150800EB700837BD4680BD80B582B000AF78607B6837
S3150800EB80DB68002B0BD07B68DB681846FFF7F5FEC1
S3150800EB9003461A467B681A747B681B7C01E07B680F
S3150800EBA01B7C18460837BD4680BD80B582B000AFCD
S3150800EBB078607B68DB68002B04D07B68DB681846C6
S3150800EBC0FFF7C1FE7B6800221A7400BF0837BD46EE
S3150800EBD080BD80B582B000AF78607B68DB68002BAB
S3150800EBE004D07B68DB681846FFF7BAFE7B6801220B
S3150800EBF01A7400BF0837BD4680BD80B483B000AF25
S3150800EC0078607B68DB6818460C37BD465DF8047B80
S3150800EC10704780B483B000AF78607B6800221A72B0
S3150800EC207B68012283F848207B68062283F88120C6
S3150800EC3000BF0C37BD465DF8047B704780B582B0CF
S3150800EC4000AF78607B689B68002B04D07B689B6864
S3150800EC501846FFF7DEFF00BF0837BD4680BD80B502
S3150800EC6082B000AF78607B685B68002B02D07B6857
S3150800EC705B6898477B681B681C331B6878689847ED
S3150800EC8000BF0837BD4680BD80B485B000AFF860C8
S3150800EC900B467A60FB7200BF1437BD465DF8047BED
S3150800ECA07047000080B582B000AF7860054A7B687F
S3150800ECB01A60786805F002FD7B6818460837BD4675
S3150800ECC080BD00BF68B6060880B483B000AF786020
S3150800ECD00B46FB701346BB70BA78FB7879689800C8
S3150800ECE01346DB00134403440B442033DA791B7ABA
S3150800ECF003F00F031B0213439BB218460C37BD469D
S3150800ED005DF8047B704780B483B000AF78600B462B
S3150800ED10FB701346BB70BA78FB787968980013467F
S3150800ED20DB00134403440B4420331A7A1209D2B287
S3150800ED305B7A1B0113439BB218460C37BD465DF838
S3150800ED40047B704780B483B000AF78600B46FB70D5
S3150800ED501346BB70BA78FB78796898001346DB00CF
S3150800ED60134403440B4420339B79C3F3C013DBB22B
S3150800ED7083F00103DBB218460C37BD465DF8047B09
S3150800ED80704780B483B000AF78600B46FB701346BB
S3150800ED90BB70BA78FB78796898001346DB00134491
S3150800EDA003440B4420339B79C3F30603DBB21846AE
S3150800EDB00C37BD465DF8047B7047000080B582B00D
S3150800EDC000AF78600B46FB70FB78012B1ED17B6881
S3150800EDD0B3F91A3007EE903AF8EEE77A7B68B3F99A
S3150800EDE0183007EE103AB8EEC77AF0EE470AB0EEDA
S3150800EDF0670A53F01DFFF0EE407A9FED167A77EE1C
S3150800EE00877A9FED157A67EE877A1DE07B68B3F9F6
S3150800EE10163007EE903AF8EEE77A7B68B3F91830C1
S3150800EE2007EE103AB8EEC77AF0EE470AB0EE670A70
S3150800EE3053F0FEFEF0EE407A9FED067A77EE877A7B
S3150800EE409FED057A67EE877AB0EE670A0837BD4602
S3150800EE5080BD00BFDB0F4940E12E654280B483B018
S3150800EE6000AF78607B6893F82130C3F30303DBB205
S3150800EE7018460C37BD465DF8047B704780B582B0EE
S3150800EE8000AF786000220021786800F01CF800BF07
S3150800EE900837BD4680BD80B582B000AF78600B46A6
S3150800EEA0FB70FB78202B05D1FF220021786800F043
S3150800EEB00AF804E00022FF21786800F004F800BF91
S3150800EEC00837BD4680BD80B483B000AF78600B4676
S3150800EED0FB701346BB707B68FA7883F846207B681C
S3150800EEE0BA7883F847207B68012283F84D2000BF53
S3150800EEF00C37BD465DF8047B704780B483B000AF1D
S3150800EF007860084611461A460346FB700B46BB70E6
S3150800EF1013467B707B68FA7883F848207B68BA7852
S3150800EF2083F849207B687A7883F84A207B6801222F
S3150800EF3083F84D2000BF0C37BD465DF8047B70474B
S3150800EF4080B582B000AF786039603B681B14D9B2CF
S3150800EF503B681B12DAB23B68DBB27868FFF7CDFF75
S3150800EF6000BF0837BD4680BD80B483B000AF786067
S3150800EF700B46FB701346BB707B68FA7883F84B2008
S3150800EF807B68BA7883F84C207B68012283F84D2089
S3150800EF9000BF0C37BD465DF8047B704780B584B06A
S3150800EFA000AFF860B9603B601346FB71F868FA7900
S3150800EFB03B68B96804F068F8FB6878331846FFF7C9
S3150800EFC071FE084AFB681A60074AFB689A67FB687D
S3150800EFD07833184605F072FBFB6818461037BD46AD
S3150800EFE080BD00BF2CB606085CB6060880B483B0A0
S3150800EFF000AF78607B685B7D18460C37BD465DF8C8
S3150800F000047B704780B584B000AFF8600B467A6021
S3150800F010FB72FB687833F97A7A68184605F089FA3C
S3150800F02000BF1037BD4680BD80B582B000AF78609E
S3150800F0307B687833184605F041FB786800F055F888
S3150800F0407B685B68002B05D17B687833FF211846FF
S3150800F050FFF776FF00BF0837BD4680BD80B582B092
S3150800F06000AF78607B687833184605F027FB00BF49
S3150800F0700837BD4680BD80B596B000AF7860396068
S3150800F08007F108034F220021184654F0EFFE5223D9
S3150800F0903B7211237B728023BB72FF233B733B6851
S3150800F0A05B78FB733B681B783B743B689B787B7487
S3150800F0B03B68DB78BB743B681B79FB743B685B7900
S3150800F0C03B753B689B797B753B680022DA7107F1D3
S3150800F0D008034F221946786800F01AF800BF583717
S3150800F0E0BD4680BDA0F17800C5E780B584B000AF05
S3150800F0F0786043233B7302237B7307F10C030222D8
S3150800F1001946786800F004F800BF1037BD4680BD80
S3150800F11090B587B002AFF860B9601346FB71FB681B
S3150800F1209868FB689989FB689B7DFA68D27DFC79AB
S3150800F130019200932346BA6803F042F800BF1437D9
S3150800F140BD4690BD80B483B000AF7860044A7B6842
S3150800F1501A607B6818460C37BD465DF8047B704715
S3150800F160DCB5060880B582B000AF786039607B6888
S3150800F1701846FFF7E7FF074A7B681A607B68181D81
S3150800F180054B00223968FFF709FF7B6818460837E0
S3150800F190BD4680BD8CB50608F085060880B582B0E8
S3150800F1A000AF7860084611461A460346FB700B46C0
S3150800F1B0BB7013467B707B6803F17C007B78BA785A
S3150800F1C0F978FFF79AFE00BF0837BD4680BD80B5BF
S3150800F1D082B000AF78600B46FB701346BB707B6845
S3150800F1E07C33BA78F9781846FFF76EFD0346184659
S3150800F1F00837BD4680BD80B582B000AF78600B4643
S3150800F200FB701346BB707B687C33BA78F97818466E
S3150800F210FFF779FD034618460837BD4680BD80B519
S3150800F22082B000AF78600B46FB707B687C33FA7857
S3150800F2301146184605F06DF9034618460837BD46C7
S3150800F24080BD80B582B000AF78600B46FB707B68E6
S3150800F2507C33FA781146184605F022F90346184613
S3150800F2600837BD4680BD80B582B000AF78600B46D2
S3150800F270FB707B687C33FA781146184605F090F8DF
S3150800F280034618460837BD4680BD80B582B000AF34
S3150800F29078600B46FB707B687C33FA781146184613
S3150800F2A005F0B4F8034618460837BD4680BD80B554
S3150800F2B082B000AF78600B46FB707B687C33FA78C7
S3150800F2C011461846FFF77AFDF0EE407AB0EE670A67
S3150800F2D00837BD4680BD80B582B000AF78600B4662
S3150800F2E0FB701346BB707B687C33BA78F97818468E
S3150800F2F0FFF747FD034618460837BD4680BD80B56B
S3150800F30082B000AF78600B46FB701346BB707B6813
S3150800F3107C33BA78F9781846FFF714FD0346184681
S3150800F3200837BD4680BD80B582B000AF78607B687F
S3150800F3307C331846FFF792FD034618460837BD4644
S3150800F34080BD80B582B000AF78607B687C33184694
S3150800F350FFF794FD00BF0837BD4680BD80B582B073
S3150800F36000AF78600B46FB707B687C33FA781146F1
S3150800F3701846FFF790FD00BF0837BD4680BD80B52B
S3150800F38082B000AF78600B46FB701346BB707B6893
S3150800F3907C33BA78F9781846FFF795FD00BF083729
S3150800F3A0BD4680BD80B582B000AF78600B46FB7065
S3150800F3B01346BB707B687C33BA78F9781846FFF732
S3150800F3C0D3FD00BF0837BD4680BD80B582B000AF0B
S3150800F3D078607B6804331846FFF708FE034618462C
S3150800F3E00837BD4680BD80B582B000AF78607B68BF
S3150800F3F00433184603F0B9FE00BF0837BD4680BD82
S3150800F40080B582B000AF78607B6804331846FFF792
S3150800F41015FC00BF0837BD4680BD80B483B000AF79
S3150800F42078607B680022DA717B6818460C37BD461F
S3150800F4305DF8047B7047000080B582B000AF786045
S3150800F440114A7B681A607B68043300221A605A6086
S3150800F4507B6804331846FFF7E0FF7B680C3300220D
S3150800F4601A605A607B680C331846FFF7D6FF7B682C
S3150800F4700022A3F84C20786805F001FC7B68184642
S3150800F4800837BD4680BD00BF00BB060880B483B000
S3150800F49000AF78600B46FB70FB787A680C339B00EC
S3150800F4A013445B68C3F30B239BB218460C37BD465F
S3150800F4B05DF8047B704780B483B000AF78600B4674
S3150800F4C0FB70FB787A680C339B001344DB88C3F324
S3150800F4D00B139BB218460C37BD465DF8047B704784
S3150800F4E080B483B000AF78600B46FB70FB787A680F
S3150800F4F00C339B0013441B79C3F3C013DBB283F0B0
S3150800F5000103DBB218460C37BD465DF8047B70472D
S3150800F51080B483B000AF78600B46FB70FB787A68DE
S3150800F5200C339B0013441B79C3F30603DBB218465E
S3150800F5300C37BD465DF8047B7047000080B582B085
S3150800F54000AF78600B46FB70FB78012B22D17B68F5
S3150800F550B3F92D301BB25B4207EE903AF8EEE77A24
S3150800F5607B68B3F92B301BB25B4207EE103AB8EE54
S3150800F570C77AF0EE470AB0EE670A53F059FBF0EE89
S3150800F580407A9FED177A77EE877A9FED167A67EEBF
S3150800F590877A20E07B68B3F929301BB207EE903AE8
S3150800F5A0F8EEE77A7B68B3F92B301BB25B4207EEBD
S3150800F5B0103AB8EEC77AF0EE470AB0EE670A53F08B
S3150800F5C037FBF0EE407A9FED067A77EE877A9FED65
S3150800F5D0057A67EE877AB0EE670A0837BD4680BDBA
S3150800F5E0DB0F4940E12E654280B582B000AF7860F6
S3150800F5F000220021786800F01CF800BF0837BD46D5
S3150800F60080BD80B582B000AF78600B46FB70FB7892
S3150800F610202B05D1FF220021786800F00AF804E0C3
S3150800F6200022FF21786800F004F800BF0837BD46BD
S3150800F63080BD80B483B000AF78600B46FB7013467C
S3150800F640BB707B68FA7883F842207B68BA7883F8BF
S3150800F65043207B68012283F84A2000BF0C37BD4649
S3150800F6605DF8047B704780B483B000AF78600846C5
S3150800F67011461A460346FB700B46BB7013467B7051
S3150800F6807B68FA7883F847207B68BA7883F848203D
S3150800F6907B687A7883F849207B68012283F84A20B8
S3150800F6A000BF0C37BD465DF8047B704780B582B055
S3150800F6B000AF786039603B681B14D9B23B681B12EF
S3150800F6C0DAB23B68DBB27868FFF7CDFF00BF0837D0
S3150800F6D0BD4680BD80B487B000AFF860B9607A6077
S3150800F6E0BB687B617B685A1E7A60002B14BF0123B6
S3150800F6F00023DBB2002B10D07B695A1C7A611B7879
S3150800F7001A46FB68DBB253409B00074A13441A6843
S3150800F710FB681B0A5340FB60E4E7FB6818461C3786
S3150800F720BD465DF8047B70476CB6060880B584B0A4
S3150800F73000AFF860B9603B601346FB71F868FA7968
S3150800F7403B68B96803F0A0FCFB6878331846FFF7F6
S3150800F75073FE0A4AFB681A60094AFB689A67FB68DF
S3150800F760002283F8C620FB687833184605F087FA26
S3150800F770FB6818461037BD4680BD00BFC4BA0608E8
S3150800F780F4BA060880B483B000AF78607B685B7D06
S3150800F79018460C37BD465DF8047B704780B584B0C3
S3150800F7A000AFF8600B467A60FB72FB687833F97A2B
S3150800F7B07A68184605F087F900BF1037BD4680BD40
S3150800F7C080B582B000AF78607B687833184605F05C
S3150800F7D056FA786800F0BFF87B685B68002B06D19C
S3150800F7E07B6878334FF47F011846FFF75FFF00BF49
S3150800F7F00837BD4680BD80B582B000AF78607B68AB
S3150800F8007833184605F03BFA00BF0837BD4680BD79
S3150800F81090B59BB002AF7860396007F10C034F22B0
S3150800F8200021184654F022FBA2233B7331237B7335
S3150800F8307B6893F8C6301B01DBB2BB737B6893F811
S3150800F840C6300133DAB27B6883F8C6207B6893F842
S3150800F850C6300F2B0CBF01230023DBB2002B03D0CD
S3150800F8607B68002283F8C6201023FB73FF233B74B2
S3150800F870F7237B743B685B78BB743B681B78FB7427
S3150800F8803B689B783B767B6803F1840207F10C039F
S3150800F8900E331946104605F07FFA7B6803F17C02A1
S3150800F8A007F10C0319331946104605F075FA0323B8
S3150800F8B087F836303B68DB78002B01D0012300E05F
S3150800F8C0022387F839303B681B7987F83B303B6859
S3150800F8D05B7987F83C303B689B7987F83D303B6815
S3150800F8E0DB7987F83E3007F10C034B2219464FF0B7
S3150800F8F0FF30FFF7EFFE0346DB43FB65FB6DDBB22C
S3150800F90087F85730FB6D1B0ADBB287F85830FB6D5A
S3150800F9101B0CDBB287F85930FB6D1B0EDBB287F880
S3150800F9205A303B6800221A727B6898687B68998906
S3150800F9307B681B7E7A68527E07F10C04019200935D
S3150800F9404F23224602F03CFC00BF6437BD4690BDFB
S3150800F950A0F178005CE790B587B002AF78604323E2
S3150800F9603B7309237B737B6898687B6899897B68F6
S3150800F9709B7D7A68D27D07F10C04019200930223DD
S3150800F980224602F01DFC00BF1437BD4690BD00009C
S3150800F99080B582B000AF786039607B681846FFF79B
S3150800F9A0D1FB074A7B681A607B68181D054B002245
S3150800F9B03968FFF7BBFE7B6818460837BD4680BD29
S3150800F9C074BA0608F885060880B582B000AF786074
S3150800F9D0084611461A460346FB700B46BB7013468B
S3150800F9E07B707B6803F17C007B78BA78F978FFF73F
S3150800F9F03AFE00BF0837BD4680BD80B582B000AF6D
S3150800FA0078600B46FB701346BB707B687C33FA78CC
S3150800FA1011461846FFF73AFD034618460837BD460D
S3150800FA2080BD80B582B000AF78600B46FB70134688
S3150800FA30BB707B687C33FA7811461846FFF73BFDA6
S3150800FA40034618460837BD4680BD80B582B000AF6C
S3150800FA5078600B46FB707B687C33FA78114618464B
S3150800FA6005F021F8034618460837BD4680BD80B51F
S3150800FA7082B000AF78600B46FB707B687C33FA78FF
S3150800FA801146184604F0D6FF034618460837BD4601
S3150800FA9080BD80B582B000AF78600B46FB707B688E
S3150800FAA07C33FA781146184604F042FF0346184696
S3150800FAB00837BD4680BD80B582B000AF78600B467A
S3150800FAC0FB707B687C33FA781146184604F068FFA9
S3150800FAD0034618460837BD4680BD80B582B000AFDC
S3150800FAE078600B46FB707B687C33FA7811461846BB
S3150800FAF0FFF724FDF0EE407AB0EE670A0837BD46F8
S3150800FB0080BD80B582B000AF78600B46FB701346A7
S3150800FB10BB707B687C33FA7811461846FFF7F8FC09
S3150800FB20034618460837BD4680BD80B582B000AF8B
S3150800FB3078600B46FB701346BB707B687C33FA789B
S3150800FB4011461846FFF7CCFC034618460837BD464B
S3150800FB5080BD80B483B000AF78600F2318460C3799
S3150800FB60BD465DF8047B704780B582B000AF78600B
S3150800FB707B687C331846FFF737FD00BF0837BD465C
S3150800FB8080BD80B582B000AF78600B46FB707B689D
S3150800FB907C33FA7811461846FFF733FD00BF08375D
S3150800FBA0BD4680BD80B582B000AF78600B46FB705D
S3150800FBB01346BB707B687C33BA78F9781846FFF72A
S3150800FBC038FD00BF0837BD4680BD80B483B000AF9E
S3150800FBD078600B46FB701346BB7000BF0C37BD46FA
S3150800FBE05DF8047B704780B582B000AF78607B68AB
S3150800FBF004331846FFF7C6FD034618460837BD46C0
S3150800FC0080BD80B582B000AF78607B680433184643
S3150800FC1003F0ABFA00BF0837BD4680BD80B582B099
S3150800FC2000AF78607B6804331846FFF707F800BF13
S3150800FC300837BD4680BD80B483B000AF78603960B0
S3150800FC407B683A685A6000BF0C37BD465DF8047B8E
S3150800FC507047000098B500AF0F4B1B78002B0AD1F0
S3150800FC600E4B18680D4B1B681B681C68FF23002287
S3150800FC700021A0470DE0084B1B78012B09D1084B42
S3150800FC801868074B1B681B681C680023FF220021A5
S3150800FC90A04700BF98BD00BF2D10002034100020DB
S3150800FCA03810002090B583B000AF0346FB711E4A9A
S3150800FCB0FB791370FB79002B16D1CC2052F0BEFECF
S3150800FCC003461C46194B1B6819462046FFF74AFA95
S3150800FCD0174B1C60164B1B68043316491846FFF76A
S3150800FCE0AAFF134B1B681AE0FB79012B16D1CC200F
S3150800FCF052F0A4FE03461C460C4B1B6819462046C8
S3150800FD00FFF746FE0C4B1C600B4B1B680433094976
S3150800FD101846FFF790FF084B1B6800E000231846BB
S3150800FD200C37BD4690BD00BF2D10002030100020B6
S3150800FD303410002055FC00083810002080B483B029
S3150800FD4000AF78603960064B00221A70054A3B6896
S3150800FD5013607B6818460C37BD465DF8047B704710
S3150800FD602D1000203010002080B483B000AF7860DA
S3150800FD707B6818460C37BD465DF8047B704780B42F
S3150800FD8083B000AF7860084611461A460346FB70F2
S3150800FD900B46BB7013467B70002318460C37BD46CE
S3150800FDA05DF8047B704780B483B000AF786008467E
S3150800FDB011461A460346FB700B46BB7013467B700A
S3150800FDC0002318460C37BD465DF8047B704780B49F
S3150800FDD083B000AF7860002318460C37BD465DF83F
S3150800FDE0047B704780B483B000AF78600023184660
S3150800FDF00C37BD465DF8047B704780B483B000AF0E
S3150800FE007860002318460C37BD465DF8047B7047BA
S3150800FE1080B483B000AF78600B46FB7000BF0C3728
S3150800FE20BD465DF8047B704780B483B000AF786048
S3150800FE300B467B8013463B80002318460C37BD468D
S3150800FE405DF8047B704780B483B000AF78600B46DA
S3150800FE50FB70002318460C37BD465DF8047B7047D7
S3150800FE6080B483B000AF78600B46FB700123184658
S3150800FE700C37BD465DF8047B704780B483B000AF8D
S3150800FE8078607B6818460C37BD465DF8047B70477A
S3150800FE9080B485B000AF786039600023FB73FB7BC4
S3150800FEA00F2B12D8FA7B7B681E3253F82230002BB0
S3150800FEB007D1FA7B7B681E32396843F82210002383
S3150800FEC004E0FB7B0133FB73E9E7D32318461437B9
S3150800FED0BD465DF8047B704780B483B000AF786098
S3150800FEE0044A7B681A607B6818460C37BD465DF87D
S3150800FEF0047B70470CBB060880B483B000AF7860FB
S3150800FF007B6800221A707B6800225A7000229A7059
S3150800FF100022DA7000221A717B6818460C37BD4633
S3150800FF205DF8047B704780B483B000AF78607B6867
S3150800FF3000221A607B6800221A717B6800225A71B7
S3150800FF407B6818460C37BD465DF8047B704780B45D
S3150800FF5083B000AF786039603B68D3F801207B68CE
S3150800FF601A603B681A787B685A717B685A797B688D
S3150800FF701A7100BF0C37BD465DF8047B704780B424
S3150800FF8083B000AF78607B6800221A607B68002225
S3150800FF901A717B680022DA807B6818460C37BD46E2
S3150800FFA05DF8047B704780B483B000AF7860396031
S3150800FFB03B68D3F801207B681A607B680022DA80E8
S3150800FFC000BF0C37BD465DF8047B704780B485B02A
S3150800FFD000AFF860B9607A607B80FB681B79002BFC
S3150800FFE002D0012B09D029E0FB687A88DA80FB6801
S3150800FFF01B790133DAB2FB681A71FB68DB88002BC0
S3150801000015D07B681B88002B11D0FB68DB88013B68
S315080100109AB2FB68DA80BB681B685A1CBB681A600F
S315080100207B681B88013B9AB27B681A80E5E7FB6807
S31508010030DB88002B02D1FB6800221A71FB68DB887A
S31508010040002B0CBF01230023DBB218461437BD462B
S315080100505DF8047B704780B483B000AF78600846CA
S3150801006011461A460346FB700B46BB7013467B7056
S3150801007000BF0C37BD465DF8047B704780B483B07A
S3150801008000AF7860044A7B681A607B6818460C37AB
S31508010090BD465DF8047B704790BB060880B483B003
S315080100A000AF78607B6893F8503018460C37BD4628
S315080100B05DF8047B704780B483B000AF78607B68D5
S315080100C093F87A3018460C37BD465DF8047B7047BD
S315080100D080B483B000AF78600B46FB70FB78E02BE9
S315080100E00CBF01230023DBB218460C37BD465DF869
S315080100F0047B704780B483B000AF78600B467B8081
S3150801010013463B807B8840F65C22934204D13B88A8
S3150801011042F2E812934209D07B8840F20D5293428B
S3150801012006D13B8840F25A62934201D101232DE060
S315080101307B681B7D002B13D17B685B7D002B0FD160
S315080101407B689B7D002B0BD17B68DB7D002B07D160
S315080101507B681B7E002B03D17B685B7E002B14D04A
S315080101607B8840F24C5293420FD13B88B3F51A7FF4
S3150801017009D03B8840F22F42934204D03B8840F293
S31508010180D532934201D1012300E0002318460C37EA
S31508010190BD465DF8047B704780B584B000AF7860D2
S315080101A039607B681846FFF797FE7B680433184663
S315080101B0FFF764FF2B4A7B681A602B4A7B685A60F3
S315080101C07B68002283F841207B68002283F843205C
S315080101D07B68002283F846207B68002283F8482042
S315080101E07B68002283F849207B683A68DA647B6871
S315080101F0002283F850207B68012283F85E207B6801
S3150801020000221A667B68002283F878207B68002220
S3150801021083F879207B68002283F87A200023FB7310
S31508010220FB7B032B0AD8FB7B7A6818339B001344A4
S3150801023000225A60FB7B0133FB73F1E7786800F013
S315080102407DFA7B68DB6C002B06D07B68DB6C7A68F1
S3150801025011461846FFF71CFE7B6818461037BD463F
S3150801026080BD00BF50BB060884BB060890B58FB099
S3150801027002AF7860084611461A460346FB700B46DC
S31508010280BB7013467B70122387F82E3007F10803DB
S31508010290BB6200237B6200233B62786800F04EFA5A
S315080102A07B68DB6C1846FFF7E8FDF8617B6893F815
S315080102B05030002B01D0D92387E0FB691B681B68E6
S315080102C00021F869984778627B6A002B01D1D62309
S315080102D07BE07B6A1B68002B01D1D72375E07B6A1B
S315080102E01B683B627B6803F151027B6A1A607B6A71
S315080102F07A789A717B68D86C07F108030093122300
S315080103000022002105F02FFF034687F82F307B6A6C
S315080103103A6A1A6097F82F30002B46D1FB691B6899
S3150801032004331C68BB78F9780022F869A0470346AC
S315080103301A467B6883F850207B6893F85030002B67
S3150801034001D1D42341E0BB6A1B79092B17D0BB6ABB
S31508010350DA797B6883F85220BB6A5A7C7B6883F812
S315080103605420BB6A1B899AB27B68A3F87620BB6ABC
S315080103705B899AB27B68A3F87420E02325E000BF65
S315080103807B68D86C7B6893F850100023002205F02F
S3150801039087FFD12387F82F307B681B6808331B68D2
S315080103A07868984797F82F300FE000BF97F82F30F5
S315080103B00D2B02D0E12387F82F307B681B680833A1
S315080103C01B687868984797F82F3018463437BD4622
S315080103D090BD80B596B002AF7860084611461A46B8
S315080103E00346FB700B46BB7013467B707B6893F81C
S315080103F0543087F84D307B68002283F854207B6897
S31508010400DB6C1846FFF739FDB864BB6C1B681B68C3
S315080104107A6892F850201146B86C984778647B6CD4
S31508010420002B01D1D62385E14FF4967040F07AFC72
S315080104307B68D86C7B6893F850300022002105F060
S315080104402FFF034687F84F3097F84F30002B03D01C
S315080104507B6C00229A7165E17B6C00229A71BB6CF8
S315080104601B681B687A6892F850201146B86C984741
S3150801047078647B6C002B01D1D6235BE17B6C7A789F
S315080104809A717B68D86C7B6893F850107B685133F6
S31508010490012204F0EEFD034687F84F3097F84F30F6
S315080104A0002B40F028817B68B3F8763040F24C5235
S315080104B0934277D17B68B3F87430B3F51A7F0DD0C0
S315080104C07B68B3F8743040F22F42934206D07B68BA
S315080104D0B3F8743040F2D532934263D1642040F0C8
S315080104E021FC7B68D86C7B6893F850107B6893F87D
S315080104F05120012305F002FF034687F84F3097F88C
S315080105004F30002B40F0F9807B681B7D002B13D1FF
S315080105107B685B7D002B0FD17B689B7D002B0BD104
S315080105207B68DB7D002B07D17B681B7E002B03D103
S315080105307B685B7E002B19D07B68B3F87430B3F502
S315080105401A7F06D07B68B3F8743040F22F42934283
S3150801055006D17B6814331946786802F0B0F805E0CD
S315080105607B6814331946786802F0E9F87B68D86C19
S315080105707B6893F850107B6893F85120002305F0A7
S31508010580BDFE7B68D86C7B6893F850100023002267
S3150801059005F086FE7B681B6808331B6878689847F0
S315080105A0D123C7E0002387F84E3097F84E2097F8F5
S315080105B04D309A425ED27B68B3F8763040F65C22BB
S315080105C0934206D17B68B3F8743042F2E81293423B
S315080105D00DD07B68B3F8763040F20D52934220D1A4
S315080105E07B68B3F8743040F25A62934219D17B683A
S315080105F01A1D07F108031146184602F0F3F87B683D
S31508010600D86C7B6893F8501097F84E2007F10803C9
S3150801061000931346002205F0F6FD034687F84F308E
S3150801062018E07B681A1D07F108031146184602F0FF
S3150801063027F97B68D86C7B6893F8501097F84E2099
S3150801064007F1080300931346002205F0DCFD034673
S3150801065087F84F3097F84F30002B50D17B6893F8C5
S315080106605E30032B05D897F84E30013387F84E30A4
S315080106709BE700BF7B6893F85E30032B45D97B68FF
S31508010680D86C7B6893F850107B6893F85E207B687A
S31508010690513304F0EEFC034687F84F3097F84F3094
S315080106A0002B2ED17B68D86C7B6893F850107B6839
S315080106B093F851207B6893F85D3005F01FFE0346D9
S315080106C087F84F3097F84F30002B1CD17B6864228E
S315080106D0A3F884207B680022A3F882207B68002285
S315080106E083F881207B6800221A727B68012283F8CD
S315080106F07A2000231EE000BF14E000BF12E000BF0D
S3150801070010E000BF0EE000BF0CE000BF7B68D86CAC
S315080107107B6893F850100023002205F0C1FDD12310
S3150801072087F84F307B681B6808331B6878689847D9
S3150801073097F84F3018465037BD4680BD80B584B00E
S3150801074000AF78600023FB73FB7B032B45D8FA7B4C
S31508010750796813465B0013440B44513300221A701F
S31508010760FB7B002B01D0002000E00820FA7B79688A
S3150801077013465B0013440B44523302461A70FA7B44
S31508010780796813465B0013440B4403F15002D3788E
S315080107906FF30003D370FA7B796813465B00134441
S315080107A00B4403F15002D3786FF34103D370FB7BFB
S315080107B0002B01D0012100E00F21FA7B786813464E
S315080107C05B001344034403F15002D37861F38703B2
S315080107D0D370FB7B0133FB73B6E70023FB73FB7B0B
S315080107E0032B1CD8FB7B7A6818339B0013445B6880
S315080107F0002B10D0FB7B7A6818339B001344596889
S31508010800FB7B7A6818339B0013445B681B680833C3
S315080108101B6808469847FB7B0133FB73DFE77B6858
S31508010820002283F841207B68002283F842207B68F6
S31508010830002283F846207B68002283F847207B68DC
S31508010840002283F87D207B68002283F850207B688C
S31508010850012283F85E207B6800221A667B680022E3
S3150801086083F878207B68002283F87A207B68002247
S3150801087083F8792000BF1037BD4680BD80B485B0A6
S3150801088000AF7860084611461A460346FB700B46C8
S31508010890BB7013467B707B78002B5DD17B68FA7839
S315080108A083F85D20FB69DB7803F00303032B14D17E
S315080108B0FB699B785BB2002B0FDA0123FB73FA7B8A
S315080108C0796813465B0013440B4403F15002D3784D
S315080108D0012161F38703D3700EE0FB69DB7803F02E
S315080108E00303022B3AD1FB699B785BB2002B01DA31
S315080108F0022300E00323FB73FB699B78FA7B03F071
S315080109000F03D8B2796813465B0013440B4451337D
S3150801091002461A70FB699B889BB2FA7BD8B2796842
S3150801092013465B0013440B44523302461A707B6824
S3150801093093F87820FB699B799A4204D2FB699A79E4
S315080109407B6883F878207B6893F85E300133DAB2E6
S315080109507B6883F85E2002E000BF00E000BF143721
S31508010960BD465DF8047B7047A0F10400FFF786BF1A
S3150801097080B582B000AF78607868FFF7DFFE7B68E4
S31508010980DB6C1846FFF779FA03461A6808321268CB
S31508010990796891F850101846904700231846083789
S315080109A0BD4680BD80B582B000AF78607B6893F89C
S315080109B07A3083F00103DBB2002B01D000231DE05E
S315080109C040F0A4F902467B681B6ED31ADB43DB0FA2
S315080109D0DBB2002B11D040F099F902467B6893F8F7
S315080109E078301A447B681A66786800F00BF87868DC
S315080109F000F022FB786800F04BFE00231846083702
S31508010A00BD4680BDB0B588B002AF78604023BB81D2
S31508010A107B68D86C7B6893F850107B6893F85440D0
S31508010A207B6889337A6892F8782007F10C05019278
S31508010A3000932B46224604F084FC0346FB73FB7B9A
S31508010A40002B03D0FB7B042B40F0F1827B6893F8E3
S31508010A508930013B352B00F2EA8201A252F823F0D4
S31508010A60410C0108A10C0108F90D0108E30E010862
S31508010A70550E0108A10F0108870E01081910010872
S31508010A80191001082F1001082F1001081910010863
S31508010A9019100108390B0108191001082F1001084E
S31508010AA02F10010819100108191001082F10010843
S31508010AB02F1001086F0F0108990F01081910010875
S31508010AC01910010819100108191001082F10010839
S31508010AD02F1001082F1001082F10010819100108FD
S31508010AE02F1001082F1001082F1001082F100108D7
S31508010AF02F1001082F1001082F1001082F100108C7
S31508010B002F1001082F1001082F1001082F100108B6
S31508010B102F1001082F1001082F1001082F100108A6
S31508010B200910010819100108111001082F100108F0
S31508010B302F100108191001087B6893F88E30002BD5
S31508010B4040F06C827B68B3F8863043F001039AB2B1
S31508010B507B68A3F886207B6893F88C30012B14D127
S31508010B607B6893F88D30102B0FD17B6893F88F2013
S31508010B707B6883F840207B68B3F8863043F04003EE
S31508010B809AB27B68A3F8862059E07B6893F88C3083
S31508010B90042B2AD17B6893F88D30102B25D17B68DD
S31508010BA0B3F8863003F40073002B14D17B6893F8ED
S31508010BB08F30002B0FD17B6893F8973003F0080329
S31508010BC0002B04D07B68012283F8792003E07B6837
S31508010BD0002283F879207B68B3F8863043F40073E2
S31508010BE09AB27B68A3F8862029E07B6893F88C3053
S31508010BF0092B40F013827B6893F88D30102B40F057
S31508010C000D820023FB75FB7D052B0ED8FB7D9A1DF6
S31508010C10FB7D79680A4492F889107A6813440A4672
S31508010C201A75FB7D0133FB75EDE77B68B3F88630F2
S31508010C3043F020039AB27B68A3F88620EEE1EDE142
S31508010C407B6893F88830042B21D97B6893F8433065
S31508010C50002B04D17B6893F84830002B17D07B68AA
S31508010C60002283F888207B68002283F841207B686C
S31508010C70002283F843207B68002283F846207B689C
S31508010C80002283F848207B680A2283F881207B6842
S31508010C9093F888300133DAB27B6883F88820C6E195
S31508010CA07B6893F88B30002B00F0BA810023BB7563
S31508010CB07B6893F88B30BA7D9A4280F0B1817B6864
S31508010CC093F88B30DB00DAB2BB7D194649000B4439
S31508010CD0DBB21344BB7300237B757B7D022B11D8D2
S31508010CE07B7D1A1DBB7B1A447B7D79680A4492F881
S31508010CF089107A6813440A4683F87E207B7D01337E
S31508010D007B75EAE77B6893F84330002B38D07B681C
S31508010D1093F88030002B33D17B6893F87F30052B0D
S31508010D202ED17B6893F87E3003F00C03002B27D075
S31508010D307B68012283F87C2000233B753B7D052BCC
S31508010D4014D83B7DD91CBA7D13465B0013445B005E
S31508010D50CA183B7D79680A4492F889107A6813445F
S31508010D600A461A773B7D01333B75E7E77B68B3F89B
S31508010D70863043F080039AB27B68A3F886203AE06E
S31508010D807B6893F84830002B31D07B6893F87F3025
S31508010D9003F00F03052B2AD17B6893F87E3003F005
S31508010DA0C803002B23D00023FB74FB7C052B14D826
S31508010DB0FB7CD91CBA7D13465B0013445B00CA1839
S31508010DC0FB7C79680A4492F889107A6813440A46C2
S31508010DD01A77FB7C0133FB74E7E77B68B3F8863047
S31508010DE043F080039AB27B68A3F8862003E0BB7DB3
S31508010DF00133BB755CE713E17B68B3F8863043F4CE
S31508010E0080739AB27B68A3F886207B6893F88B3047
S31508010E10002B1AD17B6893F88C301AB27B6893F849
S31508010E208D301B021BB203F470631BB213431BB252
S31508010E309AB27B685A837B68B3F8863043F002031B
S31508010E409AB27B68A3F88620F1E07B68062283F8CC
S31508010E508120ECE07B6893F88B30002B40F0E28030
S31508010E607B68B3F8863043F004039AB27B68A3F82B
S31508010E7086207B68B3F8863023F002039AB27B6832
S31508010E80A3F88620CEE07B6893F88B30002B40F0E0
S31508010E90CB800023BB74BB7C1D2B18D8BB7C03F10C
S31508010EA00902BB7C79680A4492F889107A68134466
S31508010EB00A4683F82220BB7C7A68134493F82230C9
S31508010EC0002B03D0BB7C0133BB74E4E700BF7B680E
S31508010ED0B3F8863043F008039AB27B68A3F88620F4
S31508010EE0A2E000237B747B7C052B0ED87B7C9A1CA5
S31508010EF07B7C79680A4492F889107A6813440A4611
S31508010F001A777B7C01337B74EDE700233B743B7CCA
S31508010F10022B10D83B7C03F108023B7C79680A4412
S31508010F2092F889107A6813440A4683F87E203B7C36
S31508010F3001333B74EBE77B6893F87F3003F00F03CB
S31508010F40052B0AD17B6893F87E3003F0C803002B82
S31508010F5003D07B68012283F847207B68B3F8863083
S31508010F6043F010039AB27B68A3F886205FE07B689A
S31508010F7093F84330002B03D0786800F0ECFE56E076
S31508010F807B681B69002B03D0786800F0E4FE4EE00D
S31508010F90786800F093FF4AE0786800F0CAFF46E0F7
S31508010FA07B6893F88B30002B23D17B6893F8433009
S31508010FB0002B0CD07B6893F8413083F00103DBB238
S31508010FC0002B04D07B68012283F841202EE07B6840
S31508010FD093F84830002B29D07B6893F8463083F084
S31508010FE00103DBB2002B21D07B68012283F846205E
S31508010FF01CE07B685B8B1946786801F082F87B6890
S31508011000102283F8812011E0786800F0CDFF0EE008
S31508011010786801F010F80AE000BF08E000BF06E0B2
S3150801102000BF04E000BF02E000BF00E000BF00BF50
S315080110301837BD46B0BD00BF80B582B000AF786035
S315080110407B6893F88130132B00F2EF8201A252F8E4
S3150801105023F000BFA5100108DF100108651101087A
S3150801106085110108A5110108F91101089F12010846
S31508011070CD120108071301082F130108651301088A
S31508011080C313010801140108271501082B160108C5
S315080110906D1501089B1501082F1201086512010833
S315080110A0851201087B68B3F8823001339AB27B68EE
S315080110B0A3F882207B68B3F882207B68B3F8843072
S315080110C09A4240F2B482786800F07DFB7B6801227F
S315080110D083F881207B680022A3F88220A7E27B6837
S315080110E0B3F8823001339AB27B68A3F882207B6811
S315080110F0B3F8863003F00103002B0BD07B6800227E
S31508011100A3F882207B68022283F88120786801F09F
S3150801111030F88EE27B68B3F882207B68B3F88430B6
S315080111209A4240F286827B68B3F884301A46920066
S3150801113013445B009AB27B68A3F884207B68B3F8F2
S315080111408430B3F5FA6F04D97B684FF4FA62A3F8D1
S3150801115084207B68002283F881207B680022A3F81B
S31508011160822066E27B68B3F8863003F00103002B20
S3150801117000F061827B68032283F88120786800F099
S3150801118072FB58E27B68B3F8863003F02003002B24
S3150801119000F05382786800F08AFB7B68042283F8A2
S315080111A081204AE27B68B3F8863003F04003002BBE
S315080111B000F045827B68DB68002B0AD07B68DB6818
S315080111C01946786800F05DFC7B68052283F8812062
S315080111D035E27B6893F84930002B08D000217868FE
S315080111E000F089FB7B68112283F8812027E27B685E
S315080111F0062283F8812022E27B68B3F8863003F061
S315080112000103002B00F01D827B6893F84930002BFF
S3150801121008D00021786800F06EFB7B68112283F8FC
S3150801122081200EE27B68062283F8812009E27B6829
S31508011230B3F8863003F40073002B00F004827B6850
S3150801124093F87930002B08D00121786800F09DFCCD
S315080112507B68122283F88120F5E17B68062283F8F0
S315080112608120F0E17B68B3F8863003F00103002B97
S3150801127000F0EB81786800F04DFC7B68132283F857
S315080112808120E2E17B68B3F8863003F00103002B85
S3150801129000F0DD817B68062283F88120D7E17B682F
S315080112A093F84830002B04D17B6893F84330002B20
S315080112B007D0786800F08FFC7B68072283F88120C5
S315080112C0D8E17B680A2283F88120D3E17B68B3F8E9
S315080112D0863003F08003002B00F0BB81786800F0AC
S315080112E0B2FC7B6893F87C30002B07D0786800F055
S315080112F074FB7B680C2283F88120AAE17B680822AB
S3150801130083F88120A5E17B68B3F8863003F00103F1
S31508011310002B00F0A0817B68002283F87C20786886
S3150801132000F0ACFC7B68092283F8812093E17B6895
S31508011330B3F8863003F48073002B00F08E817B6846
S31508011340B3F8863003F00203002B07D0786800F063
S31508011350ADFE7B680A2283F881207EE1786800F079
S315080113608DFC7AE17B6893F8413083F00103DBB2A7
S31508011370002B00F074817B6893F8433083F00103F6
S31508011380DBB2002B00F06B817B6893F8463083F063
S315080113900103DBB2002B00F062817B6893F84830C9
S315080113A083F00103DBB2002B00F05981786800F065
S315080113B029FA7B6801221A727B680B2283F881203D
S315080113C04DE17B68B3F8863003F01003002B0AD091
S315080113D07B6800221A72786800F0FFFA7B680C2293
S315080113E083F881203DE17B68B3F8863003F0040376
S315080113F0002B00F036817B68102283F8812030E1CA
S315080114007B68B3F8863003F00803002B00F02B81C4
S315080114107B68223308229949184653F02FFB034665
S31508011420002B47D17B68012283F842207B68002282
S3150801143083F844207B68002283F845207B680022D4
S3150801144083F87B207B68223316228D49184653F090
S3150801145015FB0346002B04D17B68012283F844203F
S3150801146028E07B68223316228649184653F006FB84
S315080114700346002B10D17B68012283F87B207B6809
S3150801148093F87B207B6883F844207B6893F8442093
S315080114907B6883F845200DE07B68223313227A495D
S315080114A0184653F0EBFA0346002B03D17B68012259
S315080114B083F87B207B6893F88030002B17D17B68F3
S315080114C093F87F30252B12D17B6893F87E30082B51
S315080114D00DD17B68223313226C49184653F0CEFA94
S315080114E00346002B03D17B68012283F87D207B68A4
S315080114F093F84330002B04D17B6893F84830002BCE
S3150801150009D07B6893F87C30002B04D07B680822CD
S3150801151083F88120A7E0786800F017FA7B680D2226
S3150801152083F881209FE07B68B3F8863003F00203D5
S31508011530002B00F09A807B6893F87D30002B03D04E
S315080115407B68012283F846207B6800225A727B68F1
S3150801155000229A727B680022DA727B680022A3F85D
S3150801156086207B680F2283F881207EE07B68B3F8AA
S31508011570823001339AB27B68A3F882207B68B3F87C
S315080115808230B3F57A7F72D97B680022A3F882206C
S315080115907B680A2283F8812069E07B68B3F8863084
S315080115A003F00403002B64D07B680022A3F886208D
S315080115B07B68893340220021184652F057FC7B6824
S315080115C0C93340220021184652F050FC7B6800229C
S315080115D083F843207B6893F843207B6883F842208D
S315080115E07B6893F842207B6883F841207B68002258
S315080115F083F87C207B6893F87C207B6883F84820F5
S315080116007B6893F848207B6883F847207B6893F8C2
S3150801161047207B6883F846207B68002283F87D2073
S315080116207B680A2283F8812023E000BF22E000BFFD
S3150801163020E000BF1EE000BF1CE000BF1AE000BFAB
S3150801164018E000BF16E000BF14E000BF12E000BFBB
S3150801165010E000BF0EE000BF0CE000BF0AE000BFCB
S3150801166008E000BF06E000BF04E000BF02E000BFDB
S3150801167000E000BF00BF0837BD4680BD00860608EA
S315080116800C860608248606083C860608508606083F
S31508011690B0B586B002AF786040237B817B68D86C91
S315080116A07B6893F850107B6893F857407B68C93379
S315080116B07A6892F8782007F10A05019200932B4679
S315080116C0224603F03EFE03467B737B7B002B25D126
S315080116D07B89002B22D00023FB73FB7B032B1DD8B0
S315080116E0FB7B7A6818339B0013445B68002B11D087
S315080116F0FB7B7A6818339B0013445868FB7B7A682E
S3150801170018339B0013445B681B681B687A68C932E7
S3150801171011469847FB7B0133FB73DEE70023BB7356
S31508011720BB7B032B1CD8BB7B7A6818339B001344FD
S315080117305B68002B10D0BB7B7A6818339B00134477
S315080117405968BB7B7A6818339B0013445B681B682E
S3150801175004331B6808469847BB7B0133BB73DFE735
S3150801176000BF1037BD46B0BD80B58CB008AFF86074
S31508011770B9601346FB80FB68B3F8863023F0010392
S315080117809AB2FB68A3F88620FB68D86CFB6893F8C5
S315080117905010FB6893F8512000230793BB68069302
S315080117A0FB880593FB880493002303930023029384
S315080117B00023019300230093202303F0EAFC00BFD2
S315080117C01037BD4680BD80B582B000AF78607B68B2
S315080117D00022A3F886207B68032283F889207B6888
S315080117E00C2283F88A207B68002283F88B207B6889
S315080117F08933032219467868FFF7B6FF00BF083711
S31508011800BD4680BD80B582B000AF78607B68B3F80D
S31508011810863023F010039AB27B68A3F886207B688A
S315080118201A2283F889207B680C2283F88A207B6830
S31508011830012283F88B207B68DB68002B04D07B6848
S31508011840032283F88C2003E07B68022283F88C202C
S315080118507B688933042219467868FFF785FF00BF3C
S315080118600837BD4680BD80B582B000AF78607B6819
S31508011870B3F8863023F020039AB27B68A3F8862052
S315080118807B68092283F889207B68102283F88A20DD
S315080118907B68002283F88B207B68893303221946EB
S315080118A07868FFF761FF00BF0837BD4680BD80B580
S315080118B082B000AF78607B68B3F8863023F04003C6
S315080118C09AB27B68A3F886207B68012283F889206F
S315080118D07B68102283F88A207B68002283F88B2094
S315080118E07B688933032219467868FFF73DFF00BFF5
S315080118F00837BD4680BD80B582B000AF78600B461B
S31508011900FB707B68B3F8863023F400739AB27B6860
S31508011910A3F886207B68042283F889207B68102235
S3150801192083F88A207B68012283F88B207B68FA7802
S3150801193083F88C207B688933042219467868FFF777
S3150801194013FF00BF0837BD4680BD80B582B000AF22
S3150801195078607B68B3F8863023F002039AB27B6815
S31508011960A3F886207B68092283F889207B680422EC
S3150801197083F88A207B68072283F88B207B681A7F85
S315080119807B6883F88C207B685A7F7B6883F88D2077
S315080119907B689A7F7B6883F88E207B68DA7F7B6811
S315080119A083F88F207B6893F820207B6883F8902042
S315080119B07B6893F821207B6883F891207B68002255
S315080119C083F892207B6889330A2219467868FFF7DB
S315080119D0CBFE00BF0837BD4680BD80B582B000AFDB
S315080119E078607B68B3F8863023F008039AB27B687F
S315080119F0A3F886207B68192283F889207B6804224C
S31508011A0083F88A207B680A2283F88B207B681A7FF1
S31508011A107B6883F88C207B685A7F7B6883F88D20E6
S31508011A207B689A7F7B6883F88E207B68DA7F7B6880
S31508011A3083F88F207B6893F820207B6883F89020B1
S31508011A407B6893F821207B6883F891207B680122C3
S31508011A5083F892207B68002283F893207B68002212
S31508011A6083F894207B68002283F895207B68893364
S31508011A700D2219467868FFF777FE00BF0837BD467D
S31508011A8080BD90B585B000AF786039607B68132258
S31508011A9083F889207B680C2283F88A203868F6F750
S31508011AA0C1FB0346DBB20133DAB27B6883F88B20CC
S31508011AB00023FB73FC7B3868F6F7B4FB03469C42AC
S31508011AC00ED2FB7B3A681A44FB7B033311787A689A
S31508011AD013440A4683F88920FB7B0133FB73E9E744
S31508011AE0FB7B03337A681344002283F889207B68D9
S31508011AF003F189043868F6F795FB03469BB204336C
S31508011B009BB21A4621467868FFF72EFE00BF1437A6
S31508011B10BD4690BD80B582B000AF78607B68012272
S31508011B2083F889207B680C2283F88A207B6808223F
S31508011B3083F88B207B68FF2283F88C207B68FF2241
S31508011B4083F88D207B68FF2283F88E207B68FF222D
S31508011B5083F88F207B68FF2283F890207B681F22F9
S31508011B6083F891207B68FF2283F892207B68002204
S31508011B7083F893207B6889330B2219467868FFF727
S31508011B80F3FD00BF0837BD4680BD80B582B000AF02
S31508011B9078600B46FB707B68562283F889207B6840
S31508011BA00C2283F88A207B68012283F88B20FB7834
S31508011BB0002B01D0012200E000227B6883F88C20EB
S31508011BC07B688933042219467868FFF7CDFD00BF83
S31508011BD00837BD4680BD80B582B000AF78607B68A6
S31508011BE0B3F8863023F080039AB27B68A3F886207F
S31508011BF07B68012283F889207B68042283F88A207E
S31508011C007B68052283F88B207B68332283F88C2036
S31508011C107B688B2283F88D207B689E2283F88E2031
S31508011C207B68302283F88F207B680A2283F890200C
S31508011C307B688933082219467868FFF795FD00BF46
S31508011C400837BD4680BD80B582B000AF78607B6835
S31508011C50022283F889207B68042283F88A207B681C
S31508011C60002283F88B207B6889330322194678681A
S31508011C70FFF77AFD00BF0837BD4680BD80B582B043
S31508011C8000AF78607B681C331946786800F004F861
S31508011C9000BF0837BD4680BD80B582B000AF786009
S31508011CA039607B68B3F8863023F481739AB27B680E
S31508011CB0A3F886207B68052283F889207B6804229D
S31508011CC083F88A207B680D2283F88B203B681A7873
S31508011CD07B6883F88C203B685A787B6883F88D206B
S31508011CE03B689A787B6883F88E203B68DA787B684C
S31508011CF083F88F203B681A797B6883F890203B68C4
S31508011D005A797B6883F891207B68182283F8922098
S31508011D107B68CC2283F893207B68012283F8942080
S31508011D207B68002283F895207B68002283F8962039
S31508011D307B68002283F897207B68002283F8982025
S31508011D407B688933102219467868FFF70DFD00BFB5
S31508011D500837BD4680BD90B585B000AF78607B6811
S31508011D600D2283F889207B68042283F88A207B6800
S31508011D70172283F88B207B681A7F7B6883F88C206F
S31508011D807B685A7F7B6883F88D207B689A7F7B689E
S31508011D9083F88E207B68DA7F7B6883F88F207B68DF
S31508011DA093F820207B6883F890207B6893F821209C
S31508011DB07B6883F891207B6893F84330002B3FD0EA
S31508011DC07B68062283F892207B6893F87B30002B88
S31508011DD013D00023FB73FB7B052B22D8FA7BFB7BF5
S31508011DE00A3379680A44117D7A6813440A4683F8E6
S31508011DF08920FB7B0133FB73EDE70023BB73BB7BB8
S31508011E00052B0ED8BA7BBB7B0A3379680A44117F46
S31508011E107A6813440A4683F88920BB7B0133BB736E
S31508011E20EDE710237B737B7B192B3CD87B7B7A6888
S31508011E301344002283F889207B7B01337B73F2E705
S31508011E407B681B691846F6F7EDF90346DAB27B6833
S31508011E5083F8922000233B733C7B7B681B691846F9
S31508011E60F6F7E0F903469C420FD27B681A693B7B79
S31508011E701A443B7B0A3311787A6813440A4683F875
S31508011E8089203B7B01333B73E6E73B7B0F2B0AD863
S31508011E903B7B0A337A681344002283F889203B7B0B
S31508011EA001333B73F1E77B6889331A22194678684F
S31508011EB0FFF75AFC00BF1437BD4690BD80B582B006
S31508011EC000AF78607B680E2283F889207B6804223C
S31508011ED083F88A207B68062283F88B207B681A7F21
S31508011EE07B6883F88C207B685A7F7B6883F88D2012
S31508011EF07B689A7F7B6883F88E207B68DA7F7B68AC
S31508011F0083F88F207B6893F820207B6883F89020DC
S31508011F107B6893F821207B6883F891207B68893355
S31508011F20092219467868FFF71FFC00BF0837BD4626
S31508011F3080BD80B582B000AF78607B680C2283F8DB
S31508011F4089207B68042283F88A207B68062283F825
S31508011F508B207B681A7F7B6883F88C207B685A7F85
S31508011F607B6883F88D207B689A7F7B6883F88E204F
S31508011F707B68DA7F7B6883F88F207B6893F820205B
S31508011F807B6883F890207B6893F821207B6883F827
S31508011F9091207B688933092219467868FFF7E4FBA3
S31508011FA000BF0837BD4680BD80B582B000AF7860F6
S31508011FB07B682B2283F889207B68042283F88A2090
S31508011FC07B68092283F88B207B681A7F7B6883F8F4
S31508011FD08C207B685A7F7B6883F88D207B689A7F83
S31508011FE07B6883F88E207B68DA7F7B6883F88F208D
S31508011FF07B6893F820207B6883F890207B6893F8A8
S3150801200021207B6883F891207B68032283F892203C
S315080120107B68002283F893207B68002283F894204A
S315080120207B6889330C2219467868FFF79DFB00BF48
S315080120300837BD4680BD80B582B000AF78607B6841
S315080120402C2283F889207B68042283F88A207B68FE
S31508012050062283F88B207B681A7F7B6883F88C209D
S315080120607B685A7F7B6883F88D207B689A7F7B68BB
S3150801207083F88E207B68DA7F7B6883F88F207B68FC
S3150801208093F820207B6883F890207B6893F82120B9
S315080120907B6883F891207B68893309221946786819
S315080120A0FFF762FB00BF0837BD4680BD80B582B029
S315080120B000AF78607B68112283F889207B68042247
S315080120C083F88A207B68022283F88B207B685B8BE6
S315080120D0DAB27B6883F88C207B685B8B1B12DBB2D8
S315080120E003F00F03DAB27B6883F88D207B688933A6
S315080120F0052219467868FFF737FB00BF0837BD4642
S3150801210080BD80B582B000AF78600B467B807B6866
S31508012110B3F8863023F004039AB27B68A3F88620C5
S315080121207B68062283F889207B68042283F88A2043
S315080121307B68032283F88B207B88DAB27B6883F875
S315080121408C207B881B12DBB203F00F03DAB27B68A3
S3150801215083F88D207B68132283F88E207B68893368
S31508012160062219467868FFF7FFFA00BF0837BD4609
S3150801217080BD80B582B000AF78607B68242283F881
S3150801218089207B680C2283F88A207B68032283F8DE
S315080121908B207B68042283F88C207B68082283F8CD
S315080121A08D207B68002283F88E207B68893306227E
S315080121B019467868FFF7D8FA00BF0837BD4680BDCB
S315080121C0B0B58AB002AFF8607A601A460B467B81D1
S315080121D013467B726B461D467B7ADC1DBC61234622
S315080121E0013318464FF000014FF000024FF000038B
S315080121F0CB0043EA5073C2002346013318464FF019
S3150801220000014FF000024FF00003CB0043EA507380
S31508012210C200234601330733DB08DB00ADEB030DB0
S3150801222002AB00337B617B89DAB27B691A707B89E1
S315080122301B125BB203F00F035BB243F020035BB2E0
S31508012240DAB27B695A707B7A0433DAB27B699A709F
S315080122507B7A04331B12DAB27B69DA707B697A7A84
S315080122601A717B7A1B12DAB27B695A717B6997F804
S3150801227030209A717B6997F83420DA710023FB8341
S315080122807B7A9BB2FA8B9A420BD2FB8B7A681A44F9
S31508012290FB8B083311787A69D154FB8B0133FB83A5
S315080122A0EEE7FB68D86CFB6893F85010FB6893F867
S315080122B05A207B7A9BB208339CB27B6900932346EA
S315080122C003F046F90346FB74FB7C002B02D064201D
S315080122D03EF028FDAD4600BF2037BD46B0BD80B5EE
S315080122E086B002AFF8607B600B467B8113467B7232
S315080122F0FB68022283F80921FB687A7A83F80A21A6
S31508012300FB68042283F80B21FB68002283F80C2161
S315080123103B8BDAB2FB6883F80D213B8B1B12DAB2D1
S31508012320FB6883F80E217B681A78FB6883F80F210E
S315080123307B685A78FB6883F81021FB6803F2091257
S31508012340798900230193012300930823F868FFF78D
S3150801235037FF00BF1037BD4680BD80B586B002AFD6
S31508012360F8607B600B467B8113467B72FB68032210
S3150801237083F80921FB687A7A83F80A21FB6808221F
S3150801238083F80B21FB68002283F80C217B681A78F5
S31508012390FB6883F80D217B685A78FB6883F80E2160
S315080123A0BB691A78FB6883F80F21BB695A78FB6801
S315080123B083F81021FB683A7F83F81121FB68002214
S315080123C083F81221FB68002283F81321FB68002297
S315080123D083F81421FB6803F2091279890023019312
S315080123E0012300930C23F868FFF7EAFE00BF1037B4
S315080123F0BD4680BD80B586B002AFF8607B600B46EE
S315080124007B8113467B72FB68042283F80921FB68EA
S315080124107A7A83F80A21FB68082283F80B21FB687C
S31508012420002283F80C217B681A78FB6883F80D2152
S315080124307B685A78FB6883F80E21FB68002283F8CB
S315080124400F21FB68002283F81021FB68012283F81B
S315080124501121FB68022283F81221FB68FF2283F807
S315080124601321FB68FF2283F81421FB6803F2091282
S31508012470798900230193012300930C23F868FFF758
S315080124809FFE00BF1037BD4680BD80B586B002AF3E
S31508012490F8607B600B467B8113467B72FB680522DD
S315080124A083F80921FB687A7A83F80A21FB680A22EC
S315080124B083F80B21FB68002283F80C217B681A78C4
S315080124C0FB6883F80D217B685A78FB6883F80E212F
S315080124D0FB68002283F80F21FB68002283F810218C
S315080124E0FB68002283F81121FB68002283F8122178
S315080124F0FB68012283F81321FB68022283F8142161
S31508012500FB68A02283F81521FB68022283F81621AD
S31508012510FB6803F2091279890023019301230093C9
S315080125200E23F868FFF74CFE00BF1037BD4680BD85
S3150801253080B586B002AFF8607B600B467B81134697
S315080125407B72FB68062283F80921FB687A7A83F88D
S315080125500A21FB68042283F80B21FB68002283F811
S315080125600C217B681A78FB6883F80D217B685A78F9
S31508012570FB6883F80E21BB691A78FB6883F80F217B
S31508012580BB695A78FB6883F81021FB6803F20912C4
S31508012590798900230193012300930823F868FFF73B
S315080125A00FFE00BF1037BD4680BD80B586B002AFAD
S315080125B0F8607B600B467B8113467B72FB680722BA
S315080125C083F80921FB687A7A83F80A21FB680422D1
S315080125D083F80B21FB68002283F80C217B681A78A3
S315080125E0FB6883F80D217B685A78FB6883F80E210E
S315080125F0BB691A78FB6883F80F21BB695A78FB68AF
S3150801260083F81021FB6803F20912798900230193E3
S31508012610012300930823F868FFF7D2FD00BF10379E
S31508012620BD4680BD80B584B002AF786008461146C4
S315080126301A4603467B800B467B7013463B707B68C4
S315080126400B2283F809217B687A7883F80A217B684B
S31508012650082283F80B217B68002283F80C217B680A
S315080126603A7883F80D217B683A7C83F80E217B68DA
S31508012670002283F80F217B68002283F810217B68EA
S31508012680002283F811217B68002283F812217B68D6
S31508012690002283F813217B68002283F814217B68C2
S315080126A003F20912798800230193012300930C236D
S315080126B07868FFF785FD00BF0837BD4680BD80B540
S315080126C08EB008AF7860396001233B7300237B73B2
S315080126D00023FB75FB7D052B11D8FB7DC3F1050393
S315080126E01A463B681A44FB7D0233127807F1180132
S315080126F00B4403F80C2CFB7D0133FB75EAE77B6879
S31508012700D86C7B6893F850107B6893F851200023A6
S31508012710079307F10C0306930823059308230493EB
S315080127200023039303230293F523019309230093BB
S31508012730212302F02EFD00BF1837BD4680BD80B5A6
S315080127408EB008AF7860396005233B731023FB749C
S3150801275001233B7502237B751223BB750023FB7589
S31508012760FB7D052B0ED8FB7D3A681A44FB7D0133A8
S31508012770127807F118010B4403F80C2CFB7D013381
S31508012780FB75EDE77B68D86C7B6893F850107B681E
S3150801279093F851200023079307F10C0306930B23A3
S315080127A005930B2304930023039303230293052321
S315080127B0019309230093212302F0EBFC00BF18378C
S315080127C0BD4680BD80B483B000AF7860044A7B689B
S315080127D01A607B6818460C37BD465DF8047B70475E
S315080127E09CBB060880B582B000AF786039607B680B
S315080127F01846FFF7E7FF214A7B681A607B683A6843
S315080128005A607B6808331846FDF776FB7B681033F8
S315080128101846FDF788FB7B6818331846FDF7AFFBAA
S315080128207B68002283F830207B68002283F83120F8
S315080128307B68002283F832207B68002283F83820DF
S315080128407B6803F120027B68C3F809207B6803F1E2
S3150801285010027B68083319461046FDF778FB7B683A
S3150801286003F118027B68083319461046FDF79BFBEE
S315080128707B6818460837BD4680BD00BF44BB0608BD
S3150801288080B582B000AF786039607B681846FFF77B
S3150801289099FF214A7B681A607B683A685A607B68A7
S315080128A008331846FDF728FB7B6810331846FDF7F1
S315080128B03AFB7B6818331846FDF761FB7B680022F3
S315080128C083F830207B68002283F831207B68002258
S315080128D083F832207B68002283F838207B6803F16D
S315080128E020027B68C3F809207B6803F110027B6824
S315080128F0083319461046FDF72AFB7B6803F11802CF
S315080129007B68083319461046FDF74DFB7B68184668
S315080129100837BD4680BD00BF38BB060880B586B0FE
S3150801292000AFF8607A603B600B467B817B89FB824E
S315080129307B683B61FB8A002B0FD007F1160207F172
S3150801294010031946F86800F02DF8034683F00103D1
S31508012950DBB2002B00D1EDE700BF1837BD4680BDBD
S3150801296080B586B000AFF8607A603B600B467B8124
S315080129707B89FB827B683B61FB8A002B0FD007F1C1
S31508012980160207F110031946F86800F081F90346A3
S3150801299083F00103DBB2002B00D1EDE700BF183746
S315080129A0BD4680BDF0B589B002AFF860B9607A60FE
S315080129B0FB6820337B61FB6820333B61FB6893F836
S315080129C03030042B00F25E8101A252F823F000BFD9
S315080129D0E5290108052A0108472A01085B2A010891
S315080129E01F2B0108FB6802221A72FB6803F1100209
S315080129F0FB68083319461046FDF7A9FAFB68012258
S31508012A0083F83020FB6810337A68B968184603F0F2
S31508012A10D5FF034683F00103DBB2002B01D0002367
S31508012A2031E1FB68D3F809301A78FB6883F831205D
S31508012A30FB68D3F809305A78FB6883F83220FB68BB
S31508012A40022283F83020FB6820339A1CFB68C3F8FE
S31508012A500920FB68032283F83020FB6893F832309B
S31508012A60023B1F2B47D801A252F823F0F72A010887
S31508012A70F72A0108ED2A0108F72A0108F72A0108A9
S31508012A80F72A0108F72A0108F72A0108F72A01088F
S31508012A90F72A0108F72A0108F72A0108F72A01087F
S31508012AA0F72A0108F72A0108F72A0108F72A01086F
S31508012AB0F72A0108F72A0108F72A0108F72A01085F
S31508012AC0F72A0108F72A0108F72A0108F72A01084F
S31508012AD0F72A0108F72A0108F72A0108F72A01083F
S31508012AE0F72A0108F72A0108F72A0108FB680022D4
S31508012AF083F8332000BFFB6893F83130023BDAB222
S31508012B00FB681A72FB6803F11002FB680833194661
S31508012B101046FDF71CFAFB68042283F83020FB688F
S31508012B2093F83230052B55D0052B00F38580022BFF
S31508012B3002D0042B15D07FE0FB6810337A68B96898
S31508012B40184603F03BFF034683F00103DBB2002B73
S31508012B5001D0002397E07B695A79FB6883F8342012
S31508012B6086E0FB6810337A68B968184603F026FFD1
S31508012B70034683F00103DBB2002B01D0002382E078
S31508012B803B695B79E02B6CD13B699B79012B6AD157
S31508012B90FB6893F83830002B04D03B69DB79002BAE
S31508012BA004D165E03B69DB79012B5ED1FB68012223
S31508012BB083F833203B699A78FB6883F836203B69AA
S31508012BC0DA78FB6883F837203B69DA79FB6883F89A
S31508012BD035204DE0FB6810337A68B968184603F06A
S31508012BE0EDFE034683F00103DBB2002B01D000237F
S31508012BF049E0FB6893F83330002B38D0FB685B68F3
S31508012C00002B34D0FB685868FB685B681B681C6836
S31508012C10FB6893F83410FB6893F83650FB6893F811
S31508012C203760FB6893F83530FA68203201920093D1
S31508012C3033462A46A0471AE0FB6803F11800FB68E9
S31508012C4093F831309BB2023B9BB27A68B968FDF7BB
S31508012C50BDF9034683F00103DBB2002B08D000233C
S31508012C6011E000BF04E000BF02E000BF00E000BFC2
S31508012C70FB6803F12002FB68C3F80920FB68002200
S31508012C8083F83020012318461C37BD46F0BD00BF26
S31508012C90F0B589B002AFF860B9607A60FB68203395
S31508012CA07B61FB6820333B61FB6893F83030042B6A
S31508012CB000F25E8101A252F823F000BFD12C01086F
S31508012CC0F12C0108332D0108472D01080B2E0108A7
S31508012CD0FB6802221A72FB6803F11002FB680833CB
S31508012CE019461046FDF733F9FB68012283F83020AF
S31508012CF0FB6810337A68B968184603F05FFE034625
S31508012D0083F00103DBB2002B01D0002331E1FB681C
S31508012D10D3F809301A78FB6883F83120FB68D3F8B1
S31508012D2009305A78FB6883F83220FB68022283F857
S31508012D303020FB6820339A1CFB68C3F80920FB681E
S31508012D40032283F83020FB6893F83230023B1F2BAD
S31508012D5047D801A252F823F0E32D0108E32D010813
S31508012D60D92D0108E32D0108E32D0108E32D0108FA
S31508012D70E32D0108E32D0108E32D0108E32D0108E0
S31508012D80E32D0108E32D0108E32D0108E32D0108D0
S31508012D90E32D0108E32D0108E32D0108E32D0108C0
S31508012DA0E32D0108E32D0108E32D0108E32D0108B0
S31508012DB0E32D0108E32D0108E32D0108E32D0108A0
S31508012DC0E32D0108E32D0108E32D0108E32D010890
S31508012DD0E32D0108E32D0108FB68002283F833205F
S31508012DE000BFFB6893F83130023BDAB2FB681A720E
S31508012DF0FB6803F11002FB68083319461046FDF714
S31508012E00A6F8FB68042283F83020FB6893F8323071
S31508012E10052B55D0052B00F38580022B02D0042BF8
S31508012E2015D07FE0FB6810337A68B968184603F055
S31508012E30C5FD034683F00103DBB2002B01D0002355
S31508012E4097E07B695A79FB6883F8342086E0FB684A
S31508012E5010337A68B968184603F0B0FD034683F063
S31508012E600103DBB2002B01D0002382E03B695B79C9
S31508012E70FF2B6CD13B699B79012B6AD1FB6893F8CF
S31508012E803830002B04D03B69DB79002B04D165E08F
S31508012E903B69DB79012B5ED1FB68012283F833207C
S31508012EA03B699A78FB6883F836203B69DA78FB68D0
S31508012EB083F837203B69DA79FB6883F835204DE0DA
S31508012EC0FB6810337A68B968184603F077FD03463C
S31508012ED083F00103DBB2002B01D0002349E0FB6834
S31508012EE093F83330002B38D0FB685B68002B34D05D
S31508012EF0FB685868FB685B681B681C68FB6893F885
S31508012F003410FB6893F83650FB6893F83760FB6812
S31508012F1093F83530FA6820320192009333462A46EF
S31508012F20A0471AE0FB6803F11800FB6893F83130F3
S31508012F309BB2023B9BB27A68B968FDF747F803462C
S31508012F4083F00103DBB2002B08D0002311E000BF98
S31508012F5004E000BF02E000BF00E000BFFB6803F128
S31508012F602002FB68C3F80920FB68002283F8302099
S31508012F70012318461C37BD46F0BD00BF80B485B095
S31508012F8000AF786039600023FB73FB7B032B15D8F0
S31508012F90FB7B7A6818339B0013445B68002B09D1C5
S31508012FA0FB7B7A6818339B0013443A685A6097F991
S31508012FB00F3005E0FB7B0133FB73E6E74FF0FF3388
S31508012FC018461437BD465DF8047B704780B582B054
S31508012FD000AF786039600A4A7B681A607B683A688C
S31508012FE09A607B689B68002B05D07B689B6879682B
S31508012FF01846FFF7C3FF7B6818460837BD4680BDEC
S31508013000D4BB060880B485B000AFF860B960134632
S31508013010FB80BB681B781A46FB88DBB29A420BD148
S31508013020BB6801331B781A46FB881B1243F0200341
S315080130309A4201D1012300E0002318461437BD4600
S315080130405DF8047B704780B485B000AFF8600B4625
S315080130507A60FB7200BF1437BD465DF8047B704782
S3150801306080B483B000AF786000BF0C37BD465DF809
S31508013070047B704780B483B000AF786000BF0C371B
S31508013080BD465DF8047B704780B586B000AFF86031
S31508013090B9603B601346FB71FB68B9681846FFF7D0
S315080130A095FF1F4AFB681A60FB68002283F86820AF
S315080130B00023FB75FB7D012B09D8FA7DFB680832D5
S315080130C0002143F82210FB7D0133FB75F2E7FB680B
S315080130D09B68FA7983F84820FB689B683A681A6105
S315080130E0FB68502283F86F20FB68002283F8702062
S315080130F0FB68702283F86B20FB68002283F86C203A
S31508013100FB68712283F86D20FB68002283F86E2024
S31508013110F86800F007F8FB6818461837BD4680BD01
S31508013120A8BB060880B582B000AF78607B6800222C
S315080131305A757B68002283F869207B68002283F828
S315080131406A207B6800221A617B680A229A767B6864
S31508013150002283F871207B681B6820331B68786816
S31508013160984700BF0837BD4680BD90B585B002AF08
S3150801317078607B6893F86A30002B14D07B6898686E
S315080131807B6899897B681B7D0133DAB27B681A757E
S315080131907B681A7D7B6803F11B047B686F33009398
S315080131A02346FFF7C5F97B6898687B6899897B6828
S315080131B01B7D0133DAB27B681A757B681A7D7B68D9
S315080131C003F118047B686D3300932346FFF7B0F9C2
S315080131D07B681B6808331B68786898477B680E22EA
S315080131E09A767B68092283F8712000BF0C37BD46A1
S315080131F090BD90B587B002AF786039607B685B7D1A
S3150801320083F00103DBB2002B23D03B6808331B781C
S31508013210022B1ED13B680C331B781A463B680D33CB
S315080132201B781B021343012B13D17B689B689B7A7E
S3150801323083F00103DBB2002B0BD07B689B6801226C
S315080132409A727B689B685A8B7B689A817B680A228B
S315080132509A767B689B685B7A83F00103DBB2002B65
S315080132603AD07B689B6893F84730002B34D07B684B
S315080132705B7D83F00103DBB2002B2DD07B6893F8CD
S31508013280693083F00103DBB2002B25D03B68083394
S315080132901B78022B20D13B680C331B781A463B68F6
S315080132A00D331B781B021343112B15D17B689B68C1
S315080132B0002283F847207B689B6801225A727B6843
S315080132C0012283F869207B689B685A8B7B689A81FF
S315080132D07B68002283F8712078687B689B891A4687
S315080132E03968FFF78FFE0346002B00F0D9833B6848
S315080132F006331B781A463B6807331B781B021343B0
S31508013300012B40F09B823B6808331B78012B00F0A8
S31508013310C1833B6808331B78032B40F08D803B68DB
S3150801332010331B781A463B6811331B781B0213436B
S31508013330002B40F0AF833B6812331B781A463B6873
S3150801334013331B781B021343002B40F0A3833B68FE
S315080133500E331A787B6893F86F309A4224D13B680A
S315080133600F331A787B6893F870309A421CD13B6800
S315080133705A7A7B681A753B681A7B7B68DA763B68EA
S315080133805A7B7B681A777B681B7D0133DAB27B68C7
S315080133901A757B6898687B6899897B681A7D7B684A
S315080133A01B33FFF727F875E33B680E331A787B68FA
S315080133B093F86B309A421AD13B680F331A787B68B7
S315080133C093F86C309A4212D13B685A7A7B681A751F
S315080133D03B681A7B7B689A753B685A7B7B68DA750A
S315080133E07B681B6943F004027B681A6152E33B68F8
S315080133F00E331A787B6893F86D309A4240F04A8307
S315080134003B680F331A787B6893F86E309A4240F01E
S3150801341041833B685A7A7B681A753B681A7B7B68D5
S315080134201A763B685A7B7B685A767B681B6943F038
S3150801343040027B681A612DE33B6808331B78022B2F
S315080134405AD13B680C331B781A463B680D331B78F7
S315080134501B021343012B12D13B685A7A7B681A75F2
S315080134603B689A7B7B68DA763B68DA7B7B681A77F6
S315080134707B681B6943F480727B681A610AE33B68BF
S315080134800C331B781A463B680D331B781B02134312
S31508013490112B12D13B685A7A7B681A753B689A7B5D
S315080134A07B689A753B68DA7B7B68DA757B681B698A
S315080134B043F001027B681A61ECE23B680C331B7826
S315080134C01A463B680D331B781B021343132B40F036
S315080134D0E1823B685A7A7B681A753B689A7B7B68F6
S315080134E01A763B68DA7B7B685A767B681B6943F0F8
S315080134F010027B681A61CDE23B6808331B78052BFD
S315080135005ED13B6810331B781A463B6811331B782A
S315080135101B021343002B40F0BD823B680C331A781B
S315080135207B6893F86F309A4212D13B680D331A784B
S315080135307B6893F870309A420AD13B685A7A7B685D
S315080135401A757B681B6943F400727B681A61A1E2EC
S315080135503B680C331A787B6893F86B309A4212D120
S315080135603B680D331A787B6893F86C309A420AD116
S315080135703B685A7A7B681A757B681B6943F00202B5
S315080135807B681A6186E23B680C331A787B6893F884
S315080135906D309A4240F07E823B680D331A787B681B
S315080135A093F86E309A4240F075823B685A7A7B6886
S315080135B01A757B681B6943F020027B681A6169E208
S315080135C03B6808331B78042B55D13B680C331A78B2
S315080135D07B6893F86F309A4213D13B680D331A789A
S315080135E07B6893F870309A420BD17B6898687B6840
S315080135F099893B6809331A787B681B33FEF745FFBF
S3150801360048E23B680C331A787B6893F86B309A4228
S3150801361013D13B680D331A787B6893F86C309A425C
S315080136200BD17B6898687B6899893B6809331A7856
S315080136307B681633FEF729FF2CE23B680C331A78B0
S315080136407B6893F86D309A4240F024823B680D33CB
S315080136501A787B6893F86E309A4240F01B827B6831
S3150801366098687B6899893B6809331A787B681833A7
S31508013670FEF70BFF0EE23B6808331B78062B70D169
S315080136803B680C331A787B6893F86F309A4212D1EB
S315080136903B680D331A787B6893F870309A420AD1E1
S315080136A03B685A7A7B681A757B681B6943F48062A2
S315080136B07B681A61EEE13B680C331A787B6893F8EC
S315080136C06B309A4221D13B680D331A787B6893F89F
S315080136D06C309A4219D13B685A7A7B681A757B68AD
S315080136E098687B6899897B681A7D7B6803F16B0406
S315080136F07B68163300932346FEF757FF7B681B68E2
S3150801370008331B6878689847C4E13B680C331A7814
S315080137107B6893F86D309A4240F0BC813B680D3363
S315080137201A787B6893F86E309A4240F0B3813B6809
S315080137305A7A7B681A757B6898687B6899897B6869
S315080137401A7D7B6803F16D047B6818330093234661
S31508013750FEF72BFF7B681B6808331B687868984758
S3150801376098E13B6808331B78072B4CD13B680C332F
S315080137701A787B68DB7E9A4211D13B680D331A7839
S315080137807B681B7F9A420AD13B685A7A7B681A750D
S315080137907B681B6943F480427B681A617AE13B685E
S315080137A00C331A787B689B7D9A4211D13B680D339D
S315080137B01A787B68DB7D9A420AD13B685A7A7B681C
S315080137C01A757B681B6943F008027B681A6161E117
S315080137D03B680C331A787B681B7E9A4240F05A8103
S315080137E03B680D331A787B685B7E9A4240F05281BA
S315080137F03B685A7A7B681A757B681B6943F08002B5
S315080138007B681A6146E13B6808331B780A2B40F04E
S3150801381041813B685A7A7B681A757B6898687B6828
S3150801382099897B681A7D3B680C331C783B680D3394
S315080138301B7800932346FEF7F5FE2BE13B6806331A
S315080138401A787B6893F86F309A4240F087803B6814
S3150801385007331A787B6893F870309A427ED13B68B1
S3150801386008331B78022B31D17B68032283F8282081
S315080138703B685A7A7B6883F829203B689A7A7B6881
S3150801388083F82A207B68002283F82B207B6805228F
S3150801389083F82C207B68002283F82D207B68002280
S315080138A083F82E207B68002283F82F207B6800226C
S315080138B083F830207B68002283F831207B6828331F
S315080138C00A221946786800F06DFBE0E03B68083388
S315080138D01B78042B31D17B68052283F828203B68A5
S315080138E05A7A7B6883F829203B689A7A7B6883F839
S315080138F02A207B68002283F82B207B68052283F81F
S315080139002C207B68002283F82D207B68022283F80D
S315080139102E207B68352283F82F207B68002283F8C6
S3150801392030207B68002283F831207B6828330A22FD
S315080139301946786800F036FBA9E03B6808331B781E
S31508013940062B40F0A4803B68093319783B680A3393
S315080139501B781A46786800F03FFB98E03B68063307
S315080139601A787B6893F86D309A4262D13B680733BF
S315080139701A787B6893F86E309A425AD13B680833B5
S315080139801B78A12B40F085803DF0C0F902467B6883
S315080139905A673B6805331B781B021AB23B68043326
S315080139A01B781BB213431BB2FB817B681B6814335C
S315080139B01B68FA89D2B2013AD1B23A6809327868F3
S315080139C098473B6809331B78012B02D0022B16D086
S315080139D05FE07B681B6A002B27D07B68186A7B68C7
S315080139E01B6A1B681C68FB89DBB2023BDAB23B68BF
S315080139F00A330093134600227968A04715E07B68CD
S31508013A005B6A002B13D07B68586A7B685B6A1B6804
S31508013A101C68FB89DBB2023BDAB23B680A330093C6
S31508013A20134600227968A04701E000BF31E000BFD4
S31508013A302FE03B6806331A787B6893F86B309A4215
S31508013A4028D13B6807331A787B6893F86C309A4219
S31508013A5020D13B6808331B78A32B1BD13B68053360
S31508013A601B781B021AB23B6804331B781BB213433B
S31508013A701BB2BB817B681B6818331B68BA89D2B233
S31508013A80013AD1B23A6809327868984702E000BF2C
S31508013A9000E000BF786800F007F8786800F0B4F82D
S31508013AA000BF1437BD4690BDB0B584B002AF78608B
S31508013AB07B689B7E0E2B00F084800E2B00F39F8083
S31508013AC00A2B02D00B2B68D099E07B681B6903F49B
S31508013AD08073002B41D07B681B6923F480727B6855
S31508013AE01A617B6898687B6899897B681A7D7B6807
S31508013AF003F16F047B681B33012501950093234667
S31508013B00FEF72BFC01203DF00DF97B6898687B6870
S31508013B1099897B681A7D7B6803F16F047B681B337F
S31508013B200025019500932346FEF717FC7B681B7D4C
S31508013B300133DAB27B681A7501203DF0F3F87B6828
S31508013B4098687B6899897B681A7D7B681B33FEF7C1
S31508013B5051FC7B680B229A764CE07B681B6903F45F
S31508013B608063002B46D07B681B6923F480627B68DF
S31508013B701A617B68002283F86A207B6898687B68EB
S31508013B8099897B681A7D7B6803F16F047B681B330F
S31508013B9000932346FEF709FD2CE07B681B6903F4B5
S31508013BA00073002B28D07B681B6923F400727B689D
S31508013BB01A617B68012283F86A207B680A229A7651
S31508013BC01AE07B681B6903F48043002B16D07B68D7
S31508013BD09A687B689B8919461046FEF792FA7B68B4
S31508013BE04FF6FF729A817B681B6808331B687868F1
S31508013BF0984703E000BF02E000BF00E000BF00BF36
S31508013C000837BD46B0BD0000B0B584B002AF7860D4
S31508013C107B6893F87130013B082B00F22C8101A2D5
S31508013C2052F823F0553E0108EF3C0108273D0108EB
S31508013C30493C0108213E0108673C01086F3D01081E
S31508013C40A53D0108E13D01087B681B6903F00203F4
S31508013C50002B00F00181786800F0F9F97B680622EB
S31508013C6083F87120F8E07B681B6903F01003002BC9
S31508013C7000F0F4807B6898687B6899897B681A7D6F
S31508013C807B6803F16D047B68183301250195009360
S31508013C902346FEF762FB01203DF044F87B689868ED
S31508013CA07B6899897B681A7D7B6803F16D047B685B
S31508013CB018330025019500932346FEF74EFB7B68D2
S31508013CC01B7D0133DAB27B681A7501203DF02AF8AB
S31508013CD07B6898687B6899897B681A7D7B68183345
S31508013CE0FEF788FB7B68082283F87120B6E07B68BB
S31508013CF01B6903F00403002B00F0B2807B681B7D6F
S31508013D000133DAB27B681A757B6898687B6899898A
S31508013D107B681A7D7B681633FEF76CFB7B6803228A
S31508013D2083F871209CE07B681B6903F00203002B72
S31508013D3000F09880786800F08AF901203CF0F2FFDB
S31508013D407B681B7D0133DAB27B681A757B689868D4
S31508013D507B6899897B681A7D7B686D331324009487
S31508013D60FEF7BDFA7B68072283F871207AE07B6843
S31508013D701B6903F04003002B76D07B681B7D01335A
S31508013D80DAB27B681A757B6898687B6899897B685B
S31508013D901A7D7B681833FEF72DFB7B68082283F8AA
S31508013DA0712061E07B681B6903F02003002B5DD05D
S31508013DB07B689B68002283F846207B689B68002203
S31508013DC083F848207B6801225A757B681B68103383
S31508013DD01B68786898477B68012283F8712045E05B
S31508013DE07B681B6903F08003002B41D07B681B7D30
S31508013DF00133DAB27B681A757B6898687B6899899A
S31508013E007B681A7D7B6803F116047B686B33009324
S31508013E102346FEF78DFB7B68052283F8712027E090
S31508013E207B681B6903F00803002B23D07B689A681B
S31508013E307B689B8919461046FEF763F97B684FF63E
S31508013E40FF729A817B6800221A617B68002283F8D7
S31508013E5071200FE000BF0EE000BF0CE000BF0AE0D2
S31508013E6000BF08E000BF06E000BF04E000BF02E0B3
S31508013E7000BF00E000BF00BF0837BD46B0BD00BFA8
S31508013E80B0B584B002AF78607B6893F87130002BC7
S31508013E9040F084807B689B6893F84630002B3AD0C3
S31508013EA07B689B685B7A83F00103DBB2002B32D017
S31508013EB07B685B7D83F00103DBB2002B2BD07B682B
S31508013EC093F8693083F00103DBB2002B23D07B68BA
S31508013ED09B6801225A727B68012283F869207B68F4
S31508013EE09B685A8B7B689A817B6800221A617B687A
S31508013EF000221A757B6898687B6899897B681A7DA0
S31508013F007B686B3311240094FEF7E9F97B6802227A
S31508013F1083F8712041E07B681B6903F00103002BDC
S31508013F203BD07B6898687B6899897B681A7D7B6832
S31508013F3003F16B047B68163301250195009323462B
S31508013F40FEF70BFA01203CF0EDFE7B6898687B686A
S31508013F5099897B681A7D7B6803F16B047B68163344
S31508013F600025019500932346FEF7F7F97B681B7D2B
S31508013F700133DAB27B681A7501203CF0D3FE7B68FF
S31508013F8098687B6899897B681A7D7B681633FEF782
S31508013F9031FA7B68042283F8712000BF00BF083715
S31508013FA0BD46B0BD90B587B002AFF860B96013469B
S31508013FB0FB71FB689868FB689989FB68DB7EFA6880
S31508013FC0127FFC79019200932346BA68FEF7F8F846
S31508013FD000BF1437BD4690BD80B582B000AF78608A
S31508013FE00B46FB701346BB707B68072283F82820B3
S31508013FF07B68FA7883F829207B68BA7883F82A20BF
S315080140007B68002283F82B207B68052283F82C2005
S315080140107B68002283F82D207B68022283F82E20F4
S315080140207B68352283F82F207B68002283F83020AD
S315080140307B68002283F831207B6828330A221946D7
S315080140407868FFF7AFFF00BF0837BD4680BD90B55A
S3150801405087B002AF78607B6893F86830002B08D088
S315080140607B6893F86830012B03D07B68002283F8BC
S3150801407068207B6893F8683043F07003DBB2FB7302
S315080140807B6898687B6899897B689B7D7A68D27D0D
S3150801409007F10F040192009301232246FEF790F8D7
S315080140A000BF1437BD4690BD80B483B000AF034648
S315080140B0FB71FB79002B00F0D480FB79132B00F000
S315080140C0D080FB79012B00F0CA80FB79142B00F014
S315080140D0C680FB79022B00F0C080FB79152B00F016
S315080140E0BC80FB79032B00F0B680FB79162B00F018
S315080140F0B280FB79082B00F0AC80FB79182B00F015
S31508014100A880FB79212B00F0A480FB79262B00F0EF
S31508014110A080FB79172B00F09C80FB791B2B00F004
S315080141209880FB79332B00F09480FB79092B00F0FA
S315080141308E80FB79192B00F08A80FB79272B00F0FA
S315080141408680FB79282B00F08280FB790A2B7CD0AC
S31508014150FB79292B79D0FB790B2B74D0FB792A2B88
S3150801416071D0FB790E2B6CD0FB792B2B69D0FB799F
S31508014170242B66D0FB790F2B61D0FB792C2B5ED0D3
S31508014180FB79252B5BD0FB790C2B56D0FB792D2B94
S3150801419053D0FB790D2B4ED0FB792E2B4BD0FB79C7
S315080141A0042B46D0FB791E2B43D0FB79052B3ED039
S315080141B0FB791D2B3BD0FB79062B36D0FB791F2BC0
S315080141C033D0FB79072B2ED0FB79202B2BD0FB790B
S315080141D02F2B26D0FB79102B23D0FB79222B20D02D
S315080141E0FB79302B1BD0FB79112B18D0FB791A2BB5
S315080141F015D0FB79232B12D0FB79312B0DD0FB7906
S31508014200122B0AD0FB791C2B07D0FB79322B01D153
S31508014210132327E04FF0FF3324E0122322E0112372
S3150801422020E010231EE00F231CE00E231AE00D23C5
S3150801423018E00C2316E00B2314E00A2312E00923E5
S3150801424010E008230EE007230CE006230AE0052305
S3150801425008E0042306E0032304E0022302E0012325
S3150801426000E0002318460C37BD465DF8047B70470D
S3150801427080B584B000AF0346FB71FB791846FFF79A
S3150801428013FF0346FB73FB7B112B02D94FF0FF3358
S3150801429001E097F90F3018461037BD4680BD00007A
S315080142A080B483B000AF78600B46FB70FB78032BB4
S315080142B06ED801A252F823F0C9420108FB4201084F
S315080142C02D4301085F4301087B681B7A03F00F033E
S315080142D0DBB2072B0DD07B681B7A03F00F03DBB229
S315080142E0002B06D07B681B7A03F00F03DBB2012B88
S315080142F001D101234DE000234BE07B681B7A03F0D3
S315080143000F03DBB2012B0DD07B681B7A03F00F0379
S31508014310DBB2022B06D07B681B7A03F00F03DBB2F4
S31508014320032B01D1012334E0002332E07B681B7A99
S3150801433003F00F03DBB2032B0DD07B681B7A03F066
S315080143400F03DBB2042B06D07B681B7A03F00F033D
S31508014350DBB2052B01D101231BE0002319E07B68A1
S315080143601B7A03F00F03DBB2052B0DD07B681B7A92
S3150801437003F00F03DBB2062B06D07B681B7A03F02A
S315080143800F03DBB2072B01D1012302E0002300E072
S31508014390002318460C37BD465DF8047B704700BFFD
S315080143A080B584B000AF78600B46FB70FB78184681
S315080143B0FFF75EFF0346FB7397F90F30002B01DA0F
S315080143C000231DE097F90F30032B06DCFB7819460D
S315080143D07868FFF765FF034612E07B689B68C3F3BD
S315080143E01703194697F90F30074A13441B7821FA20
S315080143F003F303F00103002B14BF01230023DBB2EF
S3150801440018461037BD4680BDE8BB060880B586B09C
S3150801441000AF78600B46FB70FB781846FFF728FF5C
S315080144200346FB7597F91730002B01DA002331E0B3
S3150801443097F91730194A13441B781A4601239340F2
S315080144403B617B6893F84320B3F844301B0213435E
S315080144501A463B691340002B14BF01230023FB7343
S315080144607B6893F84320B3F844301B0213431A467A
S315080144703B69DB43134023F07F427B68D1B20020BE
S31508014480014383F84310120A92B200210A43A3F8A2
S315080144904420FB7B18461837BD4680BDE8BB060895
S315080144A080B584B000AF78600B46FB70FB78184680
S315080144B0FFF7DEFE0346FB7397F90F30002B01DA8F
S315080144C0002322E00E20FFF7EFFD03461A4697F96F
S315080144D00F3093420CBF01230023DBB2002B02D01D
S315080144E07B68DB7A11E00F20FFF7DEFD03461A46EB
S315080144F097F90F3093420CBF01230023DBB2002B3F
S3150801450002D07B681B7B00E0002318461037BD46A6
S3150801451080BD80B483B000AF78600B46FB70FB7832
S315080145207A6813441B7918460C37BD465DF8047B37
S31508014530704780B586B000AFF8600B467A60FB72AB
S31508014540FB7A012B40F2A6807B68002B00F0A28043
S315080145507B681B78012B0ED1FB68181D7B68591CDB
S31508014560FB7A013BDBB23C2B28BF3C23DBB21A4664
S315080145704FF054FC16E07B681B78112B40F09880AD
S31508014580FB7A032B40F29680FB68181D7B68D91CC1
S31508014590FB7A033BDBB23C2B28BF3C23DBB21A4632
S315080145A04FF03CFCFB689B68C3F31702FB681B6C66
S315080145B0C3F317039A426DD0FB689B68C3F31703CD
S315080145C01A46FB681B6CC3F31703DB43134023F03E
S315080145D07F42FB68D1B20020014383F84310120AD7
S315080145E092B200210A43A3F84420FB689B68C3F3EF
S315080145F01701FA68136C61F3170313640023FB753B
S315080146000021F868FFF74CFE0346002B03D0FB7D1B
S3150801461043F00103FB750121F868FFF741FE0346E4
S31508014620002B03D0FB7D43F00203FB750221F868DA
S31508014630FFF736FE0346002B03D0FB7D43F0040348
S31508014640FB750321F868FFF72BFE0346002B03D001
S31508014650FB7D43F00803FB75FB6893F84E30FA7D42
S315080146609A4217D0FB6893F84E305BB2DB435AB2D5
S3150801467097F9173013405BB203F00F03D9B2FA6802
S3150801468092F8433061F3030382F84330FB68FA7DFD
S3150801469083F84E20FB6893F84D30002B0BD0FB684E
S315080146A01B681B68FA6846321146F868984702E0A3
S315080146B000BF00E000BF1837BD4680BD80B485B095
S315080146C000AF78600023FB73FB7B032B08D8FB7BC9
S315080146D07A6813447F221A71FB7B0133FB73F3E774
S315080146E07A6893686FF3170393607A68136C6FF3AC
S315080146F0170313640023FB73FB7B012B08D8FB7B91
S315080147007A6813440022DA72FB7B0133FB73F3E701
S315080147100023FB73FB7B022B1BD80023BB73BB7BDC
S31508014720012B12D8FA7BBB7B796898001346DB000C
S31508014730134403440B4403F12002937943F08003A5
S315080147409371BB7B0133BB73E9E7FB7B0133FB73D6
S31508014750E0E77A68137A082161F3030313727A682A
S3150801476092F84030082161F3030382F840307A68F1
S3150801477092F843306FF3030382F843307B680022D3
S3150801478083F84E207B68002283F847207B6893F8DC
S3150801479047207B6883F846207B68002283F84A20F5
S315080147A07B6893F84A207B6883F849207B6893F8ED
S315080147B049207B6883F848207B68002283F84C20CF
S315080147C07B6893F84C207B6883F84B207B68002232
S315080147D083F84D2000BF1437BD465DF8047B70474A
S315080147E080B483B000AF78607B6800221A707B685A
S315080147F00022DA7100BF0C37BD465DF8047B7047AD
S3150801480080B584B000AF0346FB71FB791846FFF704
S315080148104BFC0346FB73FB7B122B02D94FF0FF338C
S3150801482001E097F90F3018461037BD4680BD0000E4
S3150801483080B483B000AF78600B46FB70FB78032B1E
S315080148406ED801A252F823F0594801088B4801088D
S31508014850BD480108EF4801087B68DB7E03F00F03BA
S31508014860DBB2072B0DD07B68DB7E03F00F03DBB2CF
S31508014870002B06D07B68DB7E03F00F03DBB2012B2E
S3150801488001D101234DE000234BE07B68DB7E03F079
S315080148900F03DBB2012B0DD07B68DB7E03F00F0320
S315080148A0DBB2022B06D07B68DB7E03F00F03DBB29B
S315080148B0032B01D1012334E0002332E07B68DB7E40
S315080148C003F00F03DBB2032B0DD07B68DB7E03F00D
S315080148D00F03DBB2042B06D07B68DB7E03F00F03E4
S315080148E0DBB2052B01D101231BE0002319E07B680C
S315080148F0DB7E03F00F03DBB2052B0DD07B68DB7E75
S3150801490003F00F03DBB2062B06D07B68DB7E03F0D0
S315080149100F03DBB2072B01D1012302E0002300E0DC
S31508014920002318460C37BD465DF8047B704700BF67
S3150801493080B584B000AF78600B46FB70FB781846EB
S31508014940FFF75EFF0346FB7397F90F30002B01DA79
S3150801495000231EE097F90F30032B06DCFB78194676
S315080149607868FFF765FF034613E07B68DA7E9B8B61
S315080149701B021343194697F90F30084A13441B784B
S3150801498021FA03F303F00103002B14BF01230023CB
S31508014990DBB218461037BD4680BD00BFFCBB060812
S315080149A080B586B000AF78600B46FB70FB78184679
S315080149B0FFF726FF0346FB7597F91730002B01DA37
S315080149C0002331E097F91730194A13441B781A4620
S315080149D0012393403B617B6893F83F20B3F840304D
S315080149E01B0213431A463B691340002B14BF0123CC
S315080149F00023FB737B6893F83F20B3F840301B0212
S31508014A0013431A463B69DB43134023F07F427B6815
S31508014A10D1B20020014383F83F10120A92B2002155
S31508014A200A43A3F84020FB7B18461837BD4680BDCC
S31508014A30FCBB060880B584B000AF78600B46FB70F6
S31508014A40FB781846FFF7DCFE0346FB7397F90F3030
S31508014A50002B01DA002322E00E20FFF725FB03468F
S31508014A601A4697F90F3093420CBF01230023DBB294
S31508014A70002B02D07B681B7E11E00F20FFF714FB89
S31508014A8003461A4697F90F3093420CBF01230023B8
S31508014A90DBB2002B02D07B685B7E00E00023184660
S31508014AA01037BD4680BD80B483B000AF78600B4631
S31508014AB0FB70FB787A6813441B7D18460C37BD4694
S31508014AC05DF8047B704780B586B000AFF8600B4689
S31508014AD07A60FB72FB7A012B40F2B5807B68002B6A
S31508014AE000F0B1807B681B78012B0FD1FB6803F1BD
S31508014AF014007B68591CFB7A013BDBB2282B28BFC3
S31508014B002823DBB21A464FF089F917E07B681B7830
S31508014B10312B40F0AE80FB7A022B40F2AC80FB6869
S31508014B2003F114007B68991CFB7A023BDBB2282B44
S31508014B3028BF2823DBB21A464FF070F9FB68DA7EE4
S31508014B409B8B1B0213431A46FB68DB6BC3F31703E4
S31508014B509A4270D0FB68DA7E9B8B1B0213431A4676
S31508014B60FB68DB6BC3F31703DB43134023F07F4278
S31508014B70FB68D1B20020014383F83F10120A92B2B2
S31508014B8000210A43A3F84020FB68DA7E9B8B1B02AF
S31508014B9013431946FA68D36B61F31703D3630023EA
S31508014BA0FB750021F868FFF743FE0346002B03D087
S31508014BB0FB7D43F00103FB750121F868FFF738FE19
S31508014BC00346002B03D0FB7D43F00203FB7502214C
S31508014BD0F868FFF72DFE0346002B03D0FB7D43F053
S31508014BE00403FB750321F868FFF722FE0346002B31
S31508014BF003D0FB7D43F00803FB75FB6893F84B3044
S31508014C00FA7D9A4217D0FB6893F84B305BB2DB43C7
S31508014C105AB297F9173013405BB203F00F03D9B2B2
S31508014C20FA6892F83F3061F3030382F83F30FB6874
S31508014C30FA7D83F84B20FB68B3F84C3001339AB2FE
S31508014C40FB68A3F84C20FB6893F84A30002B07D180
S31508014C50FB68DB7A002B03D1FB68DB7C002B0BD0CE
S31508014C60FB681B681B68FA6842321146F868984760
S31508014C7002E000BF00E000BF1837BD4680BD80B521
S31508014C8084B000AF78600023FB73FB7B032B08D845
S31508014C90FB7B7A6813447F221A75FB7B0133FB730E
S31508014CA0F3E77B680022DA7600229A837A68D36B67
S31508014CB06FF31703D3630023FB73FB7B012B08D820
S31508014CC0FB7B7A68134400221A76FB7B0133FB735C
S31508014CD0F3E70023FB73FB7B012B0CD8FB7B7A687C
S31508014CE00C339B0013441A7942F080021A71FB7B3C
S31508014CF00133FB73EFE77A68D37E082161F3030377
S31508014D00D3767A6892F83C30082161F3030382F876
S31508014D103C307A6892F83F306FF3030382F83F30EC
S31508014D207B68002283F84B207B6804331846FFF71B
S31508014D3057FD7B680C331846FFF752FD7B68002246
S31508014D4083F843207B6893F843207B6883F84220E5
S31508014D507B68002283F844207B68002283F845207B
S31508014D607B68002283F846207B68002283F8492065
S31508014D707B6893F849207B6883F848207B6893F819
S31508014D8048207B6883F847207B68002283F84A20FD
S31508014D9000BF1037BD4680BD80B483B000AF7860D0
S31508014DA039607B681B78FC2B58D0FC2B5ADC262BE8
S31508014DB022D0262B56DC012B02D0022B0ED051E035
S31508014DC03B6801221A703B6801337A6852781A7077
S31508014DD03B6802337A6892781A7050E03B6802227F
S31508014DE01A703B6801337A6852781A703B68023345
S31508014DF07A6892781A7042E03B6826221A707B68B4
S31508014E005A783B680133D243D2B21A707B689B78D1
S31508014E10002B03D03B68023302221A703B68043325
S31508014E207A68D2781A703B6805337A6812791A70EB
S31508014E303B6806337A6852791A707B689A793B68B7
S31508014E4009335208D2B21A703B6809331B78002B12
S31508014E5014D13B68093301221A700FE03B68FC2222
S31508014E601A700CE03B6800221A703B680133002275
S31508014E701A703B68023300221A7000E000BF7B6893
S31508014E800022DA7100BF0C37BD465DF8047B704716
S31508014E9080B483B000AF7860064A7B681A607B6885
S31508014EA000225A607B6818460C37BD465DF8047BBC
S31508014EB0704700BFFCB3060880B582B000AF7860C2
S31508014EC07B681846FFF7E4FF054A7B681A607B682A
S31508014ED04FF47A729A607B6818460837BD4680BDDA
S31508014EE018BC060880B500AF0122102102483DF022
S31508014EF001FD00BF80BD00BF0010024080B500AFB4
S31508014F000022102102483DF0F5FC00BF80BD00BF1C
S31508014F100010024080B584B000AF78600B46FB7084
S31508014F20FFF7ECFFF91C4FF0FF330122094842F065
S31508014F3099FB0023FB7307F10F014FF0FF330122A1
S31508014F40044842F0CBFCFFF7CDFFFB7B1846103730
S31508014F50BD4680BD74C4012080B584B000AF7860B9
S31508014F600B46FB701346BB70FFF7C8FFFB7843F08F
S31508014F700203DBB23B73BB787B7307F10C014FF07D
S31508014F80FF330222044842F06DFBFFF7ABFF00BF77
S31508014F901037BD4680BD00BF74C4012080B500AF7F
S31508014FA04FF4005102483DF08DFC0346184680BD7A
S31508014FB00008024080B582B000AF7860786801F0D9
S31508014FC0C5F97B68184601F0DDF97B68002283F88C
S31508014FD0B820054B11221A70786800F007F87B682B
S31508014FE018460837BD4680BD3D10002080B483B001
S31508014FF000AF78607B68002283F8B82000BF0C37C1
S31508015000BD465DF8047B704780B586B000AF786011
S315080150100B46FB701346BB707B68FA781146184637
S3150801502001F0EAF9F860FB68002B03D0FB681B68FE
S31508015030002B01D1002318E0FB681B687B61002364
S31508015040FB74FB685B79FA7C9A420DD27B691B7803
S31508015050BA789A4201D17B6907E07B6903337B61A0
S31508015060FB7C0133FB74ECE7002318461837BD4671
S3150801507080BD80B586B000AFF8607B600B46FB72D9
S315080150801346BB727B68002B01D1D82315E0FB6858
S31508015090FA7A1146184601F0AFF978617B69002B57
S315080150A001D1D62309E07B69FA7A1A717B697A6894
S315080150B01A607B69BA7A5A71002318461837BD46B1
S315080150C080BD80B586B000AFF8607B600B46FB7289
S315080150D01346BB72FB68FA7A1146184601F08CF939
S315080150E078617B69002B01D1D6234EE07B691B6869
S315080150F0002B01D1D72348E0BA7AFB7A1946F8681A
S31508015100FFF782FF02467B681A607B681B68002BE3
S3150801511001D1DB2339E07B681B689B78C3F38503E0
S31508015120DBB20F2B28BF0F23DBB21A4601239340AC
S315080151309AB23B6A1A803B6A1B88013B9AB23B6A60
S315080151401A80FB7A1A46E021F868FFF705FFD8218D
S31508015150F868FFF7DFFE0346FB747B699B79002B32
S3150801516009D0FB6893F8B820FB7C1343DBB243F004
S315080151700203DBB203E0FB7C23F00603DBB21A462B
S31508015180D821F868FFF7E8FE002318461837BD4608
S3150801519080BD90B58BB002AF7860084611461A46B5
S315080151A00346FB700B46BB7013467B700023FB76E8
S315080151B00023FB6000237B8107F10C00BA78F9789C
S315080151C007F10A03009303467868FFF77AFF034657
S315080151D0FB77FB7F002B01D0FB7FAEE07B7803F0EA
S315080151E08003002BCCBF01230023FB767B783B741D
S315080151F097F830307B7497F83430BB7497F83830A9
S31508015200FB74BB8FBB82B7F84030FB8207F11003F2
S3150801521008222021786801F015F97B89BA781021CE
S31508015220786800F0FBFA0346FB77FB7F002B01D079
S31508015230FB7F82E0BB6C002B72D0FB7E002B57D024
S31508015240B7F84030BB83FA68937843F0020393704A
S31508015250BB8B002B5FD0B7F844303B81F9687A895C
S3150801526007F1080000230193BB6C00930346786895
S3150801527000F0A6F80346FB77FB7F062B14D1F8212D
S315080152807868FFF747FE034603F02003002B0CBF9F
S3150801529001230023DBB2FA6803F00103D9B293783C
S315080152A061F341039370D3E7FB7F002B01D0FB7FAA
S315080152B043E0FB7F002B11D1FB6C002B0ED0FB6C5E
S315080152C01B681C683989B7F84020BB8BD31A9BB277
S315080152D03B8307F11803BA6CF86CA0473B89BA8B74
S315080152E0D31ABB833B89B7F844209A4212D8AFE751
S315080152F0FA68937843F001039370F9687A89B7F8E5
S315080153004400BB6C00930346786800F053F90346E2
S31508015310FB7700E000BFFB7F002B01D0FB7F0CE091
S31508015320FB7E002B01D0A02100E080217B89BA7881
S31508015330786800F073FA034600BF18462437BD465D
S3150801534090BD80B58AB002AFF8607B600B46FB72F0
S315080153501346BB720023BB610023FB8207F11800C9
S31508015360BA7AF97A07F1160300930346F868FFF744
S31508015370A8FE0346FB77FB7F002B10D0FB7F81211C
S31508015380184601F08DF8FB7A8121184601F088F854
S31508015390BB7A8121184601F083F8FB7F0CE0B969D5
S315080153A0FA8A97F82C300193BB6A00937B68F868F0
S315080153B000F006F8034600BF18462037BD4680BDF3
S315080153C080B586B000AFF860B9603B601346FB80D4
S315080153D00023FB753B681B887B82BB685B787B7403
S315080153E03B6800221A80BB689B7803F00203DBB294
S315080153F0002B01D0202300E010231A46E821F86883
S31508015400FFF7AAFDBB681A78FB880021F86800F047
S3150801541005FA0346FB75FB7D062B23D1F821F868AF
S31508015420FFF778FD034603F01003002B0CBF012399
S315080154300023DBB203F00103D9B2BA68937861F3AA
S3150801544041039370BB689B7803F00203DBB2002B20
S3150801545001D0202300E010231A46E821F868FFF757
S315080154607BFD6EE0FB7D002B6CD1C821F868FFF748
S3150801547051FD034603F00403002B0CBF012300234F
S31508015480DBB2002B02D0F023FB755CE03021F86813
S31508015490FFF740FD0346BB75BA7D7B8A9A4201DD5B
S315080154A07B8ABB753B68B3F900309BB27A8AD31AFB
S315080154B09BB2BB82B7F91430002B01DA0023BB82F9
S315080154C0BA7DB7F914309342A8BF1346DAB23B6ADC
S315080154D00821F86800F0F0FF38620422C821F8684C
S315080154E0FFF73AFD3B681A88BB7D9BB213449AB213
S315080154F03B681A80BA7D7B7C9A4204D33B681B8839
S315080155007A8A9A4213D8F821F868FFF703FD034609
S3150801551003F01003002B01D0012100E00021BA6835
S31508015520937861F3410393700023FB750BE097F8B9
S315080155302430002B3FF466AF97F8243018463BF029
S31508015540F1FB5FE700BFFB7D18461837BD4680BDF6
S3150801555080B588B002AF7860084611461A460346F8
S31508015560FB700B46BB7013463B8000233B6100234F
S31508015570FB8107F11000BA78F97807F10E03009359
S3150801558003467868FFF79DFD0346FB75FB7D002BF7
S3150801559001D0FB7D0AE03969FA8938883B6A0093AC
S315080155A00346786800F006F8034600BF1846183720
S315080155B0BD4680BD80B58AB000AFF860B9601146B6
S315080155C01A460B46FB801346BB80002387F8273013
S315080155D03B6B3B62BB88BB83BB685B78FB76FB7E18
S315080155E0002B02D0FB7E402B01D9DA2312E13BF0D6
S315080155F08DFB034603F59C5308337B61BB689B7897
S3150801560003F00103DBB2002B01D0802300E0402325
S315080156101A46E821F868FFF79FFCBB8B002B00F0C0
S31508015620DA80002387F826300023FB83FB7E9BB2B2
S31508015630BA8B934228BF13467B827B8ADAB23B6ACE
S315080156401021F86800F0FEFE7B8ADBB21A46382183
S31508015650F868FFF781FCBB681B7843F02003DBB2CF
S315080156601A46F021F868FFF777FCC821F868FFF7B2
S3150801567051FC03465BB2DB43DBB2DB09DBB2002B31
S3150801568000D0F2E78022C821F868FFF765FCF82107
S31508015690F868FFF73FFC034603F00F0387F8273046
S315080156A097F82730002B08D03BF030FB02467B6980
S315080156B0D31A002B01DA012300E00023002B00F0A6
S315080156C0818097F827300E2B12D00E2B00F3858098
S315080156D0042B02D0062B15D07FE0FB8B0133FB830D
S315080156E0FB88002B32D0FA8BFB889A422ED175E0C3
S315080156F097F82630013387F8263097F82630032B9A
S3150801570026D16BE0F821F868FFF704FC034603F09D
S315080157102003002B0CBF01230023DBB203F0010396
S31508015720D9B2BA68937861F300039370BB689B7822
S3150801573003F00103DBB2002B01D0802300E04023F4
S315080157401A46E821F868FFF707FC02E000BF00E007
S3150801575000BF00223821F868FFF7FEFB3B6A1B7879
S315080157601A461021F868FFF7F7FB7B8ADBB21A465F
S315080157703821F868FFF7F0FBBB681B7843F0200374
S31508015780DBB21A46F021F868FFF7E6FBC821F8688C
S31508015790FFF7C0FB03465BB2DB43DBB2DB09DBB2D7
S315080157A0002B00D0F2E78022C821F868FFF7D4FB66
S315080157B0F821F868FFF7AEFB034603F00F0387F8F5
S315080157C027306DE7BA8B7B8AD31ABB837B8A3A6A01
S315080157D013443B6221E700BF00E000BF97F827307A
S315080157E0002B04D000223821F868FFF7B5FBF82111
S315080157F0F868FFF78FFB034603F02003002B01D05F
S31508015800012100E00021BA68937861F300039370DF
S3150801581097F8273018462837BD4680BD80B586B02B
S3150801582000AF7860084611461A460346FB700B46D8
S31508015830BB7013463B803BF069FA034603F59C535C
S3150801584008333B610023FB750023BB750023BB822C
S315080158503BF05CFA02463B69D31ADB0FDBB2002B3D
S315080158604CD0FA78BB781343DBB21A46F021786834
S31508015870FFF772FBFF23FB753BF048FA02463B69CB
S31508015880D31ADB0FDBB2002B10D0C8217868FFF7DB
S3150801589041FB0346FB7397F90F30002BECDA8022A4
S315080158A0C8217868FFF758FB0023FB75F82178684B
S315080158B0FFF730FB034603F00F03FB75FB7D042B53
S315080158C002D00E2B0CD013E0BB8A0133BB823B8876
S315080158D0002B0FD0BA8A3B889A420BD1FB7D0EE08A
S315080158E0BB7D0133BB75BB7D032B05D1FB7D06E073
S315080158F0FB7D04E000BFABE700BFA9E7FB7D1846C7
S315080159001837BD4680BD000080B584B000AF786009
S315080159100023FB73786800F0FDFD786800F012FE3D
S3150801592003463B733B7B032B2ED801A252F823F087
S315080159304D59010841590108695901086559010874
S31508015940BF4B13221A700023FB731DE0BC4B1B7857
S3150801595003F0F003102B02D0B94B11221A70002361
S31508015960FB7311E00123FB73B54B1B7803F0F003BE
S31508015970102B08D13BF0CAF90346C833B14A136064
S31508015980AF4B20221A7000BF0023BB73BB7B0F2BC2
S315080159901BD8BA7B7B681E3253F82230002B10D0F5
S315080159A0BA7B7B681E3253F82210BA7B7B681E329B
S315080159B053F822301B680C331B6808469847034680
S315080159C0FB72BB7B0133BB73E0E79D4B1B78A02BB6
S315080159D000F02381A02B00F32F81902B00F01F816B
S315080159E0902B00F32981802B00F0FE80802B00F399
S315080159F02381512B00F0EA80512B00F31D81402BA6
S31508015A006ADC112BC0F21881113B2F2B00F214818D
S31508015A1001A252F823F000BFDF5A0108235C0108EE
S31508015A20235C0108395C0108395C0108395C010805
S31508015A30395C0108395C0108395C0108395C0108DF
S31508015A40395C0108395C0108395C0108395C0108CF
S31508015A50395C01082F5B0108395C0108395C0108CA
S31508015A60395C0108395C0108395C0108395C0108AF
S31508015A70395C0108395C0108395C0108395C01089F
S31508015A80395C0108395C0108395C0108395C01088F
S31508015A90395C01084B5B0108395C0108395C01086E
S31508015AA0395C0108395C0108395C0108395C01086F
S31508015AB0395C0108395C0108395C0108395C01085F
S31508015AC0395C0108395C0108395C0108395C01084F
S31508015AD0395C01085D5B0108502B5FD0ACE0786842
S31508015AE0FFF784FA00237B737B7B0F2B1BD87A7B0A
S31508015AF07B681E3253F82230002B10D07A7B7B68E4
S31508015B001E3253F822107A7B7B681E3253F82230F4
S31508015B101B6808331B68084698470346FB727B7B5C
S31508015B2001337B73E0E7464B12221A7084E03BF09F
S31508015B30EDF80246434B1B68D31ADB43DB0FDBB296
S31508015B40002B70D03E4B30221A700122E82178686A
S31508015B50FFF702FA3A4B40221A706DE0E82178689D
S31508015B60FFF7D8F9034603F00103002B0CBF012305
S31508015B700023DBB2002B58D0D8217868FFF7CAF981
S31508015B80034643F008033B733B7B1A46D8217868E2
S31508015B90FFF7E2F92A4B50221A7046E0C8217868C5
S31508015BA0FFF7B8F9034603F04003002B14BF01239E
S31508015BB00023DBB2002B3AD0214B51221A703BF05D
S31508015BC0A5F8034614331F4A136030E03BF09EF8EC
S31508015BD002461C4B1B68D31ADB43DB0FDBB2002BD7
S31508015BE027D0174B80221A70FB7B00220021786888
S31508015BF000F020F90346FB72FB7A002B09D0FB7AE9
S31508015C00D22B18D0104AFB7A13700D4BA0221A70AA
S31508015C1011E00B4B90221A700DE000BF0CE000BF9B
S31508015C200AE000BF08E000BF06E000BF04E000BFCD
S31508015C3002E000BF00E000BF00BF1037BD4680BDCF
S31508015C403D100020401000203C10002080B586B091
S31508015C5000AF7860084611461A460346FB700B46A4
S31508015C60BB7013467B7000237B6100233B617B6815
S31508015C700021184600F0C0FB78617B69002B01D131
S31508015C80D6233AE07B691B68002B01D1D72334E080
S31508015C907B697A789A717868BB78F978002200F07E
S31508015CA05FFC0346FB73FB7B002B01D1D42324E065
S31508015CB07B68FA7B1146184600F09EFB38613B6902
S31508015CC0002B01D1D62318E03B697A789A71FB7BC0
S31508015CD000220021786800F0E3FA0346BB73BB7B18
S31508015CE0002B09D07B68FA7B1146184600F0D0FCD8
S31508015CF00023FB73BB7B00E0002318461837BD461B
S31508015D0080BD90B585B000AF7860084611461A4641
S31508015D100346FB700B46BB7013467B700023FB736F
S31508015D20FA787B681E3253F82200FA787B681E32AD
S31508015D3053F822301B6804331C6897F820307A78A8
S31508015D40B978A0470346BB73BB7BE02B1CD1BB7854
S31508015D50002B08D10122E8217868FFF7FDF86620B3
S31508015D603AF0E0FF22E0BA787B681E3253F8220047
S31508015D70BA787B681E3253F822301B6814331B68C5
S31508015D807A781146984711E0BB7B0D2B09D1FB7B2D
S31508015D90022B06D864203AF0C5FFFB7B0133FB735F
S31508015DA0BEE7BB7B002B01D0BB7B3FE0FA787B6863
S31508015DB01E3253F82200FA787B681E3253F82230D5
S31508015DC01B681C6897F820307A78B978A04703468B
S31508015DD0BB73BB7B0D2B09D1FB7B022B06D8642039
S31508015DE03AF0A0FFFB7B0133FB7399E7BB7B002BE2
S31508015DF01BD0BB78002B08D10122E8217868FFF770
S31508015E00ABF866203AF08EFF0FE0BA787B681E324F
S31508015E1053F82200BA787B681E3253F822301B6881
S31508015E2014331B687A7811469847BB7B1846143792
S31508015E30BD4690BD80B590B002AF78600846114660
S31508015E401A460346FB700B46BB7013467B7000234C
S31508015E5087F8363007F10C033B630023FB62002306
S31508015E60BB6200233B7208237B72BB7A6FF3000384
S31508015E70BB72BB7A6FF34103BB72BB7A0F2262F323
S31508015E808703BB727868F9F7F8FF78627B6A1B6843
S31508015E901B680021786A9847F862FB6A002B01D1D2
S31508015EA0D6235CE1FB6A1B68BB62FB6A07F1080241
S31508015EB01A60FB6A7A789A7107F10C030093122328
S31508015EC000220021786800F04EF9034687F836303B
S31508015ED0FB6ABA6A1A6097F83630002B02D097F82F
S31508015EE036303CE13B6B1A7A5B7A1B0213437B849F
S31508015EF03B6B9A7ADB7A1B0213433B843B6B1B7918
S31508015F00FB773B6B5B79BB77002387F8373097F8CC
S31508015F1037300F2B00F2818097F837207B681E32C5
S31508015F2053F82230002B6ED097F837207B681E3243
S31508015F3053F8221097F837207B681E3253F822301F
S31508015F401B6810331B68084698470346002B14BF85
S31508015F5001230023DBB2002B57D197F837207B6842
S31508015F601E3253F8220097F837207B681E3253F801
S31508015F7022301B6820331B68BA7F114698470346AF
S31508015F80002B2BD097F837207B681E3253F8220056
S31508015F9097F837207B681E3253F822301B6818336E
S31508015FA01B683A8C798C98470346002B14D197F8CD
S31508015FB037207B681E3253F8220097F837207B6812
S31508015FC01E3253F822301B681C331B68FA7F1146B0
S31508015FD098470346002B01D0012300E00023002B3C
S31508015FE014D0B878FA7897F837107B780093034677
S31508015FF07868FFF786FE034687F8363097F8363015
S31508016000D12B09D102E000BF00E000BF97F8373075
S31508016010013387F837307AE700BF97F837300F2B07
S3150801602002D897F836309AE0002387F8373097F880
S3150801603037300F2B00F2888097F837207B681E329D
S3150801604053F82230002B74D097F837207B681E321C
S3150801605053F8221097F837207B681E3253F82230FE
S315080160601B6810331B68084698470346002B14BF64
S3150801607001230023DBB2002B5DD197F837207B681B
S315080160801E3253F8220097F837207B681E3253F8E0
S3150801609022301B6820331B68BA7F1146984703468E
S315080160A0002B2BD097F837207B681E3253F8220035
S315080160B097F837207B681E3253F822301B6818334D
S315080160C01B683A8C798C98470346002B14D197F8AC
S315080160D037207B681E3253F8220097F837207B68F1
S315080160E01E3253F822301B681C331B68FA7F11468F
S315080160F098470346002B01D0012300E00023002B1B
S315080161001BD1B878FA7897F837107B78009303464D
S315080161107868FFF7F6FD034687F8363097F8363084
S31508016120D12B0BD097F83630D92B07D097F83630C4
S3150801613015E000BF02E000BF00E000BF97F8373066
S31508016140013387F8373072E77B78BA78F978786857
S31508016150FFF77CFD034687F8363097F83630184640
S315080161603837BD4680BD80B58AB008AF7860084625
S3150801617011461A460346FB700B46BB7013463B8015
S31508016180BA78F978002307933B6906933B88059308
S315080161903B8804930023039301230293002301936D
S315080161A00623009380237868FEF7F3FF0346184613
S315080161B00837BD4680BD80B58AB008AF7860084605
S315080161C011461A460346FB700B46BB7013463B80C5
S315080161D0BA78F978002307937B6906933B88059378
S315080161E03B88049300230393022302933B7C019388
S315080161F00623009380237868FEF7CBFF03461846EB
S315080162000837BD4680BD80B59EB008AF78600846A0
S3150801621011461A460346FB700B46BB7013467B7044
S31508016220402387F8573007F10C033B65BA78F978AC
S3150801623007F10C0301937B78009309237868FFF72C
S31508016240BAFF034687F84F3097F84F30002B02D034
S3150801625097F84F3020E03B6D9A78DB781B021343A1
S31508016260A7F84C30BA78F9783B6E079307F10C0317
S31508016270069340230593B7F84C3004930023039300
S31508016280022302937B78019306230093802378687F
S31508016290FEF77FFF034600BF18465837BD4680BD47
S315080162A080B58CB008AF7860084611461A46034691
S315080162B0FB700B46BB7013467B70BA78F9780023DE
S315080162C007930023069300230593002304930023D1
S315080162D00393002302937B780193052300930023FC
S315080162E07868FEF756FF0346FB734FF496703AF04B
S315080162F019FDFB7B18461037BD4680BD80B58AB0AF
S3150801630008AF7860084611461A460346FB700B46E5
S31508016310BB7013467B70BA78F9780023079300237C
S315080163200693002305930023049300230393002374
S3150801633002937B7801930923009300237868FEF77B
S3150801634028FF034618460837BD4680BD80B483B08A
S3150801635000AF78607B6818460C37BD465DF8047B4C
S315080163607047000080B483B000AF7860044A7B6848
S315080163701A607B6818460C37BD465DF8047B704782
S315080163804CBC060880B582B000AF78607B681846B9
S31508016390FFF7E8FF174A7B681A607B680022DA7103
S315080163A00021786800F090F97B6800221A737B68EF
S315080163B01A1D7B689A607B6800221A717B6808221D
S315080163C05A717A6893796FF3000393717A689379AE
S315080163D06FF3410393717A6893790F2161F3870308
S315080163E09371786800F0A1F97B6818460837BD46AD
S315080163F080BD00BF38BC060880B584B000AF7860A0
S315080164000B46FB70FB78002B02D17B68083314E03E
S31508016410FB781946786800F0A1F90346FB73FB7B04
S31508016420002B08D07B6803F10801FA7B1346DB00D1
S315080164309B1A0B4400E0002300BF18461037BD46DF
S3150801644080BD000080B586B000AFF8607B600B4662
S31508016450FB721346BB72FEF751FDFB7A43F002034A
S31508016460DBB2FB7507F117014FF0FF3301220B4829
S3150801647041F0F8F8BB7A9AB24FF0FF3379680748CA
S3150801648041F0F0F8BB7A7A6813447B60FEF72AFD7F
S315080164907B6818461837BD4680BD00BF74C4012005
S315080164A080B483B000AF03463960FB7100BF0C3777
S315080164B0BD465DF8047B704780B584B000AFF860CF
S315080164C07B600B46FB721346BB72FEF717FD07F19D
S315080164D00B014FF0FF3301220D4841F0C3F8BB7A97
S315080164E01A46002178684DF0C1FCBB7A9AB24FF082
S315080164F0FF337968064841F0F1F9BB7A7A681344A3
S315080165007B60FEF7EFFC7B6818461037BD4680BDF9
S3150801651074C4012080B584B000AF78600023FB7392
S31508016520FEF73CFD0346BB73BB7B002B04D17868A1
S3150801653000F037F90346FB73FB7B18461037BD4657
S3150801654080BD000080B483B000AF7860034B1B7830
S3150801655018460C37BD465DF8047B70474410002089
S3150801656080B584B000AF7860084611461A460346DE
S31508016570FB700B46BB7013467B70FB783B733B7B0A
S3150801658023F07F03DBB2002B02D17B78072B01D9DD
S31508016590002379E0BB78002B05D07B68DB79072BD4
S315080165A001D1002370E00021786800F0D7F803468E
S315080165B0FB73FB7B002B01D1002365E03B7B002BA2
S315080165C024D1BB78002B0FD0FA7B79681346DB0000
S315080165D09B1A0B440C3341221A707B68DB79013311
S315080165E0DAB27B68DA7108E0FA7B79681346DB0070
S315080165F09B1A0B440C3301221A70FA7B79681346ED
S31508016600DB009B1A0B440C331B783DE000233B72DD
S315080166103B7BC3F30203DAB23B7A62F3C5033B72EF
S31508016620BB78002B13D03B7A43F040033B727B685F
S31508016630DB790133DAB27B68DA717B68DB7903F0DF
S315080166400703DAB23B7A62F302033B720BE03B7A49
S315080166506FF386133B727B7803F00703DAB23B7A52
S3150801666062F302033B72FA7B79681346DB009B1AD5
S315080166700B440C333A7A1A70FA7B79681346DB00B5
S315080166809B1A0B440C331B7818461037BD4680BD40
S3150801669080B584B000AF78600B46FB70FB78412B60
S315080166A003D1786800F041F80BE0FB781946786861
S315080166B000F054F80346FB73FB7B1946786800F033
S315080166C093F81037BD4680BD80B483B000AF7860BB
S315080166D00B46FB70FA7879681346DB009B1A0B4464
S315080166E00C3300221A70FA7879681346DB009B1A74
S315080166F00B440D3301221A70FA7879681346DB00C8
S315080167009B1A0B440E3300221A70FA787B68191DFE
S3150801671078681346DB009B1A03440833196000BFE7
S315080167200C37BD465DF8047B704780B584B000AF71
S3150801673078600123FB73FB7B0F2B08D8FB7B19467B
S315080167407868FFF7C1FFFB7B0133FB73F3E77B68CF
S315080167500022DA7100BF1037BD4680BD80B485B00E
S3150801676000AF78600B46FB700123FB73FB7B0F2B95
S3150801677010D8FA7B79681346DB009B1A0B440C3355
S315080167801B78FA789A4201D1FB7B04E0FB7B013343
S31508016790FB73EBE7002318461437BD465DF8047B07
S315080167A0704780B584B000AF78600023FB73C821B9
S315080167B07868FEF7AFFB0346BB73BB7B03F0200388
S315080167C0002B06D0786800F057F8FB7B43F02003CE
S315080167D0FB73FB7B1A46C8217868FEF7BDFBFB7B7A
S315080167E018461037BD4680BD80B584B000AF7860C5
S315080167F00B46FB70FB78002B3AD0FA78796813467A
S31508016800DB009B1A0B440C331B783B733B7B03F071
S315080168104003DBB2002B25D00123FB73FB7B1A4611
S31508016820397B786800F098F80346FB73FB7B002BED
S3150801683014BF01230023DBB2002B05D0FB7B1946CD
S315080168407868FFF7D1FFE9E77B68DB793A7BC2F322
S315080168500202D2B2934205D17B68DB79013BDAB2F7
S315080168607B68DA71FB7819467868FFF72DFF00E037
S3150801687000BF1037BD4680BD80B584B000AF7860D3
S31508016880F8217868FEF746FB0346FB73FB7B23F08A
S315080168903F03FB73FB7BC02B4AD0C02B55DC802BF7
S315080168A006D0802B51DC002B46D0402B20D04CE063
S315080168B0D8217868FEF72EFB034603F00203002B66
S315080168C00CBF01230023DBB2002B08D0C922D82133
S315080168D07868FEF741FB1F4B02221A7035E0CB227E
S315080168E0D8217868FEF738FB1A4B03221A702CE078
S315080168F0D8217868FEF70EFB034603F00203002B46
S315080169000CBF01230023DBB2002B08D0CB22D821F0
S315080169107868FEF721FB0F4B03221A7015E0C9228E
S31508016920D8217868FEF718FB0A4B02221A700CE088
S31508016930084B01221A7008E0D122D8217868FEF79F
S315080169400BFB044B00221A7000BF00BF1037BD466F
S3150801695080BD00BF4410002080B485B000AF7860C8
S3150801696039701346FB70FB78002B04D0FB780F2B8C
S3150801697001D8FB7800E00123FB73FB7B0F2B16D8AC
S31508016980FA7B79681346DB009B1A0B4408331B799B
S31508016990C3F3C203DAB23B78C3F30203DBB29A420A
S315080169A001D1FB7B04E0FB7B0133FB73E5E70023A5
S315080169B018461437BD465DF8047B704780B485B028
S315080169C000AFF860B9607A60FB681B68002B01D1DB
S315080169D0002331E0FB681B79002B22D07B681B88DA
S315080169E0002B1ED0BB681A68FB681B68F9684979D1
S315080169F00846F9680979411A0B4412781A70FB6836
S31508016A001B79013BDAB2FB681A717B681B88013B6B
S31508016A109AB27B681A80BB681B685A1CBB681A60E5
S31508016A20D8E7FB681B79002B01D0002304E0FB683B
S31508016A305A79FB681A71012318461437BD465DF861
S31508016A40047B704780B584B000AF78603EF0BCFA2D
S31508016A5003460B4AA2FB03231B0DBB607B68BA687E
S31508016A6002FB03F30A3BFB6000BFFB685A1EFA6090
S31508016A70002BFAD100BF00BF1037BD4680BD00BF4D
S31508016A8083DE1B4380B582B000AF0346FB80FB88DB
S31508016A9018463AF047F900BF0837BD4680BD80B5AC
S31508016AA000AF0A20FFF7CEFF00BF80BD80B584B0D6
S31508016AB000AFF8607B600B46FB7213463B81FB7A9D
S31508016AC0082B78D801A252F823F000BFB76B01084A
S31508016AD0F16A0108196B0108376B0108596B01083E
S31508016AE07B6B01088F6B01088F6B0108A16B01088D
S31508016AF00022102132483BF0FDFE0220FFF7C2FFBB
S31508016B00012210212E483BF0F5FE01224FF40041E7
S31508016B102C483BF0EFFE4EE03B89002B05D10022C5
S31508016B20202127483BF0E6FE45E0012220212448A2
S31508016B303BF0E0FE3FE03B89002B06D101224FF4F2
S31508016B40004120483BF0D6FE35E000224FF40041D3
S31508016B501C483BF0CFFE2EE03B89002B05D10022D5
S31508016B60102117483BF0C6FE04E001221021144803
S31508016B703BF0C0FEFFF793FF1DE0134B186807F1C2
S31508016B8008014FF47A73012240F06CFD13E00E4BB5
S31508016B9018683A894FF47A73796840F063FD0AE018
S31508016BA0094B1B683A897968184641F04BF9012067
S31508016BB03AF0B8F800BF012318461037BD4680BD24
S31508016BC000040240000002404810002080B582B04F
S31508016BD000AF78600A4A7B68136001224FF40041CE
S31508016BE008483BF087FE0A203AF09CF8064A07490E
S31508016BF0074801F098F900BF0837BD4680BD00BFB8
S31508016C004810002000000240AD6A0108300000204B
S31508016C1014C2012080B588B002AFF8600846114653
S31508016C201A4603467B810B463B811346FB807B89CB
S31508016C3007337B8111E03B6A1B783A89798900938E
S31508016C400223F86801F006FA3B6A01333B62FB88C6
S31508016C50083BFB807B8908337B81FB88072BEAD8B5
S31508016C60FB88002B1CD03B6A1B78FB757B89073B8D
S31508016C707B81FB7D03F00103002B05D03A897B89D3
S31508016C801946F86801F0D3F97B8901337B81FB88C2
S31508016C90013BFB80FB7D5B08FB75FB88002BE8D17C
S31508016CA000BF1837BD4680BD80B588B002AFF86011
S31508016CB0084611461A4603467B810B463B81134615
S31508016CC0FB80FB88FB82FB8A0733FB82FB8ADB0896
S31508016CD0FB82F8883A8979893B8C00930346F868E0
S31508016CE000F01FF80346002B17D012E0F8883A89FE
S31508016CF079897B6A00930346F868FFF78BFFFB8A5D
S31508016D007A6A13447B623B8901333B813B8C013BA5
S31508016D103B843B8C002BE9D100E000BF1837BD4608
S31508016D2080BD90B488B000AFF860084611461A468F
S31508016D3003467B810B463B811346FB803C893B8D91
S31508016D4023449CB22346013B9CB2FB68DA8FFB685D
S31508016D50B3F84230FA83BB833B897B8323463B8363
S31508016D60BA8B7B8B9A420DD3FA8B3B8B9A4201D80D
S31508016D70012314E07A8B3B8B9A4201D901230EE059
S31508016D8000230CE0FA8B3B8B9A4207D87A8B3B8B14
S31508016D909A4201D9012302E0002300E00023002BD7
S31508016DA001D1002331E07C89FB8823449CB2234628
S31508016DB0013B9CB2FB689A8FFB68B3F84030FA82B4
S31508016DC0BB827B897B8223463B82BA8A7B8A9A422B
S31508016DD00DD3FA8A3B8A9A4201D8012314E07A8AAA
S31508016DE03B8A9A4201D901230EE000230CE0FA8A74
S31508016DF03B8A9A4207D87A8A3B8A9A4201D9012361
S31508016E0002E0002300E0002300BF18462037BD46F4
S31508016E1090BC704790B585B000AFF860B96013466D
S31508016E20FB71BB689C68FB799AB200230121F8685B
S31508016E30A047034618461437BD4690BD90B585B0A0
S31508016E4000AFF860B9601346FB71BB689C68FB79B3
S31508016E509AB200230321F868A04700BF1437BD463C
S31508016E6090BD90B583B000AF786039603B689C6887
S31508016E700023002204217868A04700BF0C37BD46CD
S31508016E8090BD90B583B000AF786039603B689C6867
S31508016E900023012204217868A04700BF0C37BD46AC
S31508016EA090BD90B585B000AFF860B9601346FB7127
S31508016EB0BB689C68FB799AB200230221F868A0474F
S31508016EC000BF1437BD4690BD90B585B000AFF860D8
S31508016ED0B9601346FB71BB689C68FB799AB20023BB
S31508016EE00521F868A047034618461437BD4690BDE4
S31508016EF080B586B000AFF860B9607A600023FB758B
S31508016F007B681B78BB75FB7D002B10D1BB7DFF2BE6
S31508016F100AD0BB7D1A46B968F868FFF7D5FF03465C
S31508016F20002B60D1002364E00123FB755BE0BB7D88
S31508016F30FF2B0AD1BB7D1A46B968F868FFF7C4FF6B
S31508016F400346002B4DD1002353E0BB7DFE2B4ED0CB
S31508016F50BB7DEF2B45D8BB7DDF2B09D9BB7D03F064
S31508016F600F03DBB21A46B968F868FFF79AFF38E0EB
S31508016F70BB7DCF2B09D9BB7D03F00F03DBB21A46C4
S31508016F80B968F868FFF75AFF2BE0BB7DBF2B1CD900
S31508016F90B968F868FFF765FFBB7D03F00F03BB759A
S31508016FA0BB7D1B01BB75BB7D0233BB75BB7D9BB22C
S31508016FB01846FFF767FDB968F868FFF762FFBB7DFA
S31508016FC09BB21846FFF75EFD0BE0BB7DBD2B08D8CB
S31508016FD097F91630002B04DBBB7D9BB21846FFF7E9
S31508016FE051FD0023FB757B6801337B6088E700BF91
S31508016FF0012318461837BD4680BD000090B587B0F5
S3150801700000AFF860B9603B601346FB800023FB8242
S315080170103B685A1C3A601B787B757B7D3B753B7DCB
S3150801702003F00F033B757B7D1B097B753A7DFB8A54
S31508017030591CF9821946104B9A5C104B5A547A7DA1
S31508017040FB8A591CF98219460B4B9A5C0B4B5A540D
S31508017050FB88013BFB80FB88002BD9D1BB689C6868
S31508017060074B1A88054B0821F868A04701231846DB
S315080170701C37BD4690BD00BF000000204C10002003
S3150801708058BC060890B587B000AFF860B9603B6098
S315080170901346FB710023FB753B685A1C3A601B7843
S315080170A0BB75BB7D7B757B7D03F00F037B75BB7D54
S315080170B01B09BB757A7DFB7D591CF97519460F4B62
S315080170C09A5C0F4B5A54BA7DFB7D591CF9751946C2
S315080170D00A4B9A5C0A4B5A54FB79013BFB71FB79C3
S315080170E0002BD9D1BB689C68054B80220621F8681C
S315080170F0A047012318461C37BD4690BD1000002045
S315080171004C14002080B485B000AFF8607B600B4654
S31508017110FB721346BB72FB7A062B11D801A252F8F1
S3150801712023F000BF4171010841710108417101084D
S315080171304171010841710108417101084171010854
S31508017140012318461437BD465DF8047B704700BF16
S3150801715080B586B000AFF860B9601346FB71BB68AD
S315080171605B681B7AFB75BB685B681B88DBB2FA7DBB
S3150801717012FB03F3FB75FA7DFB791344FB75134A7E
S31508017180B968F868FFF7B4FEFB7D1A46B968F8686E
S31508017190FFF79AFEFB7D0133DBB21A46B968F86838
S315080171A0FFF792FE0022B968F868FFF77AFE5C22BB
S315080171B0B968F868FFF788FE0122B968F868FFF729
S315080171C070FE00BF1837BD4680BD00BFDCBC06088F
S315080171D080B586B000AFF860B9601346FB71BB682D
S315080171E05B681B7AFB75BB685B681B88DBB2FA7D3B
S315080171F012FB03F3FB75FA7DFB791344FB75134AFE
S31508017200B968F868FFF774FEFB7D1A46B968F8682D
S31508017210FFF75AFEFB7D0833DBB21A46B968F868F0
S31508017220FFF752FE0022B968F868FFF73AFE5C22BA
S31508017230B968F868FFF748FE0122B968F868FFF7E8
S3150801724030FE00BF1837BD4680BD00BFDCBC06084E
S3150801725080B58CB000AFF860B9603B601346FB712E
S31508017260FB790A3B0C2B00F2C08001A252F823F0ED
S31508017270A5720108EB730108EB730108EB730108AA
S31508017280EB73010889730108CF730108DD730108DF
S31508017290EB730108EB730108EB730108BB72010874
S315080172A0237301080222B968F868FFF7B3FD544A47
S315080172B0B968F868FFF71CFE97E0BB685B687B61F5
S315080172C07B69DB68BB627B695B897B827B8A9B08FE
S315080172D07B82002387F82F301BE097F82F301A4658
S315080172E0B968F868FFF734FF7B8ADAB2BB6AB9680E
S315080172F0F868FFF7C7FE0022B968F868FFF79EFD30
S315080173007B8ABA6A1344BB6297F82F30013387F830
S315080173102F3097F82F309AB27B691B889A42DCD3B3
S3150801732063E0BB685B68FB61FB69DB683B62FB6921
S315080173305B897B837B8B5B007B83002387F8273004
S315080173401AE097F827301A46B968F868FFF740FF38
S315080173507A8B3B6AB968F868FFF750FE0022B9686C
S31508017360F868FFF76BFD7B8B3A6A13443B6297F823
S315080173702730083387F8273097F827309AB2FB6900
S315080173801B889A42DDD330E00122B968F868FFF715
S3150801739055FD0022B968F868FFF783FDC122B9686F
S315080173A0F868FFF791FD0122B968F868FFF779FDDA
S315080173B03B681B785B08DBB21A46B968F868FFF7C1
S315080173C083FD0022B968F868FFF738FD0DE00D4A1C
S315080173D0B968F868FFF78CFD01230DE00A4AB96818
S315080173E0F868FFF785FD012306E0FA793B68B96875
S315080173F0F86801F0A9F8034618463037BD4680BD3E
S315080174005CBC0608ECBC0608F8BC060880B483B068
S3150801741000AF78600B46FB70FB787A6813447B6093
S315080174207B681B7818460C37BD465DF8047B7047A8
S3150801743080B485B000AF78600B46FB70FB787A683C
S3150801744013447B607B681B78FB817B6801337B6017
S31508017450FB891B02FB817B681B789AB2FB89134463
S31508017460FB81FB8918461437BD465DF8047B7047D6
S3150801747080B582B000AF786000217868FFF7C6FF53
S31508017480034618460837BD4680BD80B582B000AFB1
S3150801749078607868FFF7ECFF0346022B0AD0022BC7
S315080174A00ADC002B02D0012B02D005E0062304E0FA
S315080174B0032302E0062300E0032318460837BD46E6
S315080174C080BD80B582B000AF786005217868FFF786
S315080174D09DFF034618460837BD4680BD80B582B074
S315080174E000AF786006217868FFF7A2FF03461846C1
S315080174F00837BD4680BD80B582B000AF78600821E7
S315080175007868FFF795FF034618460837BD4680BDDC
S3150801751080B582B000AF78600A217868FFF776FFF8
S31508017520034618460837BD4680BD80B582B000AF10
S3150801753078600B217868FFF769FF03461846083714
S31508017540BD4680BD80B582B000AF78600C217868F1
S31508017550FFF75CFF03465BB218460837BD4680BD98
S3150801756080B582B000AF78600D217868FFF74EFFCD
S3150801757003465BB218460837BD4680BD80B582B062
S3150801758000AF78600E217868FFF740FF03465BB2CB
S3150801759018460837BD4680BD80B582B000AF786011
S315080175A00F217868FFF732FF03465BB218460837A2
S315080175B0BD4680BD80B582B000AF7860102178687D
S315080175C0FFF724FF03465BB218460837BD4680BD60
S315080175D080B582B000AF786039607868FFF755FFEB
S315080175E003461A463B68134418460837BD4680BD0C
S315080175F080B584B000AF786039607B689B681846AF
S31508017600FFF736FF0346002B01D0022B1BD13B683F
S315080176101A787B68DA773B685A787B6883F8202082
S315080176203B6803331B785AB27B681A773B68043385
S315080176301B785AB27B685A773B6805331B785AB26E
S315080176407B689A7734E03B681B78FB7397F90F30B0
S3150801765003F00F035AB27B689A777B6893F91E3059
S31508017660DBB2023BDBB25AB27B689A77FB7B1B091A
S31508017670FB7397F90F207B685A773B685B78FB7336
S31508017680FB7B03F00F03DAB27B6883F82020FB7BD0
S315080176901B09FB737B68FA7BDA773B689B78FB737C
S315080176A0FB7B1B09FB7397F90F207B681A7700BFD1
S315080176B000BF1037BD4680BD80B483B000AF786087
S315080176C07B6800221A777B680022DA777B680022BA
S315080176D083F820207B6800225A777B6800229A77F4
S315080176E000BF0C37BD465DF8047B704780B586B090
S315080176F000AF78600B46FB707B689B687B617B6893
S315080177009B681846FFF7B4FE03463B747B689B6883
S315080177101846FFF7BAFE0346FB73FF237B743B7CCF
S31508017720012B01D10F237B747B689B681846FFF7F1
S31508017730EFFE0346FB747B689B681846FFF7F5FE68
S315080177400346BB737B689B681846FFF7D4FE03465E
S31508017750BB81FB78602B09D9BB89002B06D0BB8975
S315080177607A6913447B616123FB7416E07B689B6825
S315080177701846FFF7B3FE0346BB81FB78402B09D9B0
S31508017780BB89002B06D0BB897A6913447B614123E7
S31508017790FB7402E07B6911337B61FA78BB7B9A4201
S315080177A004D97868FFF788FF002332E0FB7CBB74B5
S315080177B0BA7CBB7B9A4228D87B691B78FF2B03D1FD
S315080177C07B6901337B6117E0BA7CFB789A4205D164
S315080177D079697868FFF70CFF7B691AE07B690233E0
S315080177E01A787B7C1340DBB21A467B6913447B61AA
S315080177F0FB7B7A6913447B61BA7CBB7B9A4203D0D3
S31508017800BB7C0133BB74D7E700BF7868FFF754FF29
S31508017810002318461837BD4680BD80B58CB002AF27
S31508017820F860084611461A4603467B810B463B819A
S315080178301346FB71FB791946F868FFF757FFB861DC
S31508017840BB69002B01D1002379E0FB689B68B96904
S315080178501846FFF7BDFE7862FB68DB7FFB75FB68A0
S3150801786093F82030BB75FB6893F91D309AB27B8972
S3150801787013447B81FB6893F91E309BB23A89D31A6C
S315080178803B813B89013B3B81BB7D9BB23A89D31A3C
S315080178909BB201339AB2FB7D98B2BB7D9BB27989C3
S315080178A000930346F868FFF73CFA0346002B03D119
S315080178B0FB6893F91C3042E0FB7D0733FB75FB7DC2
S315080178C0DB08FB753B89FB83BB7D9BB2FA8BD31A1D
S315080178D0FB83FB8B0133FB83002387F8223026E0E9
S315080178E07B893B84002387F8233013E07B6A1B7866
S315080178F0FA8B398C00930023F86800F0ABFB7B6A9E
S3150801790001337B623B8C08333B8497F82330013380
S3150801791087F8233097F82320FB7D9A42E6D3FB8B21
S315080179200133FB8397F82230013387F8223097F821
S315080179302220BB7D9A42D3D3FB6893F91C301846A3
S315080179402837BD4680BD80B586B000AFF8607B603C
S315080179500B467B8113463B810023FB82FB685B6AEE
S31508017960F868984703461A463B8913443B8117E052
S315080179707B681B783A897989F868FFF74EFF0346D1
S315080179807B7597F915309AB27B8913447B8197F9F0
S3150801799015309AB2FB8A1344FB827B6801337B60FC
S315080179A07B681B78002BE3D1FB8A18461837BD463E
S315080179B080BD80B584B000AF78607B689B68002B7A
S315080179C06BD07B6893F82830002B14D17B689B68B1
S315080179D01846FFF776FD03465AB27B6883F82920D5
S315080179E07B689B681846FFF7ADFD03461A467B6818
S315080179F083F82A202DE07B6893F82830012B14D1CF
S31508017A007B689B681846FFF7C7FD03461A467B68DD
S31508017A1083F829207B689B681846FFF7CBFD034648
S31508017A201A467B6883F82A2013E07B689B68184608
S31508017A30FFF796FD03461A467B6883F829207B687B
S31508017A409B681846FFF79AFD03461A467B6883F832
S31508017A502A207B6893F929301AB27B6893F92A3070
S31508017A601BB2D31A1BB2FB817B6893F82B30402BD0
S31508017A700DD0FB89DBB2FB817B6893F82B309BB277
S31508017A80FA8912FB03F3FB81FB899B09FB81FB89BD
S31508017A90DAB27B6883F82C2000E000BF1037BD46B8
S31508017AA080BD80B582B000AF78607B68002283F81C
S31508017AB028207868FFF77DFF00BF0837BD4680BDDF
S31508017AC080B582B000AF78607B68012283F82820F0
S31508017AD07868FFF76EFF00BF0837BD4680BD80B4E2
S31508017AE083B000AF7860002318460C37BD465DF8B1
S31508017AF0047B704780B483B000AF78607B68044A22
S31508017B005A6200BF0C37BD465DF8047B704700BF5B
S31508017B10DF7A010880B485B000AF78607B6893F995
S31508017B202930FB81FB890133FB81FB891846143710
S31508017B30BD465DF8047B704780B483B000AF7860BA
S31508017B407B68044A5A6200BF0C37BD465DF8047B60
S31508017B50704700BF157B010880B584B000AF786017
S31508017B6039600023FB813B681B787B737B7B002B89
S31508017B700FD07B7B19467868FFF7B8FD7B6893F9C8
S31508017B801C309AB2FB891344FB813B6801333B6085
S31508017B90E9E700BFFB8918461037BD4680BD80B5A9
S31508017BA082B000AF786039607B689B683A689A4210
S31508017BB008D07B683A689A607868FFF7FAFE7868B1
S31508017BC0FFF798FF00BF0837BD4680BD90B585B061
S31508017BD000AFF860B9603B601346FB71BB681C686F
S31508017BE0FA793B68B968F868A04703461846143716
S31508017BF0BD4690BD80B584B000AF786039607B68BA
S31508017C009B6B0220984700230A2239687868FFF798
S31508017C10DDFF0346FB737B689B6B032098477B68F4
S31508017C209B6B00209847FB7B18461037BD4680BDE5
S31508017C3080B582B000AF786039607B689B6B0220A3
S31508017C4098477B689B6B0120984700231422396863
S31508017C507868FFF7BBFF7B683C3317223968786879
S31508017C60FFF7B4FF7B689B6B0020984700BF083776
S31508017C70BD4680BD80B584B000AF786039607B6849
S31508017C809B6B022098477B689B6B012098470023D2
S31508017C90152239687868FFF799FF0346FB73FB7B62
S31508017CA0002B06D07B683C33172239687868FFF7C2
S31508017CB08DFF7B689B6B00209847FB7B1846103726
S31508017CC0BD4680BD80B584B000AF786039607B68F9
S31508017CD09B6B022098477B689B6B01209847002382
S31508017CE0162239687868FFF771FF0346FB73FB7B39
S31508017CF0002B06D07B683C33172239687868FFF772
S31508017D0065FF7B689B6B00209847FB7B18461037FD
S31508017D10BD4680BD80B584B000AFF860B960134632
S31508017D20FB71FB1D0F22B968F868FFF74FFF034681
S31508017D3018461037BD4680BD80B586B000AFF860DD
S31508017D40B96011461A460B46FB801346BB80FB6891
S31508017D502E337B617B69FA881A807B69BA885A80D7
S31508017D607B693222B968F868FFF730FF00BF183718
S31508017D70BD4680BD80B586B000AFF860B9601146D2
S31508017D801A460B46FB801346BB80FB682E337B6184
S31508017D907B69FA881A807B69BA885A807B6997F861
S31508017DA020205A717B6997F824201A717B693B2236
S31508017DB0B968F868FFF70AFF00BF1837BD4680BDE6
S31508017DC080B584B000AF7860396007F10E034622AA
S31508017DD039687868FFF7FAFEFB8918461037BD46F9
S31508017DE080BD80B584B000AF7860396007F10E03B5
S31508017DF0472239687868FFF7E9FEFB891846103784
S31508017E00BD4680BD80B582B000AF78603960002379
S31508017E10482239687868FFF7D9FE03469BB21846A7
S31508017E200837BD4680BD80B582B000AF78607B68F3
S31508017E305B6819467868FFF7C3FF03461A467B68ED
S31508017E401A807B685B6819467868FFF7CAFF03469C
S31508017E501A467B685A807B685B6819467868FFF71B
S31508017E60D1FF0346DAB27B68DA747B6859687B68A6
S31508017E703C3317227868FFF7A9FE00BF0837BD46CD
S31508017E8080BD000080B582B000AF78607B680022B3
S31508017E909A607B680022DA607B6800225A747B68E4
S31508017EA001221A747B6822229A747B6800229A61DD
S31508017EB00121786800F0EBF87868FFF71BFE7B680C
S31508017EC0012283F828207B68002283F829207B6811
S31508017ED0002283F82A207B68402283F82B207B68BE
S31508017EE0002283F82C207B68024A9A6300BF083770
S31508017EF0BD4680BD218C010880B582B000AF78608F
S31508017F007B685B6819467868FFF774FE0346002BA1
S31508017F1001D1002303E07868FFF785FF012318469E
S31508017F200837BD4680BD80B584B000AFF860B9603A
S31508017F307A60F868FFF7A6FFFB68BA685A60FB68BB
S31508017F405B687A689A60F868FFF7D6FF03461846B1
S31508017F501037BD4680BD80B582B000AF78607B68BA
S31508017F605B6819467868FFF763FE00BF0837BD46A8
S31508017F7080BD80B582B000AF78607B689B69002BB5
S31508017F8003D07B689B69786898477B685B68194664
S31508017F907868FFF76FFE034618460837BD4680BD69
S31508017FA080B582B000AF78607B689B69002B03D0EF
S31508017FB07B689B69786898477B685B681946786827
S31508017FC0FFF780FE034618460837BD4680BD80B5D3
S31508017FD082B000AF78600B46FB707B685B68FA7805
S31508017FE019467868FFF796FE034618460837BD46D0
S31508017FF080BD80B582B000AF78607B685968002380
S3150801800010227868FFF7E2FD00BF0837BD4680BD3C
S3150801801080B582B000AF78607B6859680023112269
S315080180207868FFF7D3FD00BF0837BD4680BD80B528
S3150801803082B000AF78600B467B8013463B807B6835
S3150801804059683B887A887868FFF776FE00BF083753
S31508018050BD4680BD80B586B002AFF86008461146B8
S315080180601A4603467B810B463B811346FB71FB6827
S31508018070596838897A893B7E0193FB7900930346CF
S31508018080F868FFF777FE00BF1037BD4680BD80B49C
S3150801809083B000AF78600B46FB707B68FA7883F88B
S315080180A0342000BF0C37BD465DF8047B704780B4A9
S315080180B085B000AF78607B68DB7CFB73FB7B282B84
S315080180C001D1FF2306E07B68DB7C022B01D1032368
S315080180D000E0012318461437BD465DF8047B704756
S315080180E080B582B000AF78607B68DB7C302B08D125
S315080180F07B68FF2283F834207B68FF2283F83520CA
S3150801810007E07868FFF7D3FF034619467868FFF753
S31508018110BEFF00BF0837BD4680BD80B483B000AF3F
S3150801812078607B6800229A807B681A887B68DA8087
S315080181307B68DB88013B9AB27B68DA807B68002220
S315080181401A7200BF0C37BD465DF8047B704790B4C0
S3150801815082B000AF78607B689A887B681B88134475
S315080181609AB27B689A807B689A887B685B889A4210
S3150801817001D3002318E07B681B7A0133DAB27B68E6
S315080181801A727B68DC887B681B8823449CB27B68EF
S315080181905B889C4204D37B685C882346013B9CB27E
S315080181A07B682246DA80012318460837BD4690BC0B
S315080181B0704780B485B000AF78600B467B80134664
S315080181C03B807B68DB887A889A4294BF0123002327
S315080181D0DBB2FB737B689B883A889A422CBF0123E2
S315080181E00023DBB2BB737A883B889A428CBF012392
S315080181F00023DBB27B73FB7B3B73FA7BBB7B1340B0
S31508018200FB73BA7B7B7B1340BB737A7B3B7B134047
S315080182107B73FA7BBB7B1343FB73FA7B7B7B134331
S31508018220FB73FB7B03F00103DBB218461437BD462B
S315080182305DF8047B704780B483B000AF786039601D
S315080182403B6800221A807B689A883B685A807B685B
S315080182505A893B689A803B689B88013B9AB23B687E
S315080182609A807B68DA883B68DA8000BF0C37BD469E
S315080182705DF8047B7047000080B584B000AF786074
S3150801828039603B685B88FB81FB89BB813B685B790D
S31508018290032B13D801A252F823F000BFBD820108AF
S315080182A0AD820108BD820108B5820108BB89083380
S315080182B0BB8103E0FB89083BFB8100BFBA89FB89C7
S315080182C019467868FFF775FF034618461037BD4605
S315080182D080BD00BF80B485B000AF78607B68DB687D
S315080182E0FB60FB68BB607B685B891A46BB68134405
S315080182F0BB607B685B891A46BB681344BB60FB6835
S315080183005A1CFA6000221A70FA68BB689A42F6D1BA
S3150801831000BF00BF1437BD465DF8047B7047B0B493
S3150801832087B000AFF860084611461A4603467B81B6
S315080183300B463B811346FB71FB68DB687B61FB6877
S315080183409B883A89D31A3B81FB685C89A3089CB24E
S315080183503B89DBB29BB214FB03F39CB222467B69D1
S3150801836013447B617C89A3089CB222467B6913442A
S315080183707B617C8904F003039CB263009CB297F885
S315080183802830002B0DD103252A46234602FA03F38A
S31508018390DDB2EB43DDB27B691B782B40DAB27B6930
S315080183A01A70FB7903F00303FB71FB7922469340AC
S315080183B0FB717B691A78FB791343DAB27B691A7008
S315080183C000BF1C37BD46B0BC704780B586B002AF4A
S315080183D0F860B9601346FB71BB685A88FB689B88CD
S315080183E09A4218D3BB685A88FB68DB889A4214D824
S315080183F0BB681A88FB685B899A4210D2BB681988E0
S31508018400BB685A88BB689879FB7900930346F86874
S31508018410FFF785FF04E000BF02E000BF00E000BFF0
S315080184201037BD4680BD000090B583B000AF7860B7
S3150801843039603B681C7963B2002B04DA002239687B
S315080184407868FFF7C2FF3B685B79032B26D801A240
S3150801845052F823F0658401087384010881840108B0
S315080184608F8401083B681B8801339AB23B681A80DE
S3150801847014E03B685B8801339AB23B685A800DE089
S315080184803B681B88013B9AB23B681A8006E03B6849
S315080184905B88013B9AB23B685A8000BF6300DCB235
S315080184A0002CC8D100BF00BF0C37BD4690BD00BF28
S315080184B090B583B000AF786039603B681C7924F0C9
S315080184C03F03DAB23B689A713B689B799B09DAB23A
S315080184D03B689A71012239687868FFF776FF3B682D
S315080184E05B79032B26D801A252F823F0FD840108F3
S315080184F00B85010819850108278501083B681B8832
S3150801850001339AB23B681A8014E03B685B880133F1
S315080185109AB23B685A800DE03B681B88013B9AB2C8
S315080185203B681A8006E03B685B88013B9AB23B6868
S315080185305A8000BFA300DCB2002CC0D100BF00BF27
S315080185400C37BD4690BD00BF80B586B000AFF86058
S31508018550B9603B601346FB71BB685B687B61FB795D
S315080185600A3B3E2B00F2D38001A252F823F000BF4A
S315080185700F8701080F8701080F8701080F87010870
S315080185800F8701080F8701080F8701080F87010860
S315080185900F8701080F870108A7860108B786010812
S315080185A0D1860108EB8601080F8701080F870108A4
S315080185B00F8701080F8701080F8701080F87010830
S315080185C00F8701080F8701080F8701080F87010820
S315080185D00F8701080F8701080F8701080F87010810
S315080185E00F8701080F8701080F8701080F87010800
S315080185F00F8701080F8701089B86010891860108E4
S315080186000F8701080F8701080F8701080F870108DF
S31508018610858601080F8701080F8701080F8701085A
S315080186200F8701080F8701080F8701080F870108BF
S315080186300F8701086D8601080F8701080F87010852
S315080186400F8701080F8701080F8701080F8701089F
S315080186500F8701080F8701080F8701080F8701088F
S31508018660F5860108FF8601080987010839687869CE
S31508018670FFF702FE0346002B48D039687869FFF7F1
S31508018680D3FE43E0002239687869FFF79EFE3EE093
S3150801869039687869FFF70CFF39E00122396878698A
S315080186A0FFF793FE33E07B691846FFF736FD7869D5
S315080186B0FFF710FE2BE07B691846FFF748FD0346D6
S315080186C0002B01D1002323E07869FFF703FE1EE0A2
S315080186D07B691846FFF73BFD0346002B01D10023B2
S315080186E016E07869FFF7F6FD11E039687869FFF752
S315080186F0A2FD0CE07B695A893B681A8007E07B6911
S315080187005A883B681A8002E0022301E000BF012370
S3150801871018461837BD4680BD80B588B002AFF860E7
S31508018720084611461A4603467B810B463B8113468A
S31508018730FB80FF23FB750DE03A897989FB7D009360
S315080187400023F868FFF786FCFB88083BFB807B89DA
S3150801875008337B81FB88072BEED8FB88002B15D0C5
S31508018760FB8883F00703FB80FB880133FB80FA7DD6
S31508018770FB8803F0070302FA03F3FB753A89798943
S31508018780FB7D00930023F868FFF764FC00BF1837E8
S31508018790BD4680BD80B588B002AFF860084611466F
S315080187A01A4603467B810B463B811346FB80FF2312
S315080187B0FB750DE03A897989FB7D00930123F868F9
S315080187C0FFF748FCFB88083BFB803B8908333B8164
S315080187D0FB88072BEED8FB88002B15D0FB8883F086
S315080187E00703FB80FB880133FB80FA7DFB8803F0D6
S315080187F0070302FA03F3FB753A897989FB7D00932E
S315080188000123F868FFF726FC00BF1837BD4680BD6F
S3150801881080B588B002AFF860084611461A46034685
S315080188207B810B463B811346FB807B89FB82F8885B
S315080188303A8979893B8C00930346F868FEF771FA01
S315080188400346002B26D0FB883A897989F868FFF711
S3150801885063FF3B8C3A897989F868FFF79BFF7A8928
S31508018860FB8813447B817B89013B7B813B8C3A895D
S315080188707989F868FFF78EFF3A893B8C13443B8167
S315080188803B89013B3B81FB883A89F98AF868FFF7FE
S3150801889043FF00E000BF1837BD4680BD80B584B0F0
S315080188A000AFF860084611461A4603467B810B4617
S315080188B03B811346FB80FB883A897989F868FFF77B
S315080188C02BFF3B8901333B813B8B013B3B833B8B35
S315080188D0002BF0D100BF00BF1037BD4680BD80B563
S315080188E086B002AFF860084611461A4603467B81F0
S315080188F00B463B811346FB80F8883A8979893B8B7D
S3150801890000930346F868FEF70CFA0346002B09D0D4
S31508018910F8883A8979893B8B00930346F868FFF70B
S31508018920BDFF00E000BF1037BD4680BD80B485B0ED
S3150801893000AFF860B9603B601346FB710023184627
S315080189401437BD465DF8047B7047000080B582B0D8
S3150801895000AF78607B685B68074A934207D1064B8C
S315080189605A687B685A607868FFF75DFA00E000BFCD
S315080189700837BD4680BD00BF3C00002080B582B0E7
S3150801898000AF78607B685B68094A934206D07B68CA
S315080189905B68074A53607B68054A5A60044B054A77
S315080189A01A607868FFF73FFA00BF0837BD4680BDF1
S315080189B03C000020B989010880B58AB000AFF8608B
S315080189C0B9603B601346FB71BB685B687B62FB79E8
S315080189D0173B302B64D801A252F823F0B18A01085B
